:020000040000FA
:10000000900A002029110000233D00007910000013
:1000100079100000791000007910000079100000BC
:10002000791000007910000079100000690F0000BD
:100030007910000079100000150F0000213C00002D
:10004000E9100000E9100000E9100000E9100000CC
:10005000E9100000E9100000E9100000E9100000BC
:10006000E9100000E9100000E9100000E9100000AC
:10007000E9100000E9100000E9100000E91000009C
:10008000E9100000E9100000E9100000E91000008C
:10009000E9100000E9100000E9100000E91000007C
:1000A000E9100000E9100000E9100000E91000006C
:1000B000E9100000E9100000E9100000E91000005C
:1000C000E9100000E9100000E9100000E91000004C
:1000D000E9100000E9100000E9100000E91000003C
:1000E000E9100000E9100000E9100000E91000002C
:1000F000E9100000E9100000E9100000E91000001C
:10010000E9100000E9100000E9100000E91000000B
:10011000E9100000E9100000E9100000E9100000FB
:10012000E9100000E9100000E9100000E9100000EB
:10013000E9100000E9100000E9100000E9100000DB
:10014000E9100000000000000000000000000000B6
:10015000000000000000000000000000000000009F
:10016000000000000000000000000000000000008F
:10017000000000000000000000000000000000007F
:10018000000000000000000000000000000000006F
:10019000000000000000000000000000000000005F
:1001A000000000000000000000000000000000004F
:1001B000000000000000000000000000000000003F
:1001C000000000000000000000000000000000002F
:1001D000000000000000000000000000000000001F
:1001E000000000000000000000000000000000000F
:1001F00000000000000000000000000000000000FF
:10020000DEE61E284CBBCE8F025B00003C000000E7
:10021000008000000100000000000000000000005D
:10022000FFFF02910000000000000000000000003D
:1002300000000000000000000000000053B94AB9AF
:10024000002908BF00281CBF4FF0FF314FF0FF30DE
:1002500000F070B9ADF1080C6DE904CE00F006F8BD
:10026000DDF804E0DDE9022304B070472DE9F04F2A
:10027000099E04468946002B40F083808A42154639
:1002800045D9B2FA82F24AB1C2F1200701FA02F36B
:100290009540944020FA07F747EA03094FEA154EC4
:1002A000230C1FFA85F8B9FBFEFC0EFB1C990CFB16
:1002B00008F143EA094399420AD9EB182CBF0120FF
:1002C0000020994202D9002800F01D810CF1FF3C6A
:1002D000591AA3B2B1FBFEF00EFB101100FB08F897
:1002E00043EA0144A04505D92C1902D2A04500F2E9
:1002F0000E810138A4EB080440EA0C4000271EB12F
:10030000D4400023C6E900433946BDE8F08F002AF7
:1003100051D0B2FA82F2002A40F0AF80491B4FEA76
:10032000154E1FFA85F80127230CB1FBFEFC0EFBCE
:100330001C1108FB0CF043EA014398420AD9EB1860
:100340002CBF01210021984202D9002900F0D7805A
:100350000CF1FF3C191AA3B2B1FBFEF00EFB101119
:1003600008FB00F843EA0144A04505D92C1902D244
:10037000A04500F2C1800138A4EB080440EA0C401B
:10038000BDE78B4208D9002E74D00027C6E90001D2
:1003900038463946BDE8F08FB3FA83F767B98B4228
:1003A000C0F0A480824240F2A1803846002EABD03B
:1003B000C6E90049A8E7FFDEC7F12005BB4002FA05
:1003C00007FC01FA07F4EA4020FA05F8E94000FAD0
:1003D00007FE1A4348EA04044FEA1248200C1FFAA9
:1003E00082F9B1FBF8FA08FB1A110AFB09FB40EA93
:1003F00001418B450AD951182CBF012300238B459D
:1004000002D9002B00F088800AF1FF3AA1EB0B0122
:10041000A4B2B1FBF8F008FB101100FB09F944EAA3
:100420000141894504D9511801D289457BD8013849
:1004300040EA0A40A1EB0901A0FB0C89494544466A
:100440004B4602D306D1C64504D20138B8EB0C04A2
:1004500069EB0203002E5DD0BEEB040261EB0301E9
:1004600001FA05F522FA07F3F94000271D43C6E912
:10047000005149E73746304646E7C2F12000954033
:1004800001FA02F721FA00F34FEA154E24FA00F1BF
:100490001FFA85F894403943B3FBFEF00F0C0EFBB6
:1004A000103300FB08FC47EA03439C4507D9EB18CF
:1004B0002CBF012700279C4500D98FB30138A3EB3F
:1004C0000C0389B2B3FBFEF70EFB173307FB08FCE6
:1004D00041EA03418C4504D9691801D28C4525D8DD
:1004E000013FA1EB0C0147EA00471DE7841A61EBCD
:1004F00003030120994659E702382C443CE7ACF14C
:10050000020C2B4426E7ACF1020C2B44E0E6023847
:100510002C44EFE63746F7E6AAF1020A114475E7E4
:1005200002382B44CBE70238114481E7023F2944CB
:10053000D7E700BF704700BF2DE9E04F2746A04630
:10054000A146A246A346A4462DED108B4FF0000510
:1005500045EC185B45EC195A45EC1A5A45EC1B5A08
:1005600045EC1C5A45EC1D5A45EC1E5A45EC1F5AE9
:10057000F1EE105A4FF66076C0F6FF763540E1EEA8
:10058000105A84F3008825462646A447BDEC108BFC
:10059000BDE8E08F0B6801330B60014B1B68184707
:1005A000D01300202DE9F04F85B00E9C9B46012C06
:1005B000B8BF0124012B0CBF3023202316468246EE
:1005C000884601250A270022DFF86C900293B6FBCB
:1005D000F9F301930AB9B1451CD8019B414603F1D7
:1005E0003000D04701220135019B013F09FB136612
:1005F0000A23012FB9FBF3F9E9D1414606F1300096
:10060000D047BBF1030F02D1641B002C0EDC05B0F8
:10061000BDE8F08FBC42E7DBBBF1020FE4D84146F6
:10062000029803920135D047039ADDE74146202026
:10063000D047013CE9E700BF00CA9A3B014B186074
:10064000704700BFD0130020002307B50246019376
:1006500003480B4601A903F060F803B05DF804FB02
:10066000950500004FF02002EFF3118382F311880B
:10067000BFF36F8F0121044AC2F8401583F311883C
:10068000BFF36F8F00207047009003500A2838B5E1
:100690000446074D04D1286843680D215B689847DC
:1006A00028684368E1B25B689847204638BD00BFC0
:1006B0000800002010B5044C204601F097F82046B1
:1006C000BDE81040FFF7BABF8D06000008B504482A
:1006D00001F0AEFA034B1860FFF7ECFF002008BDF5
:1006E000804700000800002008B5114B1A686AB165
:1006F0004FF05022D2F80423D10707D500220D482D
:100700001A608368597A09B903F0DAF90A4B1A6852
:100710006AB14FF05022D2F80423920707D5002285
:1007200001211A600348BDE8084003F0C9B908BDBB
:1007300000510050801400200451005000220D4B45
:10074000C3F840214FF02002EFF3118182F31188AA
:10075000BFF36F8F084AD3F804051368C01A20F05E
:100760007F400344136081F31188BFF36F8F02F061
:1007700027B800BF005001502400002070B5154874
:1007800001F056FA10B3436801211B689847002412
:1007900001264FF480334FF400120F4D3146C5F857
:1007A0000845C5F84065C5F804330C4B15201C609E
:1007B0000B4BC3F88021224600F0F6FB152000F019
:1007C000E3FB2046074B1E602E6070BD4FF0FF30EC
:1007D000FBE700BF55490000005001504051015057
:1007E00000E100E00850015070B5254CB0F1FF3F2A
:1007F00008BF20464FF02003EFF3118583F31188E3
:10080000BFF36F8F1F4BD3F804151F4B1B68CA1A19
:1008100022F07F4612021AD4421E22EAE272A2425B
:10082000A8BF2246701C1044A04294BF1818181983
:10083000411A21F07F41134A20F07F430229C2F878
:10084000403506D985F31188BFF36F8F70BD002244
:10085000E8E7D2F804350D49C31A23F07F435C1E44
:100860008C4205D94FF40012094BC3F80021E9E787
:10087000012B02BF023020F07F40C2F84005E1E7C3
:10088000FEFFFF000050015024000020FEFF7F000B
:1008900000E100E04FF02002EFF3118382F31188B2
:1008A000BFF36F8F064AD2F80405064A1268801A11
:1008B00020F07F4083F31188BFF36F8F704700BF34
:1008C000005001502400002008B543B2002B0CDB7F
:1008D000012200F01F018A405B091049203341F8D2
:1008E0002320BFF34F8FBFF36F8F830003F1A0432B
:1008F00003F540533128D3F8002806D0002A07DA40
:1009000002F00302023A012A02D8054AC3F800287D
:10091000002103F0D5F9002008BD00BF00E100E090
:100920000001008030B54FF440444CF2040585B01E
:100930004FF440412C4803F060F821682B4803F045
:100940005CF829682A4803F058F81022002168460C
:1009500003F07EFA236868460093029400F0D0FE0C
:10096000012000F0FDFE002000F0E6FE002000F077
:100970000BFF0121002000F025FF00F019FF2C687B
:100980001C4803F03AF80820FFF79EFF24F001040A
:10099000BFF34F8FBFF36F8F64086400204621467A
:1009A00022462346B7EE000AF7EE000AB7EE001A19
:1009B000F7EE001AB7EE002AF7EE002AB7EE003A7B
:1009C000F7EE003AB7EE004AF7EE004AB7EE005AEB
:1009D000F7EE005AB7EE006AF7EE006AB7EE007A5B
:1009E000F7EE007AFFF7A8FDD5480000EC480000BC
:1009F000014900001F4900002DE9F843704802F04A
:100A0000FCFF00216F4EDFF8D891DFF800826E4DB9
:100A100056F8044BCA0301F5C07349F82340404619
:100A200002F500434F1C02F0E8FF684B14F0100F72
:100A30006749684808BF194602F0DFFF14F0040F49
:100A400014BF72212D21284602F0D7FF14F0020FA7
:100A500014BF77212D21284602F0CFFF14F0010F9B
:100A600014BF78212D21284602F0C7FF14F4807F9F
:100A700014BF6C212D21284602F0BFFF564802F01A
:100A8000BCFF202F3946C3D1544B554AC3F3C43160
:100A9000C3F30E03C3F50043C3F34313C2F80015B9
:100AA000C2F80435D2F80015D2F804254D48520199
:100AB00002F0A3FF484802F0A0FF03F0B3F801469C
:100AC00010B1494802F099FF434802F096FF4748A9
:100AD00002F093FF0021464EDFF80491DFF83081E9
:100AE000394D56F8044B4A0301F5E07349F82340A9
:100AF000404602F500534F1C02F07FFF334B14F0C9
:100B0000100F3349334808BF194602F076FF14F03E
:100B1000040F14BF72212D21284602F06EFF14F03D
:100B2000020F14BF77212D21284602F066FF14F032
:100B3000010F14BF78212D21284602F05EFF14F426
:100B4000807F14BF6C212D21284602F056FF2248D9
:100B500002F053FF202F3946C3D10024204D1E48F8
:100B600002F04BFFC5F88044224802F046FF224FB6
:100B7000C5F8C044DFF89C80204DDFF89C906E796A
:100B80002A68002E14BF3B4643462146484602F0E1
:100B900034FF66B91A48013402F02FFF1A2C05F110
:100BA0000805ECD10C48BDE8F84302F026BF2879CF
:100BB000FFF78AFE08B11348EDE71348EBE700BFE3
:100BC000B147000024440000E94700009A470000B4
:100BD00091470000BE480000E54A0000E07F0000A9
:100BE00000300050EC47000032480000624800002E
:100BF0007445000098480000A6470000A444000087
:100C0000C1480000C8480000D0480000D447000098
:100C1000844800009E470000B448000010B500283A
:100C20004BD0002A49D0264B99423CD9541803F6A0
:100C30001D239C423AD803F0E1F80020BDE81040A3
:100C4000714672467346B7EE000AF7EE000AB7EE39
:100C5000001AF7EE001AB7EE002AF7EE002AB7EEF8
:100C6000003AF7EE003AB7EE004AF7EE004AB7EE68
:100C7000005AF7EE005AB7EE006AF7EE006AB7EED8
:100C8000007AF7EE007A8EF3008C10B4F1EE10CA01
:100C90004FF66074C0F6FF740CEA040CE1EE10CA63
:100CA00010BCF4467447074B994203D9064B5418BD
:100CB0009C42C0D94FF0FF30C0E76FF01500BDE790
:100CC0000302FF002F01FF003801FF002DE9F04F64
:100CD000834685B08946002951D00027DFF8B0A0AF
:100CE000DFF8B08001AE5AF8044B98E807005C4486
:100CF00086E807000C223146204603F058F80546E6
:100D000008B9002C3ED10137052FECD16FF00D054D
:100D1000284605B0B7EE000AF7EE000AB7EE001A53
:100D2000F7EE001AB7EE002AF7EE002AB7EE003A07
:100D3000F7EE003AB7EE004AF7EE004AB7EE005A77
:100D4000F7EE005AB7EE006AF7EE006AB7EE007AE7
:100D5000BDE8F04F714672467346F7EE007A8EF3A7
:100D6000008C10B4F1EE10CA4FF66074C0F6FF7438
:100D70000CEA040CE1EE10CA10BCF44674476FF0A4
:100D80001505C5E73C222146484603F037F8BFE782
:100D9000F4450000D4430000014801F07FBF00BFCC
:100DA0000846000008B530B143683BB1006801F067
:100DB0003DF9002008BD6FF4E040FBE70048F9E78B
:100DC000EA8FFFFF38B5044618B90B4B0B485B6838
:100DD0009847656855B115F00205206807D10146AE
:100DE000074801F083F825600023636038BD1422B2
:100DF000002103F02DF8F7E724140020464A0000F4
:100E00002800002010B5044618B9134B13485B683E
:100E100098476368BBB92368ABB94FF0FF322146EE
:100E20000F4801F037F808B923681BB90A4B0D4881
:100E30005B68984714220021206803F009F8636872
:100E400043F002036360206803F09AF8636843F09C
:100E50000103636010BD00BF24140020464A000057
:100E6000280000206C4A000008B558B1436863B1FF
:100E700000684FF0FF3101F067F8054B002818BFFC
:100E8000184608BD6FF4E040FBE70248F9E700BFF1
:100E9000E98FFFFFEA8FFFFF08B5064940231422C0
:100EA000054803F052F8BDE808400449044801F041
:100EB0002DBF00BF44000020280000202046000075
:100EC0001046000004488168406A884203D0034904
:100ED0004FF080520A6070473006002004ED00E0B9
:100EE000094A0A49936809685866996608494B682F
:100EF00043F080534B60002383F31188BFF36F8F5F
:100F00009368986E704700BF300600208C46000042
:100F100000ED00E012498A684FF028001044EFF31A
:100F2000098C80E8F01F202080F31188BFF36F8FB9
:100F30000C4F4FF000664A6A8A603E60506E002394
:100F4000536680F3118804B5104602F0F1FEBDE847
:100F5000044002F1280090E8F01F8CF309887047E4
:100F60003006002004ED00E01EF0040F0CBFEFF38C
:100F70000880EFF30980816911F8021C0229FFD073
:100F800001B502F0CAFE01BD43B2002B08DB01220D
:100F900000F01F0002FA00F0024A5B0942F8230049
:100FA000704700BF00E100E043B2002B01F10101F6
:100FB000A8BF03F160434FEA4111B8BF054BC9B266
:100FC000ABBF03F5614300F00F0083F80013195421
:100FD000704700BF14ED00E073B51E460A9B05463E
:100FE0000093099B8C1803F060F80B4AA4F12003CE
:100FF00023F0070322F001029A61069A1E605A60EC
:10100000079A9A60089ADA604FF08072DA61AB64EE
:1010100000236B6602B070BD153A0000F8B51E469D
:1010200005460C4617460023E1EE103A00F0D6F9CB
:101030000A4B3C4428469D6024F0070402F078FEE9
:10104000304684F30988002163B681F31188BFF329
:101050006F8F0022002302F0DDFC00BF300600206D
:10106000014910220A60704710ED00E0404080F313
:10107000118830BF704700BFEFF30880EFF309819C
:10108000724601B500F0D2F801BD00BF30BFFFF7D6
:10109000FDBF00BF114A08B5114B22F07F029A60D4
:1010A000BFF34F8FBFF36F8FD3F8882042F4A002B5
:1010B000C3F888200B4A536823F040435360BFF3C2
:1010C0004F8FBFF36F8F0023E1EE103A00F0F0FD79
:1010D00000F0F8FD00F050F900F032FE00000000D2
:1010E00000ED00E030EF00E001B572B60B4A106A87
:1010F00000281EBF0021116202F025FF62B6EFF347
:101100000580A0F110004FEAC0000549014409C95B
:101110009847BDE801400349084700003006002019
:1011200054410000C50E000002F07FFC202080F337
:10113000118808484FF40061401880F30988EFF3E4
:1011400014800221084380F31488BFF36F8FFFF7E8
:10115000A1FF0000D00B00200C4B9A6A9A6A9A6A91
:10116000920708D55A6B9A6A120604D518B19A6A82
:1011700022F080029A620020044B9A6A9A6A9A6A64
:101180009A6A42F0FF029A620870704700ED00E030
:101190000D4B9A6A9A6A9A6A920508D59A6B9A6A6E
:1011A000120404D518B19A6A22F400429A6200200F
:1011B000054B9A6A9A6AD20558BF9A6A9A6A42F4AB
:1011C0007F429A620870704700ED00E0074B0020F4
:1011D0009A6A9A6A9A6A9A6A9A6A9A6A9A6A9A6AEF
:1011E0006FEA02426FEA12429A62704700ED00E035
:1011F0000D4B9A695A695A69D0070FD45A699107F9
:101200000CD45A69520709D45A69100706D45A698E
:10121000D10603D45A69920658BF5A695A6942F0F6
:10122000FF025A61704700BFD0ED00E0F0B5414BBE
:101230008BB05B680025C3F3080385F31188BFF307
:101240006F8F02F07F44B4F17F4F1ED112F0010482
:101250001AD0560602F0080467D482F00402C2F3E2
:10126000800564B1EFF389860022033B8DF80720E7
:10127000042B4BD8DFE803F00B4C50414800EFF350
:101280008886F1E70E46EFE725462E46ECE7294B28
:10129000DA6A92073AD4DC6A14F0804408D0283322
:1012A0001B78EBB101200DF10701FFF755FF044654
:1012B0009DF8073093B92022314602A802F09EFD26
:1012C000099B6DB3C3F3080222B96FEA53236FEA97
:1012D0004323099302A9204602F01DFD0BB0F0BD87
:1012E000154B1B782BB101200DF10701FFF750FFC3
:1012F000DDE7124B1F88BFB217B1FFF767FFD6E7D4
:101300000F4B5C69002CD3D0FFF772FF0024CFE7AE
:101310000DF107010020C8E70DF107010020E5E706
:1013200023F4FF7323F00103D3E7002CAAD1064670
:10133000012599E700ED00E029ED00E02AED00E04D
:10134000D0ED00E0024A536943F010035361704747
:1013500000ED00E0BFF34F8F0549064BCA6802F469
:10136000E0621343CB60BFF34F8F00BFFDE700BFC8
:1013700000ED00E00400FA05002320210348C21814
:101380000133412B82F80013F9D1704700E100E0EE
:1013900038B505464FF02003EFF3118483F311882D
:1013A000BFF36F8F00F0E4FF0A4B9B68AB420BD199
:1013B000094B5A68C2F3080212B92046FFF790FDA4
:1013C0005A6842F080525A602046BDE8384002F028
:1013D000F2BD00BF3006002000ED00E010B50E4B5E
:1013E00088B002930D4B0E4C03930E4B0E4A0493A0
:1013F00002AB019301A82346012100F003F9002369
:1014000007930A4B0121E41A05A80593069400F0FE
:1014100003F908B010BD00BF00000020000000006C
:101420000000012006000100000000200000002054
:1014300010B50B680C7A23F01F0204F01F031A4347
:10144000CB68640923F01F03044943EA440343F0D3
:1014500001038860CA600B6110BD00BF90ED00E021
:101460002DE9F04F8046894614460027484D85B047
:101470004F4507DA58F827305E68C6B31F2E05D8E7
:101480006FF01504204605B0BDE8F08FF206F7D1E5
:10149000D3F800A01AF01F0FF2D1504602F072FCF0
:1014A000834606EB0A00013802F06CFC8345E7D165
:1014B0001BF1160FE4D0631E5B45E1DBC5F808B0F5
:1014C000E86858F82710C5F808B02E6920F01F000A
:1014D000D1E900321A44984246F01F0602F1FF3A61
:1014E00018D1564505D15FFA8BF002F029FC01377F
:1014F000BEE7C5F808B0EB6822F01F0203F01F0337
:101500001A43EA60E0B202F01BFC10F1160FB7D0EC
:10151000441CECE7C5F808B02A69013B23F01F031F
:1015200002F01F0213435645E0B22B61EBD002F0EC
:1015300007FC10F1160FA3D0C5F808B0EA689DF8B3
:101540000830013E62F304038DF808302B699DF8E2
:1015500008205B0863F347128DF8082058F827200D
:101560000130D2E900321344009323F01F031E44DC
:10157000A6EB0A06C4B226F01F060F2C03963FF610
:101580007FAF20466946FFF753FF0134AFE700BF46
:1015900090ED00E00522034B5A60BFF34F8FBFF37D
:1015A0006F8F704790ED00E0BFF35F8F0022014B1B
:1015B0005A60704790ED00E070B50E4D2E68102E09
:1015C00015D80024FFF7F0FF0B4B0C4A1A63A64214
:1015D00005D10B4B1E70FFF7DDFF002070BD696861
:1015E000204601EB0411FFF723FF0134EFE74FF032
:1015F000FF30F3E73446000090ED00E0AAFF44001E
:101600008C06002010B5034C2278FFF729FF2070CC
:1016100010BD00BF8C0600202DE9F74F254C8A46EF
:1016200080460027A1464FF0140B234D57451ADA88
:10163000D8F804300193002B36D0D8F800100846B3
:10164000009102F09FFBDDE90013064658180138AF
:1016500002F098FB8642194A08D014235F436FF0CA
:10166000150349F8073003B0BDE8F08F16F1160FE7
:101670002660F8D01378B342F5DD0BFB0793AE601C
:10168000AE60E868197B60F3040119732969187B5F
:10169000490861F347101873EB6823F01F03636078
:1016A0002B6923F01F0323610137143408F10C0860
:1016B000BCE700BF4405002090ED00E08C06002050
:1016C00070B50C4B0E461C780546234600210A4A8D
:1016D0000F2B0BDD094951F8040BFFF7A9FE224639
:1016E00031462846BDE87040FFF7BABE93601161ED
:1016F0000133EDE78C06002090ED00E0440500206A
:1017000082680C4B9A60036883F38888436883F38C
:101710008988027B02F00101EFF3948323F0030335
:10172000920748BF43F0020309B143F0010383F37A
:101730009488704700ED02E0084AD36848B123F46A
:1017400000531B041B0C43F0BF6343F40033D3600E
:1017500070479BB243F40053F5E700BF00ED00E093
:10176000084AD36840B19BB243F4804343F0BF635F
:1017700043F40033D360704723F480431B041B0CF5
:10178000F4E700BF00ED00E0084AD36840B19BB227
:1017900043F0080343F0BF6343F40033D360704762
:1017A00023F008031B041B0CF4E700BF00ED00E06E
:1017B000034AD2F88C3043F44063C2F88C3070474F
:1017C00000ED00E0084B1A6818B142F001021A60FF
:1017D000704722F001021A601A6811B142F0020249
:1017E000F5E722F00202F2E7D0ED00E0014B1860CD
:1017F000704700BFF4130020F0B54B79012B29D0BE
:10180000032B24D110268B79032B20D1CC792CB13A
:10181000012C1CD103689B681B79C3B10A7912B1F2
:10182000022A14D10E2247F6122705680B68AD680C
:10183000BB422D6862D029D8B3F5965F61D014D829
:10184000B3F5167F5FD007D8B3F5967F5ED06FF003
:10185000220052E00026D6E7B3F5966F59D0B3F5D3
:10186000166FF4D14FF41D233CE0B3F5615F53D004
:1018700004D8B3F5165FEAD1324B33E0B3F5964F97
:101880004CD0B3F5E14FE2D12F4B2BE0B3F5E13F64
:1018900046D012D84DF6C027BB4244D005D8B3F588
:1018A000164FD4D14FF41D031CE0B3F5614F3DD06A
:1018B000B3F5963FCBD1254B14E0B3F5E12F38D0EB
:1018C00008D8B3F5613F37D0214FBB42BFD14FF0AD
:1018D000806307E0B3F5612F31D01E4FBB42B6D114
:1018E0004FF08053C5F8243534438368224303C93D
:1018F000C5F86C2583E803000020F0BD4FF4000319
:10190000F0E7154BEEE74FF41C33EBE74FF4A03351
:10191000E8E74FF49E23E5E7104BE3E7104BE1E7E0
:101920004FF0EB73DEE74FF46503DBE74FF46B0337
:10193000D8E74FF0E863D5E74FF06C73D2E74FF08C
:101940007063CFE70050270000C0750000903A0197
:1019500090D0030040420F0000B0130000F03A00A6
:1019600000A04E00026870B59268184B14684FF0E2
:101970000052856803219A601D260022C3F8741264
:10198000C3F87022C4F80C651C26C4F814654FF027
:1019900000669E60C3F86C12C3F868221B23C4F86B
:1019A00008351A232946C4F81035FFF725FF58B922
:1019B0000823C4F800351D440123C4F81001C4F8FD
:1019C0003455C4F83835236070BD00BF00258450FD
:1019D0002DE9F04300261E4C85B054F8049C1D4FA1
:1019E00001ADB14503D8002005B0BDE8F083636ABE
:1019F00097E80700D3F8008085E807000C22294605
:101A0000404602F0D4F9A0B9B8F1000F11D0636AD2
:101A100021691B681A6991420BD19A69A1699142A7
:101A200007D8E169914204D962695B6932EA03032C
:101A300007D0236A4BB1404080F311884FF0040077
:101A400002DFE36801361C44CBE7626A1360F8E703
:101A50003C020000E0430000064B1868043B1B6892
:101A6000092B05D1013801288CBF002001207047C7
:101A7000002070473401FF00054B1868043B1B68C9
:101A8000092B03D1431E584258417047002070472C
:101A90003401FF004E4A08B5136843F00203136097
:101AA000FFF7DAFF30B14FF050230022C3F81421C2
:101AB000C3F81821FFF7E0FF30B10123454A136056
:101AC000A2F63822C2F87835434B1B68092B07D1A0
:101AD000424B1B68022B02BF0122414BC3F8782501
:101AE000FFF7CAFF10B10E223E4B1A60FFF7B4FF9A
:101AF00020B100223C4B1A6001225A600022D30020
:101B000003F57F03D3F80013013108D0D3F8001395
:101B10000132D3F80433B2F5807F0B60EFD1334B41
:101B2000DA69D1073BD5324B1946D3F80024012A94
:101B3000FBD1C3F80425D1F80034012BFBD12B4B8A
:101B4000DA69D20708D5DA69294922F00102DA6197
:101B5000D1F80024012AFBD11A6A01320AD11A6A8B
:101B600022F0FF0242F020021A62214AD2F8003429
:101B7000012BFBD100221E4BC3F80425D3F800240F
:101B8000012AFBD1BFF34F8F1A491B4BCA6802F4DD
:101B9000E0621343CB60BFF34F8F00BFFDE71B6ACA
:101BA0000133C0D0134BD3F88C2042F44062C3F809
:101BB0008C20D3F8882042F47002C3F88820BFF349
:101BC0004F8FBFF36F8F0D4B0D4A1A6008BD00BFDA
:101BD000D0ED00E0384A00503001FF003401FF0032
:101BE00000400050E4AE03500C4700500080FF005E
:101BF0000090035000ED00E00400FA0504140020FA
:101C00000090D00370B50026084B53F820400130F7
:101C100053F82050A54200D870BD236820465B6869
:101C2000984700B166600C34F4E700BF78460000C6
:101C3000104B70B505461E460F4C9C4204D10E4C0D
:101C4000B44209D1002412E062681AB12268126815
:101C5000AA420CD00C34F0E763680BB90C34EFE700
:101C600023682846196802F096F80028F6D1204625
:101C700070BD00BFC81400205014002008B50B4DE3
:101C80004FF02002EFF3118382F31188BFF36F8FBF
:101C900002F030FA012104460228D8BF084602F0BB
:101CA00039FA2C62FFF7E2F9EAE700BF30060020BC
:101CB0000248034A0021121A02F0CAB800000020AC
:101CC0009006002008B50648064A0749121A02F095
:101CD00095F8BDE80840054A0549064802F08EB867
:101CE000D01300202C150020F84A0000000000004E
:101CF000F84A000000000020012208B50B4B02202A
:101D00001A70FFF77FFF0A4A0A490B4801F075FE77
:101D10000320FFF777FF00F07DFC01F0A1FC074AEC
:101D2000137B23F00103137308BD00BF8D06002051
:101D300099470000B34A0000C04A0000C4050020D3
:101D400080B5374BA2B083F308880025E023354CDB
:101D5000012784F82230E57725766576A576E57645
:101D6000636A314E43F4E0236362636A43F4002301
:101D70006362A563FFF7E6FAFFF772F94FF0FF33EE
:101D8000A362E36207AB6C222946184602F060F8B2
:101D9000264C8DF82970A0602846FFF733FF38469F
:101DA000FFF730FF00F0E8FB214B66624FF48062E2
:101DB000CDE90473CDE902551E4BCDE900551E490E
:101DC000304600F00FFC737B23F0040213F01B0F6E
:101DD000727304D1B36913B9304600F019FA174B86
:101DE000012205930F23CDE903320023144DCDE9E1
:101DF000013300934FF4A072124B1349284600F0B0
:101E0000F1FB6B7BE56023F004036B730F4B4FF426
:101E10008062C4E906330849064B0348FFF7FEF821
:101E2000D013002000ED00E0C405002030060020A3
:101E3000E74A0000F91C000090060020EC4A000070
:101E4000580500207D1C0000900A00204806002054
:101E500070B50E4B0E4CA34201D3002070BDD3E9E8
:101E6000030141EA000212F003020BD19D685A619E
:101E7000AA4201D11C33EEE75E6901320E6059615E
:101E80000144F5E76FF01500E8E700BFC814002033
:101E9000C814002010B513460C464FF02002EFF393
:101EA000118182F31188BFF36F8F42695AB12260AA
:101EB00013684361836901338361002081F31188D2
:101EC000BFF36F8F0DE01BB923606FF00B00F5E7D8
:101ED0000246044800F0FAFA18B9034B9B685B69A4
:101EE000236010BD8E0600203006002070B5044629
:101EF0000D464FF02003EFF3118683F31188BFF3F3
:101F00006F8F02F0A5F880B100212A6881664261D6
:101F1000427BD20603D183690BB900F079F93146CF
:101F2000BDE87040074802F03BB82B6862691A6050
:101F30002B686361A369013BA36186F31188BFF33A
:101F40006F8F70BD8E060020F8B504460F464FF027
:101F50002003EFF3118583F31188BFF36F8FC268FD
:101F600030495AB180688E68B04215D0B7B985F350
:101F70001188BFF36F8F6FF00F000CE08B6893F93F
:101F80000E3023618B680132E260A36085F3118813
:101F9000BFF36F8F0020F8BD2369F2E790F90E3090
:101FA00096F90E109942A8BF194621EAE1719942AB
:101FB0002BDA00F09FFA06463B46224629461A488D
:101FC00000F084FA0028E6D04FF02003EFF31185EB
:101FD00083F31188BFF36F8F236821699C4207D078
:101FE00033B193F90E309942A8BF194621EAE17145
:101FF000A06890F90E30994209D16EB129460A487D
:1020000001F0CEFF6FF00A00C5E70026D4E700F02C
:1020100071FA0028F2D1F0E785F31188BFF36F8FD2
:10202000F0E700BF300600208E06002038B5836838
:102030000446002B3BD0214A926893423AD1DA7B86
:10204000013ADA73C368012B05D0013BC36000F08D
:10205000C3F8002038BD4FF02003EFF3118583F360
:102060001188BFF36F8F0169806890F90E30994233
:1020700001D000F03FFA204601F0EAFFA06080B1F5
:1020800090F90E20226100228266427BD20603D1A3
:1020900083690BB900F0BCF82946094801F080FFBC
:1020A000D5E7E06085F31188BFF36F8FCFE76FF05E
:1020B0001500CFE74FF0FF30CCE700BF300600201F
:1020C0008E06002010B5084C23685BB1FEF7E2FBDA
:1020D0002368064A184410610021BDE810401846E4
:1020E00002F018B810BD00BF6806002030060020BE
:1020F000F8B50D464FF02003EFF3118483F31188F8
:10210000BFF36F8F4FF4004140F2E7360027002203
:10211000E1FB0067094B30461A6139464FF47A7289
:102120000023FEF78BF8064B1860064B1D60FFF787
:10213000C9FF84F31188BFF36F8FF8BD300600200C
:1021400068060020640600204FF02003EFF31181A1
:1021500083F31188BFF36F8F044B9A68D37B013BE5
:10216000D37381F31188BFF36F8F7047300600205F
:10217000094B03F12802824205D19B688B4202D1B0
:102180004B7BDB0606D1D1E9003213605A60002395
:10219000C1E90033704700BF3006002038B50D4C50
:1021A000024604F1280001F01CFF054600B9E5686D
:1021B000A3684AB95A7BD20606D1AA6922B9DA893C
:1021C0007F2A01D9636238BD9D4201D0FFF77AFFB3
:1021D0006562F8E73006002010B54FF02003EFF3FA
:1021E000118483F31188BFF36F8F084B00209A6826
:1021F000D37B0133D373FFF7D1FF84F31188BFF38F
:102200006F8FBDE8104001F0E2BE00BF3006002035
:10221000F8B54FF02003EFF3118483F31188BFF377
:102220006F8F154A114651F8283F8B421DD0E3B1FC
:10223000D66A90F90E5093F90E70AF4210DD5A68CD
:10224000C0E9003210605860437B63F07F03437342
:102250000020FFF7A3FF84F31188BFF36F8FF8BD51
:10226000B34202D01B68002BE5D1D36A0160436002
:10227000D36A1860D062E7E730060020F8B504465C
:102280004FF02003EFF3118583F31188BFF36F8FB5
:1022900090F90D30002B03DA01461848FFF768FF6C
:1022A000174A02F12801D2E90A308B421FD0F3B15C
:1022B00094F90E6093F90E70B74213DD5968C4E9C2
:1022C00000310C605C60637B906863F07F03637334
:1022D000031B58425841FFF761FF85F31188BFF394
:1022E0006F8FF8BD984202D01B68002BE2D1C4E981
:1022F0000010D36A1C60D462E5E700BF58060020D6
:1023000030060020154A164938B50C689368A34278
:10231000144603D1BDE83840FFF7D4BE00250D6058
:1023200010490968B9B1D9897F2914D80E4993F9A0
:102330000E5009688D420EDB0C498B420BD0996917
:1023400049B91169814203DC1846FFF797FFE1E7BD
:10235000091A116138BD00232361FBE73006002014
:102360006006002068060020640600205805002052
:10237000036D70B5044603B1984704F1180001F0ED
:10238000A3FE4FF02003EFF3118583F31188BFF311
:102390006F8F204601F0FBFD0646D8B194F90D3051
:1023A000002B07DA21461248FFF7E2FE637B03F0B9
:1023B0007F0363730F4B9868021B50425041FFF735
:1023C000EDFE637B43F00803637385F31188BFF36D
:1023D0006F8F70BD637B9B07F3D52146A068FFF725
:1023E000C7FE637BA66023F002036373E9E700BFC7
:1023F000580600203006002038B504464FF0200370
:10240000EFF3118583F31188BFF36F8F90F90D30CF
:10241000002B07DA01460948FFF7AAFE637B03F0A9
:102420007F036373064B9868031B58425841FFF7BC
:10243000B5FE85F31188BFF36F8F38BD58060020B5
:102440003006002070B504460D461646FFF7D4FF4F
:10245000637B43F0020363737DB12B68A5609D42EB
:1024600029D043B394F90E2093F90E1091421CDD4C
:102470005A68C4E9003214605C60731C22D04FF4C7
:10248000004540F2E730002126EAE6764FF47A7202
:10249000C5FB06010023FDF7D1FE0B49421C04F1E8
:1024A0001800BDE8704000F049B969688B4202D05D
:1024B0001B68002BD8D16B68256063606B681C605B
:1024C0006C60DAE770BD00BFEF3F000010B50C464E
:1024D0001146064A9068064A10601A46FFF7B2FF96
:1024E0002046BDE81040FEF7FBBC00BF30060020D0
:1024F000600600202DE9F84304464FF02003EFF377
:10250000118983F31188BFF36F8F01F040FD4EB244
:10251000804660B3174D214605F128073846FFF77E
:1025200027FEAB6AA673BB422A4619D0C3B1E96A3B
:1025300093F90E00B0420EDD5A68C4E9003214600F
:102540005C600120FFF72AFE89F31188BFF36F8FCB
:102550004046BDE8F883994202D01B68002BE7D1C2
:10256000D36A27606360D36A1C60D462E9E7A6730C
:10257000EAE700BF300600200021044B084603F1C3
:102580002802C3E90A22FFF7B3BD00BF30060020CE
:10259000014B9868704700BF3006002010B54FF01F
:1025A0002002EFF3118482F31188BFF36F8F427B17
:1025B000510704D484F31188BFF36F8F10BD22F04C
:1025C000040112F01B0F417303D183690BB9FFF7AC
:1025D0001FFE2146BDE81040014801F0E1BC00BFEC
:1025E0008E06002030B587B00E9D044604950D9DE3
:1025F00003950C9D02950B9D01950A9D0095FEF794
:10260000EBFC034B9B6803B11B6E236607B030BD28
:10261000300600202DE9F04F284E294DB04687B0F6
:10262000B54205F1300410D3FFF78EFD4FF4004999
:1026300040F2E7360027224CDFF888A0444521D33A
:1026400007B0BDE8F04FFFF7C7BD54F8043C059351
:1026500054F8103C049354F8143C039354F8183C79
:10266000029354F81C3C019354F8203C009354E925
:102670000A2354E90C01FFF7B5FF54F8303CDD6440
:102680002546CDE7616A4B1C04D0256821B9284650
:10269000FFF784FF3034D1E7B346BC46E9FB01BC09
:1026A0004FF47A72002358466146FDF7C7FD514644
:1026B000421C05F1180000F041F8EBE7C8140020B7
:1026C000C8140020EF3F0000034B1B680BB9FEF756
:1026D000E1B80020704700BF6C060020036840B1DD
:1026E000074A5268904204D01BB19A6881680A4434
:1026F0009A60426813605A600023C0E90033704753
:10270000081400200B4B10B51C689C4208BF002425
:10271000FFF7DAFF54B1A368181A20EAE070064BFD
:102720001B6913B19842A8BF184610BD6FF0004056
:10273000F5E700BF081400203006002070B50446FD
:102740001646C1604FF02003EFF3118583F3118823
:10275000BFF36F8FFFF7B8FF012EACBF80190130B8
:10276000164BA0601A689A4201D05E6832B95A6866
:10277000236062605A6814605C600AE09068A16837
:10278000884215DD411A91605168C4E900210C604E
:1027900054601A689A4206D0944204D1FFF7B2FFFF
:1027A0000021FEF721F885F31188BFF36F8F70BD0C
:1027B000091A9642A160DAD01268D7E708140020FF
:1027C0002DE9F04B0446FFF79DFD4FF02003EFF39A
:1027D000118583F31188BFF36F8F214F214EB846C7
:1027E000DFF884903460D9F8004032684C45D7E96E
:1027F00000BC05D024B1A368934214DD9B1AA360EA
:1028000000241BEB02004CEBE271C8E900013460CC
:10281000FFF778FF2146FDF7E7FF85F31188BFF347
:102820006F8FBDE8F08B1BEB03004CEBE371D31A09
:1028300033600023C7E90001A3602046FFF74EFF85
:1028400085F31188BFF36F8FE36898474FF020033B
:10285000EFF3118583F31188BFF36F8FC3E700BFD8
:10286000000000206C0600200814002038B5074C3A
:10287000074DAC4201D3002038BD04F114032046BB
:10288000C4E9053300F0F3FE1C34F2E7C81400205D
:10289000C814002001F09BBA0A46002101F0D8BA02
:1028A00010B5114800F048F800B110BD0F4800F015
:1028B00043F80028F9D10E4C204600F03DF80028DE
:1028C000F3D10C4B0C481C6000F036F80146002890
:1028D000EBD100F02DF8044608B1204610BD00F001
:1028E00051F82046FAE700BF1C1400201014002005
:1028F00018140020201400201414002008B50848E3
:1029000000F024F8074800F021F8074800F01EF80E
:10291000064800F01BF8BDE8084000F00BB800BF07
:102920001C1400201014002018140020141400207F
:1029300000207047704700BF08B5034B02681B6852
:1029400010689847002008BD2C14002008B5034BE0
:1029500002685B6810689847002008BD2C140020AE
:102960000268024B10689B68184700BF2C140020B7
:1029700008B5034B0268DB6810689847002008BD63
:102980002C14002070B5094C094D2069AB6898479C
:1029900018B1084B08485B6898470021074AEB6864
:1029A00011602069BDE87040184700BF3C1400204A
:1029B0002C140020241400209046000070060020F3
:1029C000F8B51A4C1A4D0746AB6820699847E8B924
:1029D000184E33687FB93BB90120174A1749C2F82E
:1029E00000050A68002AFCD101333360EB682069D6
:1029F00098470020F8BD002BF8D0012B08D0013BF0
:102A000033602069EB6898470020F3E70C48F8BD75
:102A10000A4A1368002BFCD1074A6FF07E40C2F8C7
:102A2000003500F021F83368E9E700BF3C140020CE
:102A30002C140020700600200000845010198450CF
:102A4000E98FFFFF0020704700207047430503D542
:102A50004FF0FF32024B1A60024B1860704700BF04
:102A600008118450081A8450014B1860704700BF49
:102A7000041A845008B100F003B84FF47500704791
:102A80000246074803681342FCD021B1054B0648B3
:102A90001B680B600360054B00201A60704700BF85
:102AA000001A84500411845008118450081A84506C
:102AB00000F0A0B830B129B1002301440370013007
:102AC0008142FBD1704700BF2DE9F041ADF51A7D81
:102AD0000F4605920021144612A84FF408721E46B4
:102AE00001F0B6F9002308A819462822069301F040
:102AF000AFF9002F3CD0002E3AD0002C38D0042162
:102B000006A8FFF7C9FE08A82821FFF7C5FE08A8F8
:102B100000F032F878B14FF0FF3512A84FF4087189
:102B2000FFF7C8FF06A80421FFF7C4FF28460DF5EC
:102B30001A7DBDE8F08112AB0DF11C080390CDE9C0
:102B40000163024605AB08A9CDF8008006A800F095
:102B5000E9FC0028DFD13368A342DCD3D8F80010A9
:102B60000546083138462246FFF794FE3460D4E724
:102B70004FF0FF35DAE700BF1C2330B583B002A960
:102B800041F8043D044600F0B1F90546D8B9019B6F
:102B90001C2B1BD1D4E9003201210033E16118BFA5
:102BA00001230AB143F00203A26832B9E268AAB96C
:102BB000C4E908323BB90D4D09E0E26843F0040373
:102BC00062B9C4E90832284603B030BD084D20463A
:102BD0001C21FFF761FE284603B030BD00222846C5
:102BE00043F00803C4E9083203B030BD0E0CF00016
:102BF000370CF00010B50C4C236813B10B4B1B685D
:102C00006BB900F031F938B10138062896BF084B8E
:102C1000084853F8200010BD0122044B1A6001231C
:102C20000020236010BD00BF74060020780600203D
:102C3000B0460000FE8FFFFF10B5094C23681BB1A2
:102C400001230020236010BD00F07CF80028F7D09D
:102C50000138062896BF034B034853F8200010BDE7
:102C600074060020B0460000FE8FFFFFBFF34F8FB9
:102C70000549064BCA6802F4E0621343CB60BFF318
:102C80004F8F00BFFDE700BF00ED00E00400FA0534
:102C9000014B5B68184700BF24140020024BD0E9A9
:102CA0000012C3E90012704724140020704700BFCF
:102CB00010B5044620B1BFF35F8F0020206010BD27
:102CC0000348FFF7E5FFBFF35F8F0020206010BDD2
:102CD000F046000010B5044610B10023236010BD7B
:102CE0000248FFF7D5FF0023236010BDCC4600004B
:102CF00050B10122D0E8EF3FC0E8E12F0029F9D11F
:102D0000012BF7D0BFF35F8F0020704770B40B4BDF
:102D10000668C268D0E90154C3E90242C3E900650C
:102D2000D1E903020E68064BD1E90154C3E90065FD
:102D3000C3E902401A6170BC704700BF2C14002028
:102D40003C14002010B5FFF77DFE70B9FFF7A8FD19
:102D500080B9FFF735FE80B9114B1B681B0EF02BB5
:102D60000DD00624FFF770FE00E00324FFF7C6FD38
:102D7000204610BD0424204610BD0024F2E7094A75
:102D8000094B12689A4201D00724EBE70120FFF7B4
:102D900017FE0028F1D1054B04461860E8E700BF94
:102DA00028198450241A84500000E0200C1A845002
:102DB00030B5ADF5157D4FF4087200210CA801F077
:102DC00047F8002302A819462822019301F040F891
:102DD00002A8FFF7D1FE18B105200DF5157D30BD15
:102DE0001C4D4FF0FF312868FFF7BAFD0446F0B9DB
:102DF0000020FFF7E5FDB0B90CAA02A901A800F078
:102E0000D5FB04460120FFF7DBFDF0B92868FFF78A
:102E1000AFFD10B11048FFF73BFF2046002CDBD17F
:102E20000DF5157D30BD0D48FFF732FFE4E70C4886
:102E3000FFF72EFF012CDBD12868FFF799FD002852
:102E4000CAD00548FFF724FFC6E70648FFF720FF72
:102E5000DCE700BF201400202847000040470000A6
:102E6000104700006047000008B5FFF7EBFD18B100
:102E7000FFF744FD032008BDFFF712FD68B9FFF717
:102E80009FFD60B9154B1B681B0EF02B12D0FFF78E
:102E9000DBFDFFF733FD062008BD042008BDFFF76A
:102EA000D3FDFFF72BFDFFF783FF00280CBF0020A9
:102EB000052008BD0A4A0B4B12689A4205D0FFF75D
:102EC000C3FDFFF71BFD072008BD0120FFF778FDBC
:102ED0000028E4D1044B1860E5E700BF28198450AE
:102EE000241A84500000E0200C1A845018B111B14B
:102EF0000B681C2B01D0012070474FF47F033A4A26
:102F0000D3F8101C91425AD0D3F8102C013256D06D
:102F1000D3F8102C4FF47F030260D3F8141C334A0B
:102F200091425ED0D3F8142C01325AD0D3F8142C2D
:102F30004FF47F034260D3F8182C12F5947F4DD0E4
:102F4000D3F8182C013249D0D3F8182C4FF47F0352
:102F50008260D3F81C1C264A91423CD0D3F81C2C2A
:102F6000013238D0D3F81C2C4FF47F03C260D3F861
:102F7000002C70322DD0D3F8002C013229D0D3F898
:102F8000002C4FF47F030261D3F8042CAF321ED023
:102F9000D3F8042C01321AD0D3F8042C4FF47F0359
:102FA0004261D3F8081C134A91420BD0D3F8082C85
:102FB000013207D0D3F8083C83610020704740F607
:102FC000FC02A7E740F237338361002070475122AB
:102FD000E4E79022D5E742F60412C5E740F6D8624E
:102FE000B4E742F2D002A3E7FCF8FFFFD020FFFFD6
:102FF0000429FFFF37F3FFFFA8B32DE9F0414C1E72
:10300000B4F5047F2CD25BB352B34FF0000CC9006F
:10301000E646654664464F1E03F1FF380CE0AB42BE
:1030200016D08E4501D10CF1010CA84516D0013403
:10303000BC4205F1010518D8610950F8211004F0CF
:103040001F06F1401F2E18BF01F00101002CE6D130
:103050000025A8458E464FF0010CE8D16245E6D226
:103060000348BDE8F081024870470020BDE8F081C8
:10307000370CF1002DE9F04F8FB00D46DDE9194115
:103080008346002957D12969039100211C60189BB0
:103090001960002A00F02281814A824B11686A6A15
:1030A0001B689A4257D10A2955D19BF803300693E1
:1030B0000399042308467C4A0293A2FB000292086B
:1030C000CB0002EB420204F10800A1EB4202013BFB
:1030D000DFF8D091DFF800A2049000920593189BCE
:1030E000039C1C60002C00F0CC800026049F00F0A4
:1030F000A9FA00230793069BBBF1000F3AD0002DDD
:1031000034D053BB5B000693BBF1000F36D0002DCB
:1031100034D0E3B106A9284600F084FA002800F074
:103120007D81624B984212D0009000F08BFA00989B
:103130000FB0BDE8F08F4FF47F01D1F80C0C0130D7
:103140000CBF4FF40471D1F80C1C03919DE72B6A5E
:1031500073B95648E8E75648E6E706A9284600F05E
:1031600061FA68B1534B9842DED0069B082BC9D157
:103170005148D9E7082BFBD05B0006934F48D3E7B3
:103180002946069800F030FA0028EBD1069B082B60
:1031900000F00E81042B00F03181A3F10203B3FA99
:1031A00083F35B09019301231946454A136042F8F2
:1031B000843C434B19606B6AC9F80030D9F8002091
:1031C0006B6A9A42F5D14FF000084FF0FF30CAF811
:1031D0000080FFF73BFC3B4A3B4B40461A60FFF741
:1031E00043FC0A22019839492D4B08601A602A696C
:1031F000A8F15538A8FB02126B6A120903EB4303CE
:10320000DB0303FB02F3324A9B0913600123CAF874
:1032100000300699DBF800200B0243EA016322F03C
:103220007F421343CBF8003007A800F0CDF9002807
:1032300098D1284BA8FB04281A681433089253F835
:10324000102CB6EB980F099253F80C2C0A9253F8F5
:10325000082C0B9253F8042C0C921B680D9301D18F
:10326000009B9BB93846182208A9FFF713FB183CAE
:1032700018370136002C7FF43AAF049B002B40F046
:103280009A800023189A1360069B6FE71A46384607
:1032900008A9E41AFFF7FEFA009B1F44E9E700BF04
:1032A0003811845030118450ABAAAAAA310CF10015
:1032B000300CF100020CF100320CF100350CF10081
:1032C000C4118450FEFFFF0F001184500C11845074
:1032D000D8118450141184502C118450BBF1000F6C
:1032E0003FF44CAF002D3FF449AF01230EA941F844
:1032F000203DCBF80020284600F094F900287FF408
:1033000013AF2946069800F06FF900287FF40CAF40
:10331000069F082F00F0EB80042F00F0EA80A7F151
:103320000207B7FA87F77F0901221646734B7449E3
:103330001A6018460A60943B06606A6A1A60196847
:103340006A6A9142F8D14FF000086E4B4FF0FF309F
:10335000C3F80080FFF77AFB6B4B6C4A40461A605B
:10336000FFF782FB0A226A496A4B0F601A601A99BA
:103370002B6901296A6A00F0B1806749A1FB031338
:103380001B09012102EB4202D20303FB02F3634A51
:103390009B0913605B4B19600699DBF800200B0258
:1033A00043EA016322F07F421343CBF800307FE60B
:1033B00003230193F7E6039BB3F5047F3FF661AF68
:1033C000DDE9047C204623466E6904E001200133D8
:1033D0006345144615D85A0957F8222003F01F01F7
:1033E000CA401F2918BF02F00102002BEED0A242F2
:1033F000ECD101308642EAD149480BE00223019327
:10340000D1E64FF48063DDE90310AA69FFF7F4FD0C
:1034100000285DD00023189A1360A3E62946069879
:1034200000F0E2F800287FF47CAE069C082C51D016
:10343000042C51D0A4F10204B4FA84F464090123E9
:103440001E4619462D4A136042F8843C2B4B1960E6
:103450006B6AC9F80030D9F800206B6A9A42F5D13E
:1034600000274FF0FF30CAF80070FFF7EFFA264B45
:10347000264A38461A60FFF7F7FA0A222449254BF4
:103480000C601A602A6924496B6AA1FB021203EBE3
:1034900043031209DB0303FB02F3204A9B09136079
:1034A000CAF80060069BDBF800101A0242EA0363C8
:1034B00021F07F421A43130A03F47F03134323F0DE
:1034C0007F43CBF80030029B013B02937FF407AEB1
:1034D000002029E60324B2E70224B0E74FF47F037B
:1034E000D3F80C1C013106D0D3F80C3C45E7032778
:1034F0001AE7022718E7162343E700BFC4118450D8
:10350000401184502C11845000118450FEFFFF0F95
:103510000C11845038118450ABAAAAAAD811845037
:10352000360CF1002DE9F0431B4C85B00746DDE970
:103530000D56884620684FF0FF319146FFF710FA8C
:1035400028BB0020FFF73CFAE8B90023CDE900567C
:1035500002934A46414638460C9BFFF78BFD0546D1
:103560000120FFF72DFA50B92068FFF701FA10B1DA
:103570000A48FFF78DFB284605B0BDE8F0830848F0
:10358000FFF786FBF0E70748FFF782FBDDE7064819
:10359000FFF77EFBD5E700BF20140020284700007E
:1035A00060470000404700001047000010B50124AC
:1035B00086B005ABCDE901240093002204ABFFF7F0
:1035C00059FD06B010BD00BF08B501464FF480603C
:1035D000FFF750FA00230249024A0B60136008BD4E
:1035E000C81184502C1184500138072815D8DFE801
:1035F00000F0100C140814141404CB6800204B6263
:1036000070478B6800204B6270474B6800204B620C
:1036100070470B6800204B6270470148704700BF3D
:10362000310CF1000B6802E0082B0B6006D8026A2F
:1036300013424FEA4303F7D0002070470048704719
:10364000310CF10000230449044A0B604FF4806000
:103650001360FFF7FBB900BF2C118450C4118450D4
:1036600008B5FDF7C9F9BDE80840FDF75BB9FF23D0
:103670002DE9F04F4668C372324600234FF00C0923
:103680000789016806FB07FC90F80A8061449845A9
:1036900005DC002319468F4220DCBDE8F08FBCFB1F
:1036A000F2F509FB03FED0F80CA0202D0AEB0E0466
:1036B00004F1040BC4E901BB05D8C372920822F0DF
:1036C00003020133E3E715F11F0448BF05F13E048F
:1036D00064114AF80E1001EB8401EFE7C268056837
:1036E00002F1040CEC1845F803C0956801316560DF
:1036F000956833442C609460CDE70020704770B526
:103700000D4604464520A04729465220A047294699
:103710002346BDE87040522018472DE9F04F4FF086
:10372000000806460F461C464FF0FF3AC146454684
:103730008BB00292029B187810B90BB0BDE8F08FE5
:1037400045B9252800F04B813946B047029B01332B
:103750000293EFE764286DD019D839280AD83128A8
:103760005FD22D2800F0418130284BD0252807D189
:10377000394632E1582800F0BB80632800F02A81E6
:1037800039462520B047029B3946187825E1702834
:1037900000F0A48011D869284CD06C2805D1B8F16C
:1037A0006C0F2AD14FF04C08D0E76828E8D1B8F167
:1037B000680F22D14FF04808C8E7752872D018D892
:1037C0007328DDD154F8045BAB465B461BF8010B54
:1037D000002840F0FC80B9F1030F40F00C815D1B24
:1037E000AAEB0505002D49DD39462020B047013DF3
:1037F000F8E778287CD07A28C2D1B8F1000FBFD181
:103800008046A3E7BAF1000F0EDAB9F1000F00F01D
:10381000EF80A0F1300AB9F1000F08BF4FF00209A4
:1038200094E7BAF1000FF4DB0A2303FB0A0AAAF1BA
:10383000300AF0E7B8F17A0F02D154F8045B20E0C7
:10384000B8F16C0FF9D0B8F14C0FF6D1073424F071
:103850000704F4E8022312F10041069143F100014C
:1038600007910021DDE906BC4FF0FF30614508BF3C
:10387000584505D239463046FFF741FF002565E738
:103880001546002D05DA39462D20B0476D420AF164
:10389000FF3A4B462A46CDF800A039463046FCF7A1
:1038A00081FEEBE7B8F17A0F02D154F8042B11E056
:1038B000B8F16C0FF9D0B8F14C0FF6D100214FF0F0
:1038C000FF30073424F00704F4E80223994208BFCC
:1038D0009042CFD3CDF800A04B46DEE739463020EA
:1038E000B04739467820B0474FF0080A4FF0010939
:1038F000029B1B78702B04D154F8043B04930023E3
:103900000DE0B8F16C0FF7D0B8F14C0FF4D10734DB
:1039100024F007031C4654F8082B5B68049200212E
:1039200010224FF0400B03910591ABF1040B04986A
:10393000CBF1200CABF1200120FA0BF003FA0CFCC8
:1039400040EA0C0023FA01F1084310F00F0006D101
:10395000059911B9BBF1000F22D1302103E00928EC
:103960008CBF57213021084440B239460893059254
:10397000B047039B059A01330393089BBBF1000FEB
:1039800023D1B9F1030F7FF479AF039BC3EB4A0551
:10399000002D7FF773AF39462020B047013DF7E790
:1039A000511E9245089107DBB9F1010F06D1394646
:1039B00030200993B047099B089AB6E7B9F1020F86
:1039C000FAD1099339462020F4E70595ADE7394649
:1039D000B047FAE6394654F8040BB0474EE7A8461C
:1039E000A9464FF0FF3A0125B0E64FF00309ADE6D6
:1039F0004FF00109AAE60546A8E60FB407B504A9E9
:103A000051F8040B0191FCF71FFE03B05DF804EBC5
:103A100004B07047044608B5084611461A46A04748
:103A2000FEF7B6FDFDF7B4FC7047FEF733B80C2285
:103A30008368C9B202FB01314B7A23B9087AB0FA24
:103A400080F040097047022070470268F8B5976817
:103A5000CCB286684FF02003EFF3118583F3118811
:103A6000BFF36F8F0C226243B1180B7A1BB3013B7B
:103A7000DBB20B7213BBB3503A444B605368B3B91B
:103A80000C23012103FB0473DA7A1B8902F1502213
:103A90001160002203F150231A600C21002001FB69
:103AA0000464607285F31188BFF36F8FF8BD984787
:103AB0000028E5D1F1E76FF04400F3E70020F1E7DB
:103AC00038B50C248368054604FB01340123637276
:103AD0004FF02003EFF3118183F31188BFF36F8F51
:103AE00023682BB160681A688342226008BF626055
:103AF00081F31188BFF36F8F03B938BDD3E901217A
:103B000028469047E4E703682DE9F041D0F808C063
:103B100005469F68CEB24AB10C2373435CF803306C
:103B20009A425CD013B11B68002BF9D14FF02003EF
:103B3000EFF3118083F31188BFF36F8F0C21714372
:103B40000CEB01031C7A0134E4B21C7280F311887F
:103B5000BFF36F8F32B34FF050204FF0030EC0F819
:103B600008E3587AA0B94FF0200EEFF311888EF3D6
:103B70001188BFF36F8F1060D3F804E0BEF1000F1F
:103B800020D15A604CF8012088F31188BFF36F8F61
:103B90004FF050230321C3F8041318B1D2E90131C7
:103BA00028469847012C0BD10C237343FB586BB963
:103BB0000C23012203FB0676B37A03F150231A602B
:103BC00000200EE0CEF800205A60DDE72846984736
:103BD0000028EDD131462846FFF772FFF0E76FF07D
:103BE0000F00BDE8F0810022FFF78DBF10B5002265
:103BF000044601210520FDF7D7F90520FDF7C4F99A
:103C00004FF050230222C3F8182503220020C3F8E6
:103C10000423A368C3E90000A368C3E9030010BD3F
:103C200070477047002307B501A88DF80430FEF7F0
:103C30003FFF03B05DF804FB902908B5134639D166
:103C40000A4601460020FEF73FFFBDE808407146E6
:103C500072467346B7EE000AF7EE000AB7EE001A96
:103C6000F7EE001AB7EE002AF7EE002AB7EE003A98
:103C7000F7EE003AB7EE004AF7EE004AB7EE005A08
:103C8000F7EE005AB7EE006AF7EE006AB7EE007A78
:103C9000F7EE007A8EF3008C10B4F1EE10CA4FF6F6
:103CA0006074C0F6FF740CEA040CE1EE10CA10BC9C
:103CB000F44674476FF01500C7E7FEE7FDF7DCB97F
:103CC00043B2A9B1002B12DB01215B099B0003F178
:103CD000604303F56143D3F8802200F01F0001FA2E
:103CE00000F022EA0002C3F88022D3F88032704745
:103CF000002BFCDB01225B099B0003F1604303F511
:103D00006143D3F8801200F01F0002FA00F008436C
:103D1000C3F88002E9E700F007B90146006800F047
:103D200003B908B5FDF7B2F9BDE80840FDF7CAB818
:103D300007B5002101A8FDF7C3FC03B05DF804FB43
:103D400030B50B6885B04C689DF808200D89013CA2
:103D50000093498923F01F03234465F3040261F3B0
:103D6000471223F01F030F288DF808200393044601
:103D700005D86946FDF75CFB204605B030BD6FF005
:103D80001504F9E740E800F313F4803FD8B208BF08
:103D90006FF0150070470138013910F8013F11F834
:103DA000012F934201D1002BF7D1981A704710B51B
:103DB0005AB10139841810F8012B11F8013FA042C3
:103DC00001D09A42F7D0D01A10BD1046FCE7431A32
:103DD000934210B500EB020308D3024601399A4220
:103DE0000BD011F8014F02F8014BF8E70A4412F822
:103DF000014D8A4203F8014DF9D110BDF0B581EAB9
:103E00000004A50703460BD0013B0A4491421AD196
:103E1000F0BD002AFCD011F8014B013A03F8014B28
:103E20009C07F6D19508AC001E1F0F19B94205D1A9
:103E30006FF00306234406FB0522E5E751F804CBA7
:103E400046F804CFF2E711F8014B03F8014FDDE724
:103E5000034670B5C9B29C0710D141EA012444EA77
:103E60000445940803EB8406B3420DD16FF00305BB
:103E700005FB04241C44A34209D170BD002AFCD0D8
:103E800003F8011B013AE6E743F8045BECE703F8AB
:103E9000011BF0E74FF0FF3070470B46826892E855
:103EA000030083E803000020704703689B681B68D9
:103EB000D3F88004C3F880047047036882689B6865
:103EC0001B68D3F8100138B1127A00200A70012261
:103ED000C3F810011A6070474FF0FF30704700229E
:103EE000036882B09B688DF807101B68C3F8202117
:103EF0000DF10702C3F844250122C3F848259A6052
:103F0000D3F820110029FBD0DA6002B0704708B561
:103F10000020FDF71FFA08B5FCF73EFFFCF7BCFFD9
:103F2000BDE80840FEF788BE70B505460E46FEF7B0
:103F30002FFB314604462846FFF7E9FF2046BDE83F
:103F40007040FDF725BAFFF76CBE30B500248461E0
:103F500041EA020414F00304C0E9023201610CD109
:103F60004461A34203D1C0E90000002030BD45698F
:103F700001340D6041611144F3E76FF01500F5E77E
:103F800003460020C3E90033C3E902007047437BC6
:103F9000DB0603BF8069B0FA80F04009002070475B
:103FA00021B9EFF3058008B9FCF79ABF81F31188B6
:103FB000BFF36F8F7047034620B9EFF305820AB94C
:103FC000FCF78EBF83F31188BFF36F8F70474FF0FC
:103FD0002003EFF3118083F31188BFF36F8FFFF796
:103FE000EABF0368984214BF18460020704750F893
:103FF000103C70B50446A0F11805CBB14FF020037A
:10400000EFF3118683F31188BFF36F8F294650F8C1
:10401000100CFEF7ADF814F80B3C23F0020304F883
:104020000B3C86F31188BFF36F8F002344F8103CDC
:1040300014F80B3C284623F0140304F80B3CFFF75C
:10404000A6FF20B12846BDE87040FEF7E1B870BD7C
:1040500038B54FF02003EFF3118283F31188BFF3DB
:104060006F8FFFF7BEFF044682F31188BFF36F8F97
:10407000C8B14FF02003EFF3118583F31188BFF32C
:104080006F8F01468068FEF773F8637B23F00203AD
:10409000637385F31188BFF36F8F002304F1180059
:1040A000A36000F011F8204638BD10B5029C837360
:1040B000047300230424C3734473C0E90633C0E9C6
:1040C0001333C0E9161210BD10B54FF02002EFF304
:1040D000118482F31188BFF36F8F03683BB1FEF741
:1040E000FDFA002084F31188BFF36F8F10BD6FF0CD
:1040F0001500F7E710B54FF02003EFF3118483F3B9
:104100001188BFF36F8FFEF7FDFA84F31188BFF3B8
:104110006F8F10BD70B504460E464FF02003EFF3CD
:10412000118583F31188BFF36F8FFEF7EBFA012837
:1041300005DDA04203DD31462046FCF755FB85F343
:104140001188BFF36F8F70BD7047FFFF20C1FF7FE5
:104150000100000000000000BD3C00000000000065
:10416000BD3C000000000000BD3C0000000000005D
:10417000BD3C000000000000BD3C0000000000004D
:10418000E906000000000000BD3C00000000000047
:10419000BD3C000000000000BD3C0000000000002D
:1041A000BD3C000000000000BD3C0000000000001D
:1041B000BD3C000000000000BD3C0000000000000D
:1041C000BD3C000000000000BD3C000000000000FD
:1041D000BD3C000000000000BD3C000000000000ED
:1041E000BD3C000000000000BD3C000000000000DD
:1041F000BD3C000000000000BD3C000000000000CD
:104200003D07000000000000BD3C00000000000071
:10421000BD3C000000000000BD3C000000000000AC
:10422000BD3C000000000000BD3C0000000000009C
:10423000BD3C000000000000BD3C0000000000008C
:10424000BD3C000000000000BD3C0000000000007C
:10425000BD3C000000000000BD3C0000000000006C
:10426000BD3C000000000000BD3C0000000000005C
:10427000BD3C000000000000BD3C0000000000004C
:10428000BD3C000000000000BD3C0000000000003C
:10429000BD3C000000000000BD3C0000000000002C
:1042A000BD3C000000000000BD3C0000000000001C
:1042B000BD3C000000000000BD3C0000000000000C
:1042C000BD3C000000000000BD3C000000000000FC
:1042D000BD3C000000000000BD3C000000000000EC
:1042E000BD3C000000000000BD3C000000000000DC
:1042F000BD3C000000000000BD3C000000000000CC
:10430000BD3C000000000000BD3C000000000000BB
:10431000BD3C000000000000BD3C000000000000AB
:10432000BD3C000000000000BD3C0000000000009B
:10433000BD3C000000000000BD3C0000000000008B
:10434000BD3C000000000000BD3C0000000000007B
:10435000BD3C000000000000BD3C0000994700008B
:10436000650600000000000099470000CD0600002F
:104370000000000055490000ED3B00000C44000027
:10438000874700007D0700000000000099470000FB
:10439000B91500000000000080470000651900000A
:1043A0007046000099470000D1190000000000008D
:1043B000A84A0000173F00000000000099470000D5
:1043C000511E000000000000994700006D28000009
:1043D00000000000DEE61E284CBBCE8F025B000012
:1043E000DEE61E28EAAC45B8025B0000DEE61E28C9
:1043F0004CBBCE8F025B0000E73B00004B3A000055
:10440000073B0000000000002F3A00000000000001
:104410000000000000010004000000000000000097
:104420000401080C1701000007010000070100004B
:10443000070100000701000007010000070100005C
:10444000070100000701000007010000070100004C
:10445000070100000701000007010000070100003C
:10446000070100000701000007010000070100002C
:10447000070100000701000007010000070100001C
:10448000070100000701000007010000070100000C
:1044900007010000070100000701000007010000FC
:1044A000070100004A490000420100005149000094
:1044B000050100005B490000140100006449000090
:1044C000150100006D490000390100007649000027
:1044D00009010000814900000A0000008C49000029
:1044E0000A010000964900000B010000A0490000ED
:1044F0000F010000AB49000010010000B6490000A8
:1045000011010000C14900000E010000CB4900006C
:1045100021010000D449000022010000DD49000013
:1045200023010000E649000024010000EF490000DB
:1045300018010000F74900002A010000FF490000AF
:104540003A010000074A00002C0100000F4A000059
:104550001C010000184A00001D010000214A000053
:10456000170100002B4A000031010000374A00000B
:1045700004010000170100001701000017010000EE
:1045800017010000170100001701000017010000CB
:1045900017010000070100000701000007010000EB
:1045A00007010000070100000701000007010000EB
:1045B00007010000070100000701000007010000DB
:1045C00007010000070100000701000007010000CB
:1045D00007010000070100000701000007010000BB
:1045E00007010000070100000701000007010000AB
:1045F00007010000000000000002000000040000AD
:10460000000800000010000000000000BB3C00009B
:10461000050E0000C50D0000690E0000A50D00008C
:10462000EC130020D4130020E4130020000000004D
:10463000DC130020020000003C46000000000000E7
:10464000994A000006000000E0FF0F000000002073
:10465000A14A000021000000E0FF0020BB3E000056
:10466000DF3E0000AB3E0000F91700009B3E00005B
:10467000008000500100000050140020A41400200D
:10468000B0140020C8140020C8140020F5FFFFFF5C
:10469000436F756C64206E6F74206C6F636B207059
:1046A0006F7765722073617665206D75746578002B
:1046B000FF8FFFFFFF8FFFFFFE8FFFFFFE8FFFFFCC
:1046C000FD8FFFFFFC8FFFFFFC8FFFFF43616E2715
:1046D0007420696E697469616C697A65206D75749E
:1046E00065782C20776173204E554C4C0D0A0000E4
:1046F00043616E277420756E6C6F636B206D7574EB
:1047000065782C20776173204E554C4C0D0A0000C3
:104710004661696C20746F206163717569726520F0
:104720006D757465780A00004661696C20746F20AD
:1047300072656C65617365206D757465780A00003B
:104740004661696C20746F20696E63726561736580
:1047500020504D20636F756E7465720A0000000072
:104760004661696C20746F2064656372656173656E
:1047700020504D20636F756E7465720A0000000052
:10478000554152545F30007379735F636C6F636B94
:10479000005365637572650909004E6F6E2D536590
:1047A0006375726509004E6F6E2D53656375726592
:1047B00000466C61736820726567696F6E09094411
:1047C0006F6D61696E09095065726D697373696F08
:1047D0006E730A0025303275203078253035782008
:1047E0003078253035782009002563004E6F6E2D16
:1047F0007365637572652063616C6C61626C6520C2
:10480000726567696F6E203020706C61636564202B
:10481000696E20666C61736820726567696F6E20CF
:10482000256420776974682073697A652025642E71
:104830000A00436F756C64206E6F7420696E697432
:1048400069616C697A65207365637572652073654B
:104850007276696365732028657272202564292E3B
:104860000A005352414D20726567696F6E09094411
:104870006F6D61696E09095065726D697373696F57
:104880006E730A0025303275203078253035782057
:104890003078253035780900506572697068657226
:1048A000616C0909446F6D61696E09095374617423
:1048B00075730A002530327520252D32317325732A
:1048C0000009534B49500A00094552524F520A0001
:1048D000094F4B0A0053504D3A204E5320696D61E9
:1048E000676520617420307825780A0053504D3A6E
:1048F000204E53204D535020617420307825780A83
:104900000053504D3A204E532072657365742076E3
:104910006563746F7220617420307825780A0053C3
:10492000504D3A207072657061726520746F206A14
:10493000756D7020746F204E6F6E2D5365637572A8
:104940006520696D6167652E0A004E52465F5030E2
:10495000004E52465F434C4F434B004E52465F520F
:10496000544330004E52465F52544331004E52463B
:104970005F4E564D43004E52465F554152544531AD
:10498000004E52465F554152544532004E52465FEA
:104990005457494D32004E52465F5350494D3300F3
:1049A0004E52465F54494D455230004E52465F5478
:1049B000494D455231004E52465F54494D455232A1
:1049C000004E52465F5341414443004E52465F50B1
:1049D000574D30004E52465F50574D31004E5246B3
:1049E0005F50574D32004E52465F50574D33004E88
:1049F00052465F574454004E52465F495043004E62
:104A000052465F564D43004E52465F465055004E4B
:104A100052465F45475531004E52465F4547553235
:104A2000004E52465F4450504943004E52465F4745
:104A300050494F544531004E52465F524547554C00
:104A400041544F5253006D757465785F696E697497
:104A50002063616C6C65642077697468204E554CE6
:104A60004C20706172616D6574657200436F756C86
:104A700064206E6F7420616C6C6F63617465206D6F
:104A800075746578206265666F726520696E6974F9
:104A900069616C697A696E6700464C4153485F30C2
:104AA000005352414D5F300048575F43433331302C
:104AB0005F300076322E312E39392D6E637331001E
:104AC0002A2A2A20426F6F74696E67205A657068BF
:104AD0007972204F53206275696C642025732025FC
:104AE00073202A2A2A0A006D61696E0069646C6568
:104AF0000000000000000000FB360000DC14002075
:104B000001000000F0140020010000000415002046
:104B1000010000001815002001000000953E000073
:104B200000C2010000010300000000000090D0035B
:104B30000814002008140020401400204C14002009
:104B4000441400203C140020181400200000000031
:104B50006D2C0000D52C0000AD2C0000F12C0000C5
:104B6000B12C0000880600207C060020840600206E
:104B700000000000800600205C43000000000000F0
:104B800000000000BC430000000000000000000026
:104B9000C843000000000000000000008C4300003B
:104BA000000000000000000074430000F843000013
:104BB0000C000020984300005C460000F813002021
:104BC0006843000000000000000000008043000077
:104BD0000000000000000000B043000000000000E2
:104BE00000000000A44300000000000000000000DE
:104BF000C8140020C81400200000000000000000BD
:104C00000F000000DC140020DC1400200000000075
:104C1000000000000F000000F0140020F01400203D
:104C200000000000000000000F000000041500203C
:104C30000415002000000000000000000F0000002C
:104C400018150020181500200000000000000000CA
:104C50000F000000FFFFFFFFFFFFFFFFFFFFFFFF51
:104C60000000000000000000000000000000000044
:104C70000000000000000000000000000000000034
:104C80000000000000000000000000000000000024
:104C90000000000000000000000000000000000014
:107FE0007FE97FE9F8F71ABE7FE97FE9F8F76EBE0F
:107FF0007FE97FE9FBF720BE0000000000000000E1
:10C00000C8710220A5D10000219D0100B5CF00001C
:10C01000B5CF0000B5CF0000B5CF0000B5CF000010
:10C02000B5CF0000B5CF0000B5CF00007DCF000038
:10C03000B5CF0000B5CF0000C9CE00005D9C010067
:10C04000D1CF0000D1CF0000D1CF0000D1CF000070
:10C05000D1CF0000D1CF0000D1CF0000D1CF000060
:10C06000D1CF0000D1CF0000D1CF0000D1CF000050
:10C07000D1CF0000D1CF0000D1CF0000D1CF000040
:10C08000D1CF0000D1CF0000D1CF0000D1CF000030
:10C09000D1CF0000D1CF0000D1CF0000D1CF000020
:10C0A000D1CF0000D1CF0000D1CF0000D1CF000010
:10C0B000F5EA00005FA70100D1CF0000D1CF00005A
:10C0C000D1CF0000D1CF0000D1CF0000D1CF0000F0
:10C0D000D1CF0000D1CF0000D1CF0000D1CF0000E0
:10C0E000D1CF0000D1CF00007DA70100D1CF00004B
:10C0F000D1CF0000D1CF0000D1CF0000D1CF0000C0
:10C10000D1CF0000D1CF0000D1CF0000D1CF0000AF
:10C11000D1CF0000D1CF0000D1CF0000D1CF00009F
:10C12000D1CF0000D1CF0000D1CF0000D1CF00008F
:10C13000D1CF0000D1CF0000D1CF0000D1CF00007F
:10C14000D1CF00000000000000000000000000004F
:10C1500000000000000000000000000000000000DF
:10C1600000000000000000000000000000000000CF
:10C1700000000000000000000000000000000000BF
:10C1800000000000000000000000000000000000AF
:10C19000000000000000000000000000000000009F
:10C1A000000000000000000000000000000000008F
:10C1B000000000000000000000000000000000007F
:10C1C000000000000000000000000000000000006F
:10C1D000000000000000000000000000000000005F
:10C1E000000000000000000000000000000000004F
:10C1F000000000000000000000000000000000003F
:10C20000DEE61E284CBBCE8F025B00003C00000027
:10C210003C0C01000100000000C0000000C0000054
:10C22000FFFF02910000000000000000000000007D
:10C2300000000000000000000000000053B94AB9EF
:10C24000002908BF00281CBF4FF0FF314FF0FF301E
:10C2500000F070B9ADF1080C6DE904CE00F006F8FD
:10C26000DDF804E0DDE9022304B070472DE9F04F6A
:10C27000099E04468946002B40F083808A42154679
:10C2800045D9B2FA82F24AB1C2F1200701FA02F3AB
:10C290009540944020FA07F747EA03094FEA154E04
:10C2A000230C1FFA85F8B9FBFEFC0EFB1C990CFB56
:10C2B00008F143EA094399420AD9EB182CBF01203F
:10C2C0000020994202D9002800F01D810CF1FF3CAA
:10C2D000591AA3B2B1FBFEF00EFB101100FB08F8D7
:10C2E00043EA0144A04505D92C1902D2A04500F229
:10C2F0000E810138A4EB080440EA0C4000271EB16F
:10C30000D4400023C6E900433946BDE8F08F002A37
:10C3100051D0B2FA82F2002A40F0AF80491B4FEAB6
:10C32000154E1FFA85F80127230CB1FBFEFC0EFB0E
:10C330001C1108FB0CF043EA014398420AD9EB18A0
:10C340002CBF01210021984202D9002900F0D7809A
:10C350000CF1FF3C191AA3B2B1FBFEF00EFB101159
:10C3600008FB00F843EA0144A04505D92C1902D284
:10C37000A04500F2C1800138A4EB080440EA0C405B
:10C38000BDE78B4208D9002E74D00027C6E9000112
:10C3900038463946BDE8F08FB3FA83F767B98B4268
:10C3A000C0F0A480824240F2A1803846002EABD07B
:10C3B000C6E90049A8E7FFDEC7F12005BB4002FA45
:10C3C00007FC01FA07F4EA4020FA05F8E94000FA10
:10C3D00007FE1A4348EA04044FEA1248200C1FFAE9
:10C3E00082F9B1FBF8FA08FB1A110AFB09FB40EAD3
:10C3F00001418B450AD951182CBF012300238B45DD
:10C4000002D9002B00F088800AF1FF3AA1EB0B0162
:10C41000A4B2B1FBF8F008FB101100FB09F944EAE3
:10C420000141894504D9511801D289457BD8013889
:10C4300040EA0A40A1EB0901A0FB0C8949454446AA
:10C440004B4602D306D1C64504D20138B8EB0C04E2
:10C4500069EB0203002E5DD0BEEB040261EB030129
:10C4600001FA05F522FA07F3F94000271D43C6E952
:10C47000005149E73746304646E7C2F12000954073
:10C4800001FA02F721FA00F34FEA154E24FA00F1FF
:10C490001FFA85F894403943B3FBFEF00F0C0EFBF6
:10C4A000103300FB08FC47EA03439C4507D9EB180F
:10C4B0002CBF012700279C4500D98FB30138A3EB7F
:10C4C0000C0389B2B3FBFEF70EFB173307FB08FC26
:10C4D00041EA03418C4504D9691801D28C4525D81D
:10C4E000013FA1EB0C0147EA00471DE7841A61EB0D
:10C4F00003030120994659E702382C443CE7ACF18C
:10C50000020C2B4426E7ACF1020C2B44E0E6023887
:10C510002C44EFE63746F7E6AAF1020A114475E724
:10C5200002382B44CBE70238114481E7023F29440B
:10C53000D7E700BF704700BF70B504460D4643689B
:10C540005B6913B10A46002198476368DB681BB139
:10C55000002206492046984763682A461E68002341
:10C560002046B446BDE8704019466047DC00022012
:10C5700070B512480BF038FA114C2060E0B14368F6
:10C5800006221D6800214FF48973A847A0B90D4900
:10C590000D4B20684B6040238B604368DB685BB1C8
:10C5A00001229847014638B9206843681B691BB1CE
:10C5B000BDE870400622184770BD00BF24C00100CE
:10C5C000D8000220DC000220C991010010B5044609
:10C5D000FFF7CEFF012C1CD074B1022C22D102F047
:10C5E0004FFE05F033F84FF040230122C3F8002539
:10C5F000BFF34F8F20BFFDE705210B480CF07FFEF6
:10C6000002F03EFE0122094B1A60BDE8104000F026
:10C61000CBBC052104480CF072FE02F031FE044B45
:10C620001C60F2E710BD00BFE80002207C50004013
:10C630007850004070B50D4C054614F810300E4689
:10C640008B4211D04FF0FF3109480CF053FA14F827
:10C65000153004EB4502DBB2537004F81560044852
:10C66000BDE870400CF01ABA70BD00BF5F4C0220EC
:10C670005CA10220064B9A78012A08D11A79012A76
:10C6800005D19B79DBB2012B04BF024A13707047BE
:10C690005F4C02205E4C022010B5054CFFF7EAFF0C
:10C6A0002378002BFAD00020FFF790FFF6E700BFB9
:10C6B0005E4C022043680A461BB11B6E0BB1014958
:10C6C00018477047C9C6000001480CF085BD00BF7F
:10C6D000E80002201C23064A03FB00208268D2E9FE
:10C6E0000003834238BF03F50063181A704700BF88
:10C6F000E8000220F0B50546144E154F8FB0ECB29D
:10C7000001212046FFF796FF4FF4006300220493B7
:10C7100003A94FF0FF3330460A920BF06FFB022162
:10C720002046FFF787FF01AA4FF0FF33394603A8E1
:10C730000EF075FC049A22B1064B019958680CF072
:10C74000D0FD01A80EF08EFCD9E700BF18A2022090
:10C75000ECA00220E800022038B500250B4C257023
:10C760000B480BF041F90B4B6060A3600A4B257638
:10C77000E3600A4B2A462361094B204663614FF46C
:10C78000E131BDE838400CF07BBD00BFE80002207D
:10C7900041C00100B8970220E8970220D4970220F8
:10C7A000C8A102202DE9F04F354C8FB08046FFF72D
:10C7B000D3FF0022A146E368324F6FF31033E360EA
:10C7C00023699A605FFA88F501212846FFF732FF56
:10C7D0004FF0FF32012148460CF07AFC00283AD194
:10C7E00002212846FFF726FFE36803F4F833B3F588
:10C7F000805F30D12369DB68012B2CD13B70002690
:10C8000000234FF4006208A91F480BF0D9FBDFF8A2
:10C8100084A0089D0020FFF75DFF83462B189D42F2
:10C8200024D15E4428200CF00BF9DAF80830D3E963
:10C8300000239A4202D0B6F5006FEBD30025134BCC
:10C840002A461B6803A9124804960B9306950BF021
:10C85000ABFA3D7002E03B78002BD0D10022E368B8
:10C860006FF31033E36023699A60ABE72946012236
:10C87000DAF80800019301350DF054F9019BCEE779
:10C88000D4970220674C022008A10220B4BB01000B
:10C8900018A20220E8000220F0B50746104E114D04
:10C8A0008FB0FCB220460121FFF7C4FE4FF40063B5
:10C8B0000022049303A94FF0FF3330460A920BF095
:10C8C0009DFA20460221FFF7B5FE4FF0FF3301AA83
:10C8D000294603A80EF0A3FB01A80EF0C3FBE0E776
:10C8E00018A2022024A102200B6801330B60014B27
:10C8F0001B681847F89702202DE9F04F85B00E9C71
:10C900009B46012CB8BF0124012B0CBF30232023F0
:10C9100016468246884601250A270022DFF86C90D9
:10C920000293B6FBF9F301930AB9B1451CD8019BF8
:10C93000414603F13000D04701220135019B013F00
:10C9400009FB13660A23012FB9FBF3F9E9D141462C
:10C9500006F13000D047BBF1030F02D1641B002C5D
:10C960000EDC05B0BDE8F08FBC42E7DBBBF1020F87
:10C97000E4D84146029803920135D047039ADDE797
:10C9800041462020D047013CE9E700BF00CA9A3B5E
:10C99000014B1860704700BFF8970220002307B5CD
:10C9A0000246019303480B4601A90CF08AFE03B02E
:10C9B0005DF804FBE9C800004FF02002EFF311839B
:10C9C00082F31188BFF36F8F0121044AC2F840152A
:10C9D00083F31188BFF36F8F0020704700900340EE
:10C9E000014B1860704700BFFC3B02202DE9F74F58
:10C9F000194801A90BF01EF8042300244FF00C097C
:10CA0000164DDFF854A0DFF85C802B60019BA34239
:10CA100002DD2B680E2B02DD03B0BDE8F08F00268F
:10CA200009FB04FB0E4FDAF80030394653F80B309F
:10CA300018680DF09AFA50B10136042E07F110076C
:10CA4000F1D12B685A1C2A6048F8234001E048F8CD
:10CA500026400134DAE700BF403C0220003C0220BF
:10CA600062C00100043C022010B5044C2046FFF7D0
:10CA70008FFF204601F016FB002010BD81CA000088
:10CA80002DE9F34106460324154F164D8DF8070096
:10CA90004FF0FF3138460BF0DDFB01220DF10701AD
:10CAA000002000F0CFF9804638460BF045FCB8F185
:10CAB000000F05D001232B70304602B0BDE8F08195
:10CAC0002B78002BF8D0013C07D00EF0F0FC0028AA
:10CAD000DED102200BF0B4FFDAE72C70ECE700BFE8
:10CAE000A0A10220684C022003682DE9F041D0F893
:10CAF00008C005461F69CEB24AB10C2373435CF8E7
:10CB000003309A425CD013B11B68002BF9D14FF06F
:10CB10002003EFF3118083F31188BFF36F8F0C2193
:10CB200071430CEB01031C7A0134E4B21C7280F3F4
:10CB30001188BFF36F8F22B34FF0030E2248C0F865
:10CB400008E3587AA0B94FF0200EEFF311888EF366
:10CB50001188BFF36F8F1060D3F804E0BEF1000FAF
:10CB600021D15A604CF8012088F31188BFF36F8FF0
:10CB70000321154BC3F8041318B1D2E9013128463B
:10CB80009847012C0DD10C237343FB587BB90C2320
:10CB9000012203FB0676B37A03F1804303F5A04339
:10CBA0001A6000200EE0CEF800205A60DCE728462C
:10CBB00098470028EBD1314628460DF027F8F0E7DA
:10CBC0006FF00F00BDE8F0810050004010B500226A
:10CBD00004460121052000F047FA052000F034FA50
:10CBE0000222074B0020C3F818250322C3F80423B0
:10CBF000A368C3E90000A368C3E9030010BD00BF38
:10CC00000050004008B5104B1A6862B10F4AD2F8C4
:10CC10000423D10707D500220D481A608368597A8A
:10CC200009B90CF0F3FF0B4B1A6862B1074AD2F84E
:10CC30000423920707D5002201211A600448BDE8A9
:10CC400008400CF0E3BF08BD005100400050004018
:10CC5000709F02200451004000220D4BC3F8402178
:10CC60004FF02002EFF3118182F31188BFF36F8F31
:10CC7000084AD3F804051368C01A20F07F40034423
:10CC8000136081F31188BFF36F8F0CF045B900BFBB
:10CC9000005001405C3C022070B515480AF0A4FE2B
:10CCA00010B3436801211B689847002401264FF404
:10CCB00080334FF400120F4D3146C5F80845C5F8D2
:10CCC0004065C5F804330C4B15201C600B4BC3F8B2
:10CCD0008021224600F0C8F9152000F0B5F9204661
:10CCE000074B1E602E6070BD4FF0FF30FBE700BFAA
:10CCF000A2C00100005001404051014000E100E0AD
:10CD00000850014070B5254CB0F1FF3F08BF2046E8
:10CD10004FF02003EFF3118583F31188BFF36F8F7A
:10CD20001F4BD3F804151F4B1B68CA1A22F07F460D
:10CD300012021AD4421E22EAE272A242A8BF22467E
:10CD4000701C1044A04294BF18181819411A21F001
:10CD50007F41134A20F07F430229C2F8403506D9AB
:10CD600085F31188BFF36F8F70BD0022E8E7D2F81A
:10CD700004350D49C31A23F07F435C1E8C4205D94C
:10CD80004FF40012094BC3F80021E9E7012B02BF61
:10CD9000023020F07F40C2F84005E1E7FEFFFF00CF
:10CDA000005001405C3C0220FEFF7F0000E100E0FB
:10CDB0004FF02002EFF3118382F31188BFF36F8FDE
:10CDC000064AD2F80405064A1268801A20F07F400D
:10CDD00083F31188BFF36F8F704700BF005001408D
:10CDE0005C3C0220032310B5104C114AC4E9043303
:10CDF000104BA261E3614FF4806322660E4A236206
:10CE00006266002310220D49E01DA3626362E362A3
:10CE10002367E3666367A2660DF075F8084920464C
:10CE20000DF071F82023A37110BD00BF603C0220FB
:10CE3000B2C00100794C0220694C0220BBC0010045
:10CE4000BFC00100F8B51823174C00FB033503FBE6
:10CE500000402544C46A0F46012C164611D024B167
:10CE6000022C1BD000242046F8BD28460CF0F8FE0A
:10CE7000B042F8D33246394628460CF0FFFE34461D
:10CE8000F1E728460CF0ECFE8642344628BF044603
:10CE90003946224628460CF0F1FEE4E72846BDE874
:10CEA000F8400CF005BF00BF603C022004488168D8
:10CEB000406A884203D003494FF080520A607047AD
:10CEC000304B022004ED00E02A498A684FF0280028
:10CED0001044EFF3098C80E8F01F4FF010001EEAB9
:10CEE000000F04D0D2F8CC0020F0040007E002F1DB
:10CEF0008C0080EC108AD2F8CC0050F00400C2F80C
:10CF0000CC00202080F31188BFF36F8F1A4F4FF0B1
:10CF100000664A6A8A603E60D2F884000023C2F844
:10CF2000843080F31188D2F8CC0010F0040F05D1C2
:10CF30000023E1EE103A5EF0100E05E02EF0100E28
:10CF400002F18C0090EC108AEFF3148323F00403B9
:10CF500083F31488BFF36F8F04B510460CF0E7FE1F
:10CF6000BDE8044002F1280090E8F01F8CF3098826
:10CF700070470000304B022004ED00E01EF0040F6B
:10CF80000CBFEFF30880EFF30980816911F8021CF0
:10CF90000229FFD001B50CF0BFFE01BD01491022EE
:10CFA0000A60704710ED00E0404080F3118830BF08
:10CFB000704700BFEFF30880EFF30981724601B5B7
:10CFC00000F054F901BD00BF30BFFFF7FDBF00BF47
:10CFD00001B572B60B4A106A00281EBF002111620B
:10CFE0000DF0D8FF62B6EFF30580A0F110004FEA14
:10CFF000C0000549014409C99847BDE801400349FB
:10D0000008470000304B022004B80100ADCE0000FC
:10D010000A4A0B4993680968C3F88400C3F888106A
:10D0200008494B6843F080534B60002383F3118819
:10D03000BFF36F8F9368D3F888007047304B02209E
:10D0400020C0010000ED00E043B2002B08DB01220C
:10D0500000F01F0002FA00F0024A5B0942F82300C8
:10D06000704700BF00E100E043B2002B01F1010175
:10D07000A8BF03F160434FEA4111B8BF054BC9B2E5
:10D08000ABBF03F5614300F00F0083F800131954A0
:10D09000704700BF14ED00E008B572B6044B186A83
:10D0A00018B100221A620DF075FF62B608BD00BF0C
:10D0B000304B022073B51E460A9B05460093099B20
:10D0C0008C180EF0FAF90D4AA4F1200323F007039F
:10D0D00022F001029A61069A1E605A60079A9A60CD
:10D0E000089ADA604FF08072DA61AB640023C5F809
:10D0F0008430C5F8CC3002B070BD00BFBD990100CE
:10D100002DE9F0411F4606460C4690460023E1EE0D
:10D11000103AEFF3148525F0040585F31488BFF366
:10D120006F8F00F06BF90A4B444430469E6024F048
:10D1300007040CF0FCFD384684F30988002163B62F
:10D1400081F31188BFF36F8F002200230CF036FCAF
:10D15000304B0220114A08B5114B22F07F029A6031
:10D16000BFF34F8FBFF36F8FD3F8882042F4A00234
:10D17000C3F888204FF04042C3F83422BFF34F8FEA
:10D18000BFF36F8F0023E1EE103A0AF083FC0AF040
:10D190008BFC00F001F90AF0C5FC00BF00C00000E4
:10D1A00000ED00E00CF0DEFC202080F31188084840
:10D1B0004FF40061401880F30988EFF314800221D6
:10D1C000084380F31488BFF36F8FFFF7C3FF00009D
:10D1D000087302200C4B9A6A9A6A9A6A920708D5D9
:10D1E0005A6B9A6A120604D518B19A6A22F0800224
:10D1F0009A620020044B9A6A9A6A9A6A9A6A42F082
:10D20000FF029A620870704700ED00E00D4B9A6AC9
:10D210009A6A9A6A920508D59A6B9A6A120404D59A
:10D2200018B19A6A22F400429A620020054B9A6A69
:10D230009A6AD20558BF9A6A9A6A42F47F429A6201
:10D240000870704700ED00E0074B00209A6A9A6A68
:10D250009A6A9A6A9A6A9A6A9A6A9A6A6FEA024219
:10D260006FEA12429A62704700ED00E070B53A4BE7
:10D270009CB05B680025C3F3080385F31188BFF3F6
:10D280006F8F02F07F44B4F17F4F19D1D60717D4C6
:10D29000550604D4140705D40646012504E012F00F
:10D2A00004050BD00E4600250022033B8DF8072015
:10D2B000032B49D8DFE803F00640443D0646F3E778
:10D2C0002E46F1E7244BDA6A92073DD4DC6A14F06B
:10D2D000804408D028331B78EBB101200DF1070101
:10D2E000FFF778FF04469DF8073093B9682231466E
:10D2F00002A80CF065FE099B45B3C3F3080222B9EE
:10D300006FEA53236FEA4323099302A920460CF0E6
:10D3100001FD1CB070BD114B1B782BB101200DF12C
:10D320000701FFF773FFDDE70D4B1C88A4B2002C4B
:10D33000D9D0FFF789FFD5E70DF107010020CFE72E
:10D340000DF107010020ECE70024CCE723F4FF7384
:10D3500023F00103D8E700BF00ED00E029ED00E075
:10D360002AED00E0024A536943F01003536170470D
:10D3700000ED00E0BFF34F8F0549064BCA6802F489
:10D38000E0621343CB60BFF34F8F00BFFDE700BFE8
:10D3900000ED00E00400FA05002320210348C21834
:10D3A0000133412B82F80013F9D1704700E100E00E
:10D3B00038B505464FF02003EFF3118483F311884D
:10D3C000BFF36F8F0BF08EF90A4B9B68AB420BD10A
:10D3D000094B5A68C2F3080212B92046FFF718FE3B
:10D3E0005A6842F080525A602046BDE838400DF03D
:10D3F0006ABF00BF304B022000ED00E010B50E4BBD
:10D4000088B002930D4B0E4C03930E4B0E4A0493BF
:10D4100002AB019301A82346012100F003F9002388
:10D4200007930A4B0121E41A05A80593069400F01E
:10D4300003F908B010BD00BF00000220000000008A
:10D44000000004200600010000000220000002206D
:10D4500010B50B680C7A23F01F0204F01F031A4367
:10D46000CB68640923F01F03044943EA440343F0F3
:10D4700001038860CA600B6110BD00BF90ED00E041
:10D480002DE9F04F8046894614460027484D85B067
:10D490004F4507DA58F827305E68C6B31F2E05D807
:10D4A0006FF01504204605B0BDE8F08FF206F7D105
:10D4B000D3F800A01AF01F0FF2D150460CF061FC17
:10D4C000834606EB0A0001380CF05BFC8345E7D18C
:10D4D0001BF1160FE4D0631E5B45E1DBC5F808B015
:10D4E000E86858F82710C5F808B02E6920F01F002A
:10D4F000D1E900321A44984246F01F0602F1FF3A81
:10D5000018D1564505D15FFA8BF00CF018FC0137A5
:10D51000BEE7C5F808B0EB6822F01F0203F01F0356
:10D520001A43EA60E0B20CF00AFC10F1160FB7D013
:10D53000441CECE7C5F808B02A69013B23F01F033F
:10D5400002F01F0213435645E0B22B61EBD00CF002
:10D55000F6FB10F1160FA3D0C5F808B0EA689DF8E5
:10D560000830013E62F304038DF808302B699DF802
:10D5700008205B0863F347128DF8082058F827202D
:10D580000130D2E900321344009323F01F031E44FC
:10D59000A6EB0A06C4B226F01F060F2C03963FF630
:10D5A0007FAF20466946FFF753FF0134AFE700BF66
:10D5B00090ED00E00522034B5A60BFF34F8FBFF39D
:10D5C0006F8F704790ED00E0BFF35F8F0022014B3B
:10D5D0005A60704790ED00E070B50E4D2E68102E29
:10D5E00015D80024FFF7F0FF0B4B0C4A1A63A64234
:10D5F00005D10B4B1E70FFF7DDFF002070BD696881
:10D60000204601EB0411FFF723FF0134EFE74FF051
:10D61000FF30F3E7E4BB010090ED00E0AAFF440017
:10D620007950022010B5034C2278FFF729FF2070B3
:10D6300010BD00BF795002202DE9F74F254C8A46D6
:10D6400080460027A1464FF0140B234D57451ADAA8
:10D65000D8F804300193002B36D0D8F800100846D3
:10D6600000910CF08EFBDDE90013064658180138D6
:10D670000CF087FB8642194A08D014235F436FF0F1
:10D68000150349F8073003B0BDE8F08F16F1160F07
:10D690002660F8D01378B342F5DD0BFB0793AE603C
:10D6A000AE60E868197B60F3040119732969187B7F
:10D6B000490861F347101873EB6823F01F03636098
:10D6C0002B6923F01F0323610137143408F10C0880
:10D6D000BCE700BF083D022090ED00E07950022039
:10D6E00070B50C4B0E461C780546234600210A4AAD
:10D6F0000F2B0BDD094951F8040BFFF7A9FE224659
:10D7000031462846BDE87040FFF7BABE936011610C
:10D710000133EDE77950022090ED00E0083D022052
:10D720002DE9F04F1E460023A3B0CDE9020101937D
:10D73000134613F8010B089358B1252800F0858093
:10D740000399029B9847013040F017844FF0FF3354
:10D750000193019823B0BDE8F08F232C6CD061D8E1
:10D76000002CF6D0202C0E9B08BF01230E93CDF881
:10D770002080DDF82080B74818F8014B21460CF0D6
:10D78000DFFB0028E9D12A2C66D156F8043B98F833
:10D790000040002B0993BFBF5B42099301230F9305
:10D7A000089B03F102082E2C7BD198F800302A2B1D
:10D7B00074D156F8045B08F1010818F8014B2146B2
:10D7C000A54827460CF0BCFB00286DD0434613F853
:10D7D000014B682F089307D1682C05D1482708F121
:10D7E000020398F801400893672C7BD8652C80F0E1
:10D7F0003581472C5CD8452C80F03081002CA8D096
:10D80000252C00F0B68303992520029B9847013010
:10D810009CD003992046029B9847013096D0019BEB
:10D820000233ACE32D2C0AD0302C0BD02B2C0B9BCD
:10D8300008BF01230B939AE74FF0010B97E70123F1
:10D840000F9394E701230A9391E700230A930E9321
:10D850000B930F939B468CE7A4F13003092B09909F
:10D86000A1D80A22DDF8208018F8014BA4F130037A
:10D87000092B98D8099B02FB0344A4F13003CDE99E
:10D880000883EFE7904601FB0535303D424612F82C
:10D89000013BA3F130000928F4D98EE700250A21C5
:10D8A000F4E74FF0FF358AE7CDF8208007469BE785
:10D8B000632C59D020D8582CA5D16F2C06F104091F
:10D8C000316840F02883BBF1000F00F0178330234C
:10D8D0008DF86C30002940F01B838DF86D100F46D9
:10D8E000012625E0702C00F0F58227D86E2C00F080
:10D8F000DE82E2D8692C86D1376806F10409002F50
:10D9000080F29A802D2379428DF86C300DF16D06EE
:10D9100030460A220CF0A0FB0B9B06441BA8361ACB
:10D92000002B40F02F830E9B002B40F02B83FF0F2A
:10D93000002D21DA0025AB46A846E1E0752CBCD0CD
:10D94000782CBAD0732C7FF45EAFB146002DB8BFEF
:10D950006FF00045002659F8043BB54240F0C982FB
:10D960002E4600252F4608E00027B1463D460126F9
:10D9700059F8043B8DF86C301BABEA190025AB4617
:10D98000A846921B22EAE272911906910999901910
:10D990000C1A0F9911B9002C00F3118303EB070A3D
:10D9A000534540F0118312F1FF3280F01B83F61BC8
:10D9B000B8F1000F11D09AF800000AEB0607A0F1A9
:10D9C0003003092BA7EB0A0640F21783474617F1ED
:10D9D000FF3780F01B83A6EB0806BBF1000F15D0C4
:10D9E0000AEB06071AF8018B03994046029B9847F9
:10D9F00001303FF4ABAEB8F12E0FA7EB0A06F1D120
:10DA00005F46002F00F30B83A6EB0B0695B19AF847
:10DA100000000AEB0607A0F13003092BA7EB0A066A
:10DA200040F208832E2800F005832F46002F00F3D4
:10DA30000A83761B564419E30B9B23B12B238DF8E5
:10DA40006C30394662E70E9B0BB12023F7E739466D
:10DA50001BAE5DE7C6C00100CCC0010006F107099E
:10DA600029F00709F9E80223D80240EA5250D60209
:10DA700020F00040002AC3F30A510496059073F188
:10DA80000003DDE90467CDE9166741DA2D238DF83F
:10DA90006C300DF16D0740F2FF73994253D1DDE90F
:10DAA00004120A43A4F1410407F1030340D1192CE5
:10DAB00038D849223A704E227A7046220025AB4669
:10DAC000A8461BAEBA70FD709B1B0B9A002A40F053
:10DAD000EC810E9A002A40F0E8819DF86C70A7F165
:10DAE0002D025742574105EB0806334403EB0B0662
:10DAF00022AB3B4413F81C3C303B092B00F246821E
:10DB00000A9B002B00F04582099B9A1B1BAB39E74F
:10DB10000B9B0BB12B23BAE70E9B0BB12023B6E76F
:10DB20001BAFB8E769223A706E227A706622C5E7A9
:10DB3000192C99BF4E2241216E22612194BF3A7067
:10DB40003A707970BAE7049B05980B431093CB1792
:10DB50000343462C119308BF6624DDE910231343C9
:10DB600000F01181002900F09B800026179BA1F294
:10DB7000FE3843F00043179318F1020FC0F2A4805F
:10DB8000B8F1000F00F3DD8016A808F101080CF0D1
:10DB900085FAB8F1040FF7D1002D04F0DF03B8BF08
:10DBA0000625472B40F0F880F11C02DBB54280F2DD
:10DBB000ED80023CE4B2002D00F0F480013DBBF1A9
:10DBC000000F40F0EF80002DD4BF4FF0000A4FF05F
:10DBD000010A662C40F0E88015EB060840F1EC8065
:10DBE000102366244FF00008159300224FF00063C5
:10DBF000CDE9182318F1FF3880F0E080169B189AC1
:10DC000019999B18179A41EB0202CDE9163202F0DE
:10DC10007043129300231393DDE91223134306D0BC
:10DC200016A80CF04CFA16A80CF038FA0136662C3F
:10DC300040F0E180002E40F3C880159B002B07DDEB
:10DC400015A916A80CF066FA013E07F8010BF4D1ED
:10DC5000B0463B460026BBF1000F01D1002D15DD7B
:10DC60002E2203F8012B002E00F0C080002D40F37F
:10DC7000BF80C6F1000BAB45A8BFAB46A5EB0B05BB
:10DC8000002D03DD159A002A00F3A680BAF1000FDB
:10DC900040F0C68000221BAE1A709B1B15E70139AD
:10DCA000049BDB180493059B5B410593DDE904238A
:10DCB000002A73F10003F2DADDE90423CDE916232B
:10DCC00053E716A80CF0EAF9DDE916EC0023002171
:10DCD000CDF830C00D93BB48DDE90C23994208BF55
:10DCE000904208F10108ECD30520AEFB0023CDE9FA
:10DCF0000623079B013E00FB0C334FF0000C0793FB
:10DD0000DDE90623CDE91623002100236FF0004250
:10DD100007988B4208BF824208D2BCF1000F3FF443
:10DD20002BAFDDE90623CDE9162325E7069B08F195
:10DD3000FF38DB180693079B4FF0010C5B410793FC
:10DD4000E2E716A80CF0BBF9DDE916AE4FF0000CC7
:10DD500008F1FF380136002300216FF0004099429E
:10DD600008BF704506D2BCF1000F3FF409AFCDE902
:10DD700016AE05E71AEB0A0A4EEB0E0E08F1FF3855
:10DD80004FF0010CE7E70026B046FDE6AD1BBBF106
:10DD9000000F04D1662416E74FF0000A19E74FF090
:10DDA000000A19E74FF0000A05F101081023984511
:10DDB0001593A8BF984618E76624F7E718A80CF053
:10DDC0007EF918A80CF06AF914E73B4630224FF0B0
:10DDD000000803F8012B3EE715A916A806930CF0DE
:10DDE00099F9069B013D03F8010B49E7B34647E764
:10DDF0004FF0000B4AE715A916A80CF08BF9302854
:10DE0000387018BF06F1FF36BBF1000F38D1002D76
:10DE100036DC7B1CBAF1000F44D04FF0000BD84623
:10DE20001A4613F8011D3029FAD02E2918BF1346BF
:10DE3000002504F0DF02452A7FF42CAF002EB4BF8A
:10DE40002D222B221946B8BF7642632E01F8024BD1
:10DE50005A7008DD642096FBF0F200FB126602F1B6
:10DE60003004D91C9C700A2096FBF0F20B4600FB94
:10DE7000126602F13004303603F8024B4E7009E7A7
:10DE80002E22BB1C7A70002DC4DD159A002AC1DD3C
:10DE900015A916A806930CF03DF9069B013D03F861
:10DEA000010BF0E7D346D046C3E701271BE6B14696
:10DEB000682F59F8043B05D001DC482F07D0019AA0
:10DEC0001A6001E0019A1A804E46089A30E4019ADD
:10DED0001A70F9E7B14647F63003102259F8041BCF
:10DEE0000DF16E00ADF86C300CF0B6F80227861C10
:10DEF0001EE59A5D002A47D001362EE51BAC0822AC
:10DF000020460CF0A9F81BAEA61B064400270FE51F
:10DF10000DF16D04F3E7752C05D10A221BA80CF056
:10DF20009BF80646F2E7BBF1000F12D047F630032C
:10DF30000DF16E08ADF86C30102240460CF08CF8F4
:10DF4000582C09D01BAEA8EB060606444FEA4B0737
:10DF5000EEE40DF16C08EFE71BAA1378A3F1610161
:10DF600019299CBF203B137012F8013B002BF4D100
:10DF7000E8E703992046FFF7E4BB019B01330193D7
:10DF8000B146A1E70127D3E41546EBE41BAB002221
:10DF9000FAE41BAB0A9AF7E4CDE909320399029B34
:10DFA00020209847DDE9093201303FF4CFAB1AF168
:10DFB000FF3AF1D20199214401915446EEE4A24680
:10DFC000F5E700BF3233333313F8010B039909939C
:10DFD000029B0A929847DDE9093201307FF4E0ACF8
:10DFE000FFF7B4BB03993020029B09929847013098
:10DFF000099A7FF4D8ACFFF7A9BBDDE90231984755
:10E0000001303FF4A3AB1AF8010FD8E40399302094
:10E01000029B984701307FF4DAACFFF797BB039976
:10E020003020029B9847013007F1FF377FF4E9ACBD
:10E03000FFF78CBBDDE90231984701303FF486AB36
:10E040001AF8010FE7E403993020029B984701304A
:10E0500007F1FF377FF4EAACFFF778BB03991AF8B2
:10E06000010B029B984701303FF470ABA6EB0A030B
:10E07000002BF3DC019B069A002C134401937FF7DD
:10E0800023AF254606E003992020029B98470130E4
:10E090003FF45CAB15F1FF35F5D2019B23440193AE
:10E0A00012E700BF014B1860704700BF649A02205E
:10E0B0000CB41FB509B90DF10300CDE9020107AB9E
:10E0C000069A02A905480193FFF72AFB0022029B4A
:10E0D0001A7005B05DF804EB02B0704749A1010069
:10E0E00038B5074C074DAC4200D138BD23681B68DA
:10E0F0005B681BB11B680BB1204698472034F2E7E0
:10E1000040A2022060A2022038B5084C084DAC4263
:10E1100000D138BD206803210C300CF03BF810B959
:10E1200020460CF03DF82034F1E700BF40A2022069
:10E1300060A2022008B5094B1A786AB90121312082
:10E1400019700521FEF790FF3120FEF77DFF4FF09B
:10E150000042034BC3F80423002008BD7A5002207C
:10E160000010034070B5036882681B69514C187930
:10E1700001F01F0343EA40130020D4F80453EDB22A
:10E1800000F5A27654F82660C6F30426B34270D197
:10E1900025FA00F6F6076CD5850005F1804505F5F2
:10E1A0004435D5F8106526F00106C5F8106501253F
:10E1B00005FA00F0C4F808033F4D05EB8305D5F8D8
:10E1C000000220F44030C5F800029068C84010F00A
:10E1D00001004DD0D068C84010F0010048D050690F
:10E1E000C84010F0010050D09069C840C00744D426
:10E1F0001069D269C84022FA01F100F0010001F073
:10E200000101884214BF01210221002505F5A272F7
:10E2100054F8220010F0030031D1AA0002F180422C
:10E2200002F54432D2F810651B0203F4F85326F4C9
:10E23000473626F4407643EA014105F14003C2F82F
:10E2400010659B00D2F810659BB203F1804303F583
:10E2500044333143C2F810151860D2F8103543F03A
:10E260000103C2F81035012303FA05F5C4F804537D
:10E2700070BD0130082883D19EE70321C5E7013531
:10E28000082DC3D16FF01200F2E71369D269534031
:10E2900023FA01F111F0010F14BF4FF400324FF4D3
:10E2A0004032D5F8003223F440331343C5F800322E
:10E2B000DEE700BF00100340002584402DE9F74F42
:10E2C0008046856803F47040B0F5804F1E4640D00C
:10E2D00009DCB0F5805F3ED0B0F5405F3DD090B135
:10E2E0006FF0150032E0B0F5E04F38D004DCB0F547
:10E2F000A04FF5D1032006E0B0F5404F31D0B0F586
:10E30000504FEDD1072006F44077B7F5807F2AD033
:10E31000A7F5007463426341012919BFD4B2A14635
:10E320004FF01F0900244FF0010B06F0010C4FEADB
:10E330004C0747EA0C0747EA0020DFF8A0A040EAB4
:10E34000830706F00203A1450FD2002003B0BDE809
:10E35000F08F0220D7E70120D5E70420D3E705207E
:10E36000D1E70620CFE70323D6E7D8F800201269CB
:10E37000117904F01F0242EA411280324AF82270F9
:10E38000A9680BFA04F2002B25D01143A960696932
:10E39000B0064CBF114391436961A96970064CBF37
:10E3A00011439143A961296970074CBF11439143FF
:10E3B0002961E96930064CBF0A4321EA0202EA6199
:10E3C000214640460193FFF7CDFE0028BED101341F
:10E3D000E4B2019BB7E721EA0201D7E700258440B8
:10E3E0004F492DE9F0410D68002D60D04D4B0026BE
:10E3F0009A681B68DFF838E11F69D2E9020303401D
:10E40000D2E90504204323EA00033868D46912697D
:10E41000006954404440012023EA040493BB0B608C
:10E42000002301201F464049404ED1F8042300FA42
:10E4300003FC1CEA020F0DD056F8232052B103F55D
:10E44000A27251F8222046F82370C2F3042200FA87
:10E4500002F214430133082BE7D154BB85B10124E8
:10E460000025304BDFF8C8C09A681B681E69D2E9E6
:10E4700002130B40D2E90510014323EA01037BBBE1
:10E48000BDE8F08103420FD097F804C006F01F02E8
:10E4900042EA4C120EEB8202D2F800C223EA0003D9
:10E4A0002CF4403CC2F800C201364000B6E72C46CE
:10E4B000B6E71C4FD7F80880D8F800100029CDD057
:10E4C0000E68D8F80C308A682340134203D04B689A
:10E4D000224638469847002EC0D031463668F0E7CD
:10E4E0001C421AD0307905F01F01D76941EA40116A
:10E4F00010690CEB81017840E84010F0010F14BF67
:10E500004FF400374FF44037D1F8000223EA0403F8
:10E5100020F440303843C1F8000201356400AEE712
:10E520007C110340AC9F0220001003400011034007
:10E5300000258440F0B54B79012B29D0032B24D141
:10E5400010268B79032B20D1CC792CB1012C1CD136
:10E5500003681B691B79C3B10A7912B1022A14D16D
:10E560000E2247F6122705680B682D69BB422D68FD
:10E5700062D029D8B3F5965F61D014D8B3F5167F71
:10E580005FD007D8B3F5967F5ED06FF0220052E0DF
:10E590000026D6E7B3F5966F59D0B3F5166FF4D1D0
:10E5A0004FF41D233CE0B3F5615F53D004D8B3F5BD
:10E5B000165FEAD1324B33E0B3F5964F4CD0B3F54A
:10E5C000E14FE2D12F4B2BE0B3F5E13F46D012D81B
:10E5D0004DF6C027BB4244D005D8B3F5164FD4D171
:10E5E0004FF41D031CE0B3F5614F3DD0B3F5963FEA
:10E5F000CBD1254B14E0B3F5E12F38D008D8B3F5D3
:10E60000613F37D0214FBB42BFD14FF0806307E05D
:10E61000B3F5612F31D01E4FBB42B6D14FF08053BE
:10E62000C5F8243534438368224303C9C5F86C25F3
:10E6300083E803000020F0BD4FF40003F0E7154B22
:10E64000EEE74FF41C33EBE74FF4A033E8E74FF469
:10E650009E23E5E7104BE3E7104BE1E74FF0EB7348
:10E66000DEE74FF46503DBE74FF46B03D8E74FF0C9
:10E67000E863D5E74FF06C73D2E74FF07063CFE7F4
:10E680000050270000C0750000903A0190D00300B0
:10E6900040420F0000B0130000F03A0000A04E000E
:10E6A0000368F0B51D696B792BB32B682D79D3F80E
:10E6B0000C75D3F8142507F18006D3F81045D3F86C
:10E6C0000805164BC1B10121B94099600321571CBF
:10E6D00043F826101EBF0021803243F8221055B1A6
:10E6E000012282409A600322803043F820200022D9
:10E6F000803443F82420F0BD022143F82610561C34
:10E700001CBF803243F82210002DF4D00222803446
:10E71000803043F8242043F82020ECE70025844093
:10E72000F8B50546002201210820FEF79DFC0820CF
:10E73000FEF78AFC4FF480222B68AF681B69032127
:10E740001C682C4B12209A600022C3F84812C3F8B0
:10E750004422C4F80C051120C4F814054FF400102D
:10E760009860C3F85412C3F84C221523C4F8083536
:10E7700013233946C4F810352846FFF7DBFE06465A
:10E7800008BB0123FA683B61FAB104222B68AC682C
:10E790001B69E0681B681849C3F80423174A5C30FA
:10E7A000C3F804230822C3F8002532460CF0F0FE1B
:10E7B000E368C3F88450E0683246114910300CF029
:10E7C000E7FEE3689D633046F8BD0822C4F80025E3
:10E7D00007F11402C4F81001C4F83425BA68C4F86B
:10E7E000383592682360C4F84425C4F84805A3600E
:10E7F000E360E8E70025844031A4010010034A00EB
:10E800000BA701002DE9F04F036889B01B69D0F810
:10E8100008908DF80710D3F80080D9F80C30044622
:10E820004BB10026D9F80C309A680ABB0122DA6095
:10E83000984BC8F808330023C8F820310DF10703BE
:10E84000C8F844350123C8F84835C8F80830D8F866
:10E850002021002AFBD0C8F80C30D9F80C3023B1A5
:10E860000022DA608B4BC8F8043309B0BDE8F08FA2
:10E870000CF01DFE0028D5D023681B691D68D5F853
:10E88000081149B1A368C5F80861DA68D2F8883080
:10E890000133C2F88830C5E7D5F8243103B3C5F891
:10E8A0002411D5F880741422C5F8807403A80BF0E5
:10E8B000B1FB06238DF80C30FB0700F1DD80B807B3
:10E8C00000F1DC80790700F1DB8007F008072046C3
:10E8D00003A98DF810700BF09DFD20460BF018FF7A
:10E8E000D5F84C31C3B114220021C5F84C6103A8FE
:10E8F000A7680BF08FFB0323204603A98DF80C308B
:10E900000BF088FDF868036D5A1C05D08365426DD5
:10E9100011465C300AF09AFBD5F81031002B4BD031
:10E92000A768C5F81061F86890F88C30002B43D0C8
:10E930002368426C1B69D3F800A0012380F88E3055
:10E940000AB1CAF800305C300CF02EFEDAF83C2533
:10E95000D7F80CA00021DAF8403003A8A2EB030B93
:10E96000DAF84C2000935A44CAF84C20CAF88820A0
:10E9700014220BF04FFB0222009B8DF80C20DAF8DA
:10E980003C2003A920460492CDE9053B0BF042FD53
:10E9900004238DF80C30FB6803A9DB6B204604933D
:10E9A0000BF038FDFB685A6CDA63002A6AD0C3E9C1
:10E9B0001066FB6883F88E60D5F8443133B34FF0AE
:10E9C000040AA76814220021C5F8446103A80BF0CB
:10E9D00021FBFB6803A9DB6B204604938DF80CA098
:10E9E0000BF018FDFB68DE635B6C43B103A92046A6
:10E9F00004938DF80CA00BF00DFDFB685E640523FD
:10EA000003A920468DF80C300BF004FDD5F8203119
:10EA10005BB101212368C5F820611B691A68A368EE
:10EA2000D160D86810300CF0BFFDD5F85831002BFC
:10EA30003FF4F8AEA368C5F85861DD68AB68002BF9
:10EA40003FF4F0AE236814221B6900211B6803A861
:10EA5000D3F84C750BF0DEFAAB6803A9CDE90437A7
:10EA6000EB6820469F421CBF01238DF80C30AE603E
:10EA7000EE600BF0CFFCD5E6012728E7022726E75A
:10EA8000042724E7052303A920468DF80C300BF05A
:10EA9000C1FC8EE700014000002208B511462A2083
:10EAA000FEF7E2FA02F0C2FD014B1860002008BD3B
:10EAB0003C3D022070B50D4B0D4C1A680A2500260E
:10EAC0002346196881420ED051B15968511AB1429A
:10EAD000C4BF1C460E46013D03F10803F1D1234695
:10EAE000013A18605A60184670BD00BF403D0220D0
:10EAF0004C3D0220684620F007018D4619B50D4BAC
:10EB0000D3E8EF2F0132C3E8E12F0029F8D106F056
:10EB1000E5FF094B1C683CB9FEF7BEFAFEF7C6F9E3
:10EB2000BDE8194085467047201D09F0B7FF2468ED
:10EB3000F1E700BF403D0220443D02202DE9F04FA7
:10EB4000884689B00CF016FDD8F800300646002B38
:10EB50000F4603D109F028FF3C206EE0BCBF4FF008
:10EB6000FF33C8F800300122002102A80CF05BFC42
:10EB70000DF1040A4FF02003EFF3118B83F311889A
:10EB8000BFF36F8F09F084FFFFF794FF33494368A9
:10EB90000A68894693424FF0000308D10193304B35
:10EBA0005A68002A4CD1C3E900AA012300E0426060
:10EBB0008BF31188BFF36F8F002B3DD0D8F8001076
:10EBC00002A809F097FF4FF02003EFF3118B83F3B6
:10EBD0001188BFF36F8F0020214B1A6852B1524544
:10EBE00039D1019988BB58681960904200D15960A9
:10EBF0000023019309F04CFFFFF75CFFD9F80030C8
:10EC000043608BF31188BFF36F8FD8F80090B9F190
:10EC1000FF3F11D00CF0AEFC16EB090247EBE97395
:10EC2000141A63EB0105002C75F10003B8BF002432
:10EC3000C8F80040002C8FD0002009B0BDE8F08F4C
:10EC4000C2F800A0C3F804A0AFE701605968914280
:10EC500008BF5860CCE710461268BFE7403D02206D
:10EC6000443D02202D2810B504460CD028DC0E2887
:10EC700009D011DC082806D009DC022803D00528B9
:10EC800001D0012818D10BF068FD046010BD0C28DC
:10EC9000F9D047DC0928F5E7282873D005DC1828C7
:10ECA000F1D0232843D01628ECE72A28EBD042DB0A
:10ECB0002B28E8D02C2842D00BF04FFD334B34E00A
:10ECC0003C28E0D015DC3328DDD005DC3028DAD054
:10ECD000322838D02F28D5E73628D4D001DC342884
:10ECE000D0E73828CFD03928E6D10BF036FD3923CC
:10ECF0001BE07D2833D009DC702828D073282AD067
:10ED00006928D9D10BF029FD37230EE07F282FD0B9
:10ED100029DB802831D08128CED10BF01EFD40F2B6
:10ED2000D47302E00BF019FD0D230360AEE70BF086
:10ED300014FD0B23F9E70BF010FD2923F5E70BF089
:10ED40000CFD2C23F1E70BF008FD3E23EDE70BF063
:10ED500004FD4323E9E70BF000FD4423E5E70BF056
:10ED6000FCFC4823E1E70BF0F8FC40F2D173DCE750
:10ED70000BF0F3FC40F2D273D7E70BF0EEFC40F25D
:10ED8000D373D2E70BF0E9FC2423CEE7ADBAADBADA
:10ED90004FF08052014BC3F80021704700E100E0C2
:10EDA0004FF08052014BC3F88021704700E100E032
:10EDB0004FF00052014BC3F80021704700E100E022
:10EDC0004FF00052014BC3F88021704700E100E092
:10EDD00008B50023074AC2E90033074AD2E8EF1F0B
:10EDE000C2E8E03F0028F9D10BF0E2FCBDE80840A2
:10EDF0000BF0D3BC443D0220403D0220B0F58D7F96
:10EE00003CD004DC012844D04FF0FF30704740F282
:10EE10000223984252D040F203239842F4D10139A0
:10EE20001329F1D801A353F821F000BFC9EE000067
:10EE30008DEE0000ADEE00009FEE0000B1EE000090
:10EE4000B5EE0000B9EE000009EE000009EE00008A
:10EE500009EE000009EE000009EE000009EE0000D6
:10EE600009EE000009EE000009EE000009EE0000C6
:10EE700009EE000009EE0000A3EE000001390529AB
:10EE8000C2D8DFE801F0031517190C210223136023
:10EE90000AE0142905D0192905D00429B4D1042386
:10EEA000F5E71423F3E71160002070470323EEE732
:10EEB0000523ECE70623EAE70723E8E70229E5D084
:10EEC0000329F3D001299FD10123E0E70122034B5D
:10EED0001860036802489A76FDF782BD9C3D0220C7
:10EEE000ACBC010007B5019018B1D0F8983A0C30CD
:10EEF000984701A9024809F01FF803B05DF804FB28
:10EF0000D0A0022073B506460C460BF027F8104B34
:10EF100002461B680F48DD6A314600230068A84797
:10EF200001300ED108F096FD03685B420093012387
:10EF30008DF8043014B19DF804302370009802B0AD
:10EF400070BD4FF0FF326946034809F023F9F1E73D
:10EF5000FC3B0220A03D0220F0A1022008B5094B95
:10EF600040F201221B6800211B6866209847064B6F
:10EF70001860013004D108F06DFD0068404208BD02
:10EF80000020FCE7FC3B0220A03D022010B586B02B
:10EF9000FFF7E4FF044668B90A23CDE90400CDE990
:10EFA0000203CDE90000054B4FF480620449054897
:10EFB00009F068FE204606B010BD00BFC9EF000092
:10EFC000C8650220B43D02202DE9FF476A4E6B4F11
:10EFD000B0464FF0FF3201A9384608F081FF002308
:10EFE000674C01992268C1F8983A556A02938DF8E6
:10EFF0000C3040F68C220C313068A847002825469A
:10F0000031DA236830685B68984720BBFFF7A6FFBA
:10F0100008BB01238DF80C3008F01CFD03685B422F
:10F0200002930199D1F8983A002B7CD101A9384676
:10F0300008F082FF534B9B68002BCAD19DF80C202F
:10F04000042AC6D0504A13604FF0FF3202A94F483D
:10F0500009F04CF8BDE72B68D8F800005B689847CA
:10F0600004B0BDE8F08740F68C23984207D0DDF865
:10F070000490484490F80BA0BAF1000F02D06FF052
:10F080003603CDE7042309F10C04414920468DF8ED
:10F090000C300AF01BFF0546E8B18DF80CA0CDF846
:10F0A00008A000232A1B01322B709DF80C30019917
:10F0B000042B4ED0374D2B68002B52D0364C206895
:10F0C00000284ED093422AD90C310AF079FF002350
:10F0D0002B602360A5E7314920460AF0F7FE05467C
:10F0E00040B1022309F117008DF80C300AF052FEEE
:10F0F0000290D6E72A4920460AF0E8FE054608B104
:10F100000323EFE7274920460AF0E0FE054668B3EF
:10F1100001238DF80C306FF007030293C1E76FF005
:10F1200023030293D3E7204B00224B600B460A6077
:10F1300043F8082FD3E8EF2F42F00100C3E8E40FB3
:10F14000002CF7D1D3073FF575AF18480CF00BF83A
:10F1500070E7002A3FF465AF154B1B68C1F8983A79
:10F160005FE7002A3FF45DAF074BF6E720460AF061
:10F17000F5FE421C99E700BFA03D0220D0A002206E
:10F18000FC3B022074A10220A43D0220F0A1022039
:10F19000F6C00100B03D0220AC3D0220F9C00100E4
:10F1A00005C1010011C10100E5EE0000704B022015
:10F1B000A83D02202DE9F0410546884617461E4627
:10F1C0000A4C4FF0FF31204609F094FC084B3146C1
:10F1D000C3F80080074B28461F60FFF793FE0546E3
:10F1E000204609F05BFC2846BDE8F08174A10220AE
:10F1F000AC3D0220B03D022038B50546064C4FF02C
:10F20000FF31204609F076FC044B1D602046BDE826
:10F21000384009F043BC00BF74A10220A83D022081
:10F2200010B50024034B0448C3E90044FFF7E4FF92
:10F23000204610BD843E022049F20000014809F03A
:10F240007BB800BFB4A1022038B505464FF0FF31AE
:10F25000094808F0FFFF094B1B681BB9BDE838409F
:10F26000FFF7ECBF1C689A68294658689047002C45
:10F27000F4D023462468F6E7B4A10220843E02209D
:10F2800008B5002304481A461946FFF793FF0028E3
:10F2900018BF6FF0040008BD17C101002DE9F0434D
:10F2A00000261E4C85B054F8049C1D4F01ADB1459D
:10F2B00003D8002005B0BDE8F083636A97E8070033
:10F2C000D3F8008085E807000C22294640460AF062
:10F2D00067FEA0B9B8F1000F11D0636A21691B68FD
:10F2E0001A6991420BD19A69A169914207D8E169E3
:10F2F000914204D962695B6932EA030307D0236A49
:10F300004BB1404080F311884FF0040002DFE36806
:10F3100001361C44CBE7626A1360F8E73CC2000088
:10F320009CBB010020B150F8081B090C00F052B83A
:10F33000704700BF014806F04BBC00BFECBC0100A9
:10F34000002310B582B0019361B970B1044601AADF
:10F35000092006F075FE18B9019B0BB10833236034
:10F3600002B010BD0F2002B010BD0E2002B010BDC3
:10F3700001F47043B3F5E04F0BD160B1034630F8B0
:10F38000082C092042EA014143F8081D194606F0FD
:10F390003FBE0F2070470E20704700BF20B1A0F184
:10F3A0000801092006F07EBE0E20704718B1014604
:10F3B000092006F089BF0E20704700BF10B5044633
:10F3C0000068FFF7F3FFA06818B1BDE8104001F036
:10F3D0000FB910BD30B53B4B85B01D68002D4CD02A
:10F3E00048F20203994253D01CD948F203039942D0
:10F3F0005AD049F20103994247D100244368026878
:10F40000CDE90244CDE90023E869694603685B68F9
:10F41000984701304ED020462B6843F480332B6050
:10F4200005B030BD48F2010399422ED1C368002BCC
:10F4300035D1286810F480003ED02B689BB2012B98
:10F4400005D12B681B0C1B0443F002032B601E4BE1
:10F450001A7802F0FF01002A31D01C4A117809B94C
:10F4600001211170002018702B6823F480032B6099
:10F470002B6843F400032B60D2E700680028CFD04C
:10F48000FFF794FF284605B030BD002005B030BD21
:10F490002B6813F480030BD0C0680028E4D00E233F
:10F4A00000206B6005B030BDC368012BA5D1F6E725
:10F4B0001846B5E70220B3E70E236B60B0E7034AB6
:10F4C0001170CFE7903E02207B5402207C54022032
:10F4D000002310B50749084A084C09482370036007
:10F4E0000B701360FFF726FF003018BF0120404269
:10F4F00010BD00BF7B5402208C3E02207C540220B1
:10F50000903E022000232DE9F047662882B0009348
:10F5100072D1022989466FD140F205239A42924660
:10F520006AD1484F3D68002D7CD18046464A6846E6
:10F5300006F0CAF8009B0646002B7DD0294604221F
:10F5400042483B600AF066FD009C2946C4E90389F5
:10F55000C4F814A001A8FFF7F3FE00283CD1012253
:10F560000421019B3A4D58739873D873587298725E
:10F57000D87219722A701A732268184642F48002EF
:10F58000226047F20101FFF7F3FE38BB4FF400029F
:10F590004FF0FF331146304606F042F9044610B3EF
:10F5A000009A002E136843F400331360009A136826
:10F5B00023F480031360009A136823F4000313609C
:10F5C00036DA002320463B604FF0FF36FFF74AFB58
:10F5D000304602B0BDE8F0870C24E1E70198FFF760
:10F5E000DDFE0524DCE7304606F08EF950B14468B4
:10F5F00044B100234360D3E71620FFF733FB4FF0FD
:10F60000FF36E5E7009A136843F400331360009A6D
:10F61000136823F480031360009A136823F4000333
:10F620001360D5E70120FFF71DFB4FF0FF36CFE752
:10F63000304606F0A7F8C4E71820FFF713FB4FF099
:10F64000FF36C5E7903E0220BDF300008C3E02204D
:10F650007B5402202DE9F04385B000295ED0002ABA
:10F6600016465BDD1F4680460D4606F04DF9044602
:10F67000002859D0C069BA070368DB6824D59847C9
:10F6800001303BD02368E06913F4803338D0002187
:10F6900023683A4623F480332360CDE90211CDE993
:10F6A0000056036869469B6898470546E069036809
:10F6B000DB689847013003D0236843F4803323602C
:10F6C000284605B0BDE8F083226812F08059D6D1F3
:10F6D0009847431CD6D14FF48032236A1146002B41
:10F6E00008BF0346404606F09BF858B14FF0FF357F
:10F6F000FFF7B8FA284605B0BDE8F0832320F5E708
:10F700001D46D4E7404606F0FFF803460028B9D06E
:10F7100040680028B6D0C3F80490E7E71620FFF74A
:10F72000A1FA4FF0FF35CBE70920FFF79BFA4FF026
:10F73000FF35C5E72DE9F04182B000295BD0042AEE
:10F7400059D11E4607460D4606F0DEF8044600284D
:10F7500067D0B00726D523689B035ED500262368B3
:10F76000002123F40033236001A8D5F80080FFF7BF
:10F77000E7FDF8B90425019B47F20301C3F80C80AB
:10F7800058729872D8721D721846FFF7F1FD8046C4
:10F7900040BBCEB92846236843F40033236002B04F
:10F7A000BDE8F0812368D900D5D423689A0336D503
:10F7B0000126D4E70C20236843F400332360FFF7CD
:10F7C00051FA4FF0FF30EAE74FF480324FF0FF3349
:10F7D0001146384606F024F898B1236843F4003304
:10F7E0002360ECE70198FFF7D9FD2368052043F477
:10F7F00000332360E3E71620FFF734FA4FF0FF30C1
:10F80000CDE7384606F080F803460028C2D04068AD
:10F810000028BFD0C3F80480DFE77320CFE70920BA
:10F82000CDE70920FFF71EFA4FF0FF30B7E700BF22
:10F83000F0B5012985B068D01E4640F205239942F3
:10F8400040F095800746154606F05EF8044600280D
:10F8500000F0B280012D19D0022D10D02A250368A6
:10F8600023F4800323602368284623F400032360E5
:10F87000FFF7F8F94FF0FF35284605B0F0BD16B197
:10F880000A9B012B49D023681625E9E7002EFAD000
:10F890000A9B042BF7D1002103A8FFF751FD054671
:10F8A00000286AD10398082229460C300AF0B2FBDE
:10F8B000039831460A9A0C300AF082FB0823039819
:10F8C00047F20201037245728572C572236843F4E0
:10F8D00080032360FFF74CFD002851D14FF4000254
:10F8E0004FF0FF331146384605F09AFF05460028D1
:10F8F0003BD1384606F008F800284FD04368002B6B
:10F900004CD000221D4642602FE00A9C009406F075
:10F9100023F80546284605B0F0BD002103A8357838
:10F92000FFF70EFD48BB012D08BF264B4FF0040228
:10F9300008BF1D700023039847F201014372C560A0
:10F940008372C3720272236843F480032360FFF75B
:10F950000FFD0646A0B94FF400024FF0FF331146E9
:10F96000384605F05DFF054680B1236878E72A2018
:10F97000FFF778F94FF0FF357EE723680C256FE736
:10F980000398FFF70BFD0525236869E7384605F066
:10F99000BBFF40B1456835B14660E6E73146042219
:10F9A00009480AF00DFB236823F4800323602368D1
:10F9B00023F4000323605FE70920FFF753F94FF0BA
:10F9C000FF3559E77B5402208C3E0220F0B5012917
:10F9D00083B0089E30D01F4640F20523994234D1AF
:10F9E000154605F091FF002837D0012D15D0022DC6
:10F9F0000BD187B3336873B30023012218461A4929
:10FA000009783970326003B0F0BD0920FFF72AF998
:10FA10004FF0FF33184603B0F0BDE7B13368032B56
:10FA200019D93846042211490AF0CAFA00230422DF
:10FA30001846326003B0F0BD009605F0C3FF0346E0
:10FA40000028E3D1184603B0F0BD2A20FFF70AF9D9
:10FA50004FF0FF33DEE71620D8E70920FFF702F961
:10FA60004FF0FF33D6E700BF7C5402208C3E0220CB
:10FA700010B5044605F048FF38B1204605F082FE77
:10FA80000023054A1846136010BD0920FFF7EAF865
:10FA90004FF0FF3010BD00BF903E0220006804F020
:10FAA000D1BA00BFF0B583B00F461546064605F043
:10FAB0002BFF002847D0036804469B0343D5036807
:10FAC000294623F400330360036801A843F40013BC
:10FAD000236004F08DFAA0BB0422019B1A725872B5
:10FAE0009872D872DE6085B91846012104F094FA44
:10FAF000D0B94FF40032304611464FF0FF3305F0D5
:10FB00008FFEA8B9284603B0F0BD394618682A46CA
:10FB10000AF056FA0121019804F07EFA0028E8D094
:10FB2000019B186804F08EFA019804F083FA2320F0
:10FB3000236843F400332360FFF794F84FF0FF305D
:10FB4000E1E70C20F4E71620F6E700BF04F04ABA1C
:10FB50002DE9F041002582B002AB43F8085D8046F4
:10FB60000F461846164602211D4A05F0ADFD009BC2
:10FB700004460BB3C3E903875E61294601A804F07C
:10FB800037FAE8B90422019B052158729872D8729D
:10FB90001A72DC60184604F03FFAD8B902224FF01E
:10FBA000FF331146204605F03BFE054648B9009A52
:10FBB000136843F400331360204602B0BDE8F081BF
:10FBC0000C25204605F0DEFD2846FFF74BF84FF0E8
:10FBD000FF34F1E7019804F02DFA2325F1E700BF87
:10FBE0009DFA0000F0B583B0064605F08DFE0028B2
:10FBF0003DD00D2307680360036804469B031FD4B0
:10FC0000002101A804F0F4F920BB0422019B062185
:10FC100058729872D8721A72DE60184604F0FCF9B5
:10FC2000D0B90E224FF0FF331146304605F0F8FDF3
:10FC30000546A8B9304605F0A5FD284603B0F0BD3D
:10FC40000368002123F40033036001A804F0D0F915
:10FC50000028DAD00C2503E0019804F0EBF9232505
:10FC600027602846FEF7FEFF4FF0FF35E5E7162533
:10FC7000F7E700BF2DE9F04184B0884615461E46DF
:10FC8000074605F041FE002849D00023CDE9008554
:10FC900016F002050446CDE902330ED01EE0002D19
:10FCA00033D14FF48032236A1146002B08BF4FF046
:10FCB000FF33384605F0B4FD05462368E06923F4B8
:10FCC00080332360036832469B6869469847B0F1E9
:10FCD0000008E4DB404604B0BDE8F0810368C06979
:10FCE00023F480332360036832469B686946984753
:10FCF000B0F10008EEDAB8F1FF3FEBD12320FEF7B8
:10FD0000B1FF404604B0BDE8F081B8F1FF3FE1D15A
:10FD10002846FEF7A7FF404604B0BDE8F081162054
:10FD2000FEF7A0FF4FF0FF38D4E700BF05F04ABE52
:10FD300005F012BE70B5064684B0C0680D4605F0E9
:10FD4000E3FD044648B303689BB2012B1FD0036850
:10FD50009BB20D2B29D003689BB2022B2DD0033D03
:10FD6000012D17D8002573683268CDE90255CDE919
:10FD70000023E069694603685B689847013019D041
:10FD80002846236843F48033236004B070BD022DFD
:10FD9000E5D10560002004B070BD30680028F9D0BE
:10FDA00004F050F9204604B070BD022DD7D10E23C7
:10FDB0000360EFE7022004B070BD03689B02CED55C
:10FDC000022DCCD1036823F400130360036843F4CD
:10FDD00000330360DEE700BF50F8081B090C01F098
:10FDE0002FB900BF014805F0F3BE00BFFCBC010005
:10FDF000002310B582B0019358B1044601AA062031
:10FE000006F01EF918B9019B0BB10833236002B04C
:10FE100010BD072002B010BD11F4704F0BD160B1BE
:10FE2000034630F8082C062042EA014143F8081D39
:10FE3000194606F0EDB80F2070470720704700BF45
:10FE400020B1A0F10801062006F02CB90720704768
:10FE500018B10146062006F037BA0720704700BFE8
:10FE60002DE9F04FDFF8CCC083B000900CF13C0BD3
:10FE7000DCF808302BB1DCF80020009C1078A042A0
:10FE800006D00CF10C0CE345F2D103B0BDE8F08FC5
:10FE9000DCF804A003EB0A08C245F2D25368CDF89F
:10FEA00004C0D6469C46D2F810909789AEEB0A0063
:10FEB000DFB3B9F8022090421CD36546002409F153
:10FEC000040303E05A880433824215D833F8046CE3
:10FED0000134A74202FB0655A0EB02001E46F1D1F9
:10FEE000002081420DD00EF1010EF045DED1DDF88B
:10FEF00004C0C6E765464E46338800FB0350814286
:10FF0000F1D1BEF5007FDDF804C0BAD00123084A64
:10FF10004FEA5E1152F821000EF01F0E03FA0EFE9A
:10FF20004EEA000042F82100AFE73846D9E700BFAB
:10FF3000943E0220D83E0220002850D06D4BD3F8CA
:10FF4000882090424BD82DE9F04FD3F88CB083B085
:10FF5000BBF1000F54D00BF1FF32914600264FF059
:10FF60001208654F01920BF1110E06EB090253F8CE
:10FF700038400132520804EB440C02F1120153F8EC
:10FF8000315057F82CA053F83E4003EBC80CDCF876
:10FF900004C005EB450504EB4404DAF810A057F85B
:10FFA000255057F824403AF82CA003EBC10103EB8D
:10FFB000CE0C49682D692469DCF804C0504535F839
:10FFC000215034F82C1015D9884211D2A84208D9F2
:10FFD000561CB145C0F0878002F11308C5E7002028
:10FFE000704702F1FF394E457DD802F1110EBCE792
:10FFF00009F10106B34507D0102E01D0B34508D84A
:020000040001F9
:10000000002003B0BDE8F08F019A102A18BF1646F1
:10001000F6D0DFF8E8C003EBC608D8E9242402EBE9
:10002000420257F8223007EB8202D2F804E01D6941
:10003000002C56D02A467046A40005EB04095188CE
:10004000043291450844FAD12919B1F802A082443A
:10005000824518D941095CF8212000F01F0422FADA
:1000600004F919F0010F07D013E05CF8212022FAFF
:1000700004F919F0010F0CD1013082454FEA5011FB
:1000800000F01F04F1D101365E4508F10808C4D321
:10009000B6E7012606FA04F49E8922EA0402A0EBE0
:1000A0000E004CF821205C68002EA9D06A8882429C
:1000B00011D800212B1D03E05A88043382420AD84C
:1000C00033F8045C01318E4202FB0544A0EB0200D0
:1000D0001D46F1D194E72B8800FB034003B0BDE837
:1000E000F08F7046B0E7BBF1100F08BF0F2690D01D
:1000F00086E700BF143F0220D83E0220943E022033
:1001000000284CD06B4B1A68904248D82DE9F04F2C
:100110005F6883B00097002F51D07A1E9646002169
:100120004FF0010C644C019201EB0E02013253F8C6
:100130003C50520802F1010805EB450553F8379091
:1001400054F825A053F8386009EB490503EBCC09B6
:10015000D9F8049006EB4606DAF810A054F82660A9
:1001600054F825503AF829A003EBC80B03EBC70954
:100170003669DBF804B02D69D9F80490504536F89B
:100180002B6035F8295013D9A84210D2B04208D9B3
:10019000C6454146C0F0878008F1010CC4E7002045
:1001A000704702F1FF3E71457DD81746BCE73946DE
:1001B000009A8A4207D0102901D08A4208D800202C
:1001C00003B0BDE8F08F019A102A18BF1146F6D08F
:1001D000DFF8E8C0DDF8009003EBC108D8E902269B
:1001E00002EB420254F8223004EB8202D2F804E01F
:1001F0001F69002E55D03A467046B60007EB060A36
:100200005588043292452844FAD1BD19B5F802B098
:100210008344834518D945095CF8252000F01F0662
:1002200022FA06FA1AF0010F07D013E05CF8252035
:1002300022FA06FA1AF0010F0CD1013083454FEA79
:10024000501500F01F06F1D10131494508F10808A9
:10025000C4D3B4E70121B1409E8922EA0102A0EB98
:100260000E004CF825205C68002EA8D07A888242C7
:1002700011D800213B1D03E05A88043382420AD87A
:1002800033F8045C01318E42A0EB020002FB05440E
:100290001F46F1D193E73B8800FB034003B0BDE864
:1002A000F08F7046B1E7009A102A08BF0F218FD057
:1002B00085E700BF143F0220D83E0220943E022072
:1002C00070B5002201253348510950F8214002F051
:1002D0001F0305FA03F301322343B2F5007F40F810
:1002E0002130F1D100242C4B21463C222B481C60AC
:1002F00009F090FE10210522294B2A4EC3E9004443
:10030000D9605961D9615962D9625963D963596415
:10031000D9645965D9655966D9665967D9679A60AC
:100320001A619A611A629A621A639A631A649A64E9
:100330001A659A651A669A661A679A67C3E9202150
:10034000C3E92244C3E92421C3E92621C3E92821C2
:10035000C3E92A21C3E92C21C3E92E21C3E93021B5
:10036000C3E93221C3E93421C3E93621C3E9382185
:10037000C3E93A21C3E93C21C3E93E21C3F8041192
:10038000C3F80021C3F80C11C3F8082120463570CA
:1003900070BD00BF943E0220D43E0220D83E022011
:1003A000143F02207D5402202DE9F04F874B87B087
:1003B0001B78002B00F08C8028B321B30B78DFF87A
:1003C000188203EB031308EBC3035B68B1F80CC09E
:1003D0006344102B11D84FF0000A89467C4B7D4FA7
:1003E0001B684FEA8C0E0093B96891B10AF1010ABB
:1003F000BAF1050F07F10C07F6D148F2071B584672
:1004000007B0BDE8F08F48F20E1B584607B0BDE8B4
:10041000F08FBCF1000F61D00D460C46D9F81030BA
:100420000EEB030B5A8833F8046B15449B4502FB13
:100430000644F7D1D9F80830A342D7D3009B2B4408
:10044000B3F5007FD2D2634C0AEB4A029200C0F8A7
:1004500000A0A01844F80290009A8B46C0E901253C
:1004600099F801205A48012A0360C8D0B9F80C3025
:10047000002BC4D00025CDF80490CDF80CA0CDF809
:1004800014B0019B1F781A693B0103EB0709009325
:1004900008EBC903596832F82540029139BB039A29
:1004A000DD609A60009B3B441F4608EBC3014B682C
:1004B00058F83720013394424B6012D9019B48F819
:1004C00037409B8901359D42DBD3DDF814B096E7B8
:1004D00048F2081B584607B0BDE8F08F009B654600
:1004E000AEE7019B01359B89AB42CAD8EDE70026F8
:1004F00001F1FF3A049506EB0A0009EB060201320E
:10050000013058F832C04008324D09EB000109EBC8
:100510000A03013101330CEB4C0C58F831E055F86B
:100520002CB058F833C008EBC2020EEB4E0E0CEBA9
:100530004C0CDBF810B0526855F82EE055F82CC082
:1005400008EBC10108EBC3033BF82220DEF810E002
:100550004968DCF810C05B6894423EF821103CF812
:1005600023302DD99C422DD28C4224D9461CB24531
:10057000C1D21026049D029AB24211D9009B3B447D
:100580001A44334408EBC20A08EBC3090822514657
:100590000AEB0200AAF1080A09F012FDD145F5D1D3
:1005A000009B03993B443344013308EBC30248F8F2
:1005B0003310556076E700F1FF3A56459BD9D8E7EE
:1005C000049DD8E7049D0AF10106D4E77D5402207A
:1005D000D43E0220D83E0220143F0220034B1B7859
:1005E0000BB1FFF78DBD1846704700BF7D54022048
:1005F000044B1B7823B118B101460020FFF730BC33
:10060000704700BF7D540220034B1B780BB1FFF7EE
:1006100093BC1846704700BF7D540220044B1B78E2
:1006200023B118B101460120FFF71ABC704700BF83
:100630007D54022050F8081B090C04F0C3BD00BF14
:10064000014805F0C5BA00BF0CBD0100002310B57C
:1006500082B0019358B1044601AA042005F0F0FCD1
:1006600018B9019B0BB10833236002B010BD0720FD
:1006700002B010BD01F47043B3F5E04F0BD160B18F
:10068000034630F8082C042042EA014143F8081DD3
:10069000194605F0BDBC0F2070470720704700BF0A
:1006A00020B1A0F10801042005F0FCBC0720704730
:1006B00018B10146042005F007BE0720704700BFAF
:1006C0002DE9F0470C460B68464F23F400330B60CE
:1006D0000B68C60023F480130B6007EB060A82B098
:1006E000DAF80430896947F281020546D4F80080BF
:1006F00003F0C6FC00286FD0DAF804208146002AF7
:100700005FD1394B711903EB8101242209F11400E7
:1007100009F056FCD9F8083049462433C9F80830A6
:1007200022684346120C120442F00A02226020465C
:1007300047F2810203F0C4FC034670B92368DB0072
:100740000FD44FF0FF334FF6FF720B21284603F012
:10075000CBFC034650B1C4F80080184602B0BDE897
:10076000F0877323184602B0BDE8F0874FF080622F
:100770004FF0FF331146284603F0B6FC034630BB6A
:1007800057F8350038B10193FFF732FF019B3E4423
:10079000736047F835301846226822F08062226084
:1007A0002268120C120442F00C022260226842F409
:1007B00000322260226842F48012226002B0BDE85A
:1007C000F08757F83510006809F0FAFB99E7732BAA
:1007D000C3D0C4F80080C0E70C23184602B0BDE8BF
:1007E000F08700BF684102202440022000207047AB
:1007F00038B520F00803022B06D02F20FEF732FA7E
:100800004FF0FF35284638BD14464A1E012A28D825
:1008100014BB012906BF01234FF482744FF487747F
:100820001A4603F08DFC051E26DB154B05EBC500B3
:1008300003EB80002422134909F0C2FB284605F08F
:1008400063F80368446123F480130360036823F4AE
:1008500000330360284638BD012908D0B4F5877FEE
:10086000DED01620FEF7FEF94FF0FF35CAE7B4F5EB
:10087000827FF6D10B46D3E74FF0FF35C2E700BFCA
:10088000244002201CBD010038B5044605F03CF8A8
:1008900080B10B4D55F8340038B1FFF7A9FE0023A5
:1008A00005EBC40245F8343053602046BDE83840BB
:1008B00003F0F2BC0920FEF7D5F94FF0FF3038BD48
:1008C000684102202DE9F0470D46DDE9088916460A
:1008D0001F46044605F018F800283BD003689BB279
:1008E0000C2B39D003689BB20B2B11D1204B04EB9E
:1008F000C40413F82430022B38D00369012B14BF31
:1009000039202A20FEF7AEF94FF0FF30BDE8F0871E
:100910000369012B0BD0022B01D03920F2E70368C9
:100920009BB2022B07D003689BB2042B03D0036851
:100930009BB2052BF1D10E4B04EBC40213F822300D
:10094000022BEAD101462046FFF7BAFE002803D069
:10095000D8DCD9E70920D5E7CDE908893B463246FE
:1009600029462046BDE8F04703F006BD2320C9E72D
:10097000244002202DE9F0470D46DDE9088916469E
:100980001F46044604F0C0FF002838D003689BB21D
:100990000C2B0FD003689BB20D2B0BD00369012BDE
:1009A0001AD0022B10D02320FEF75CF94FF0FF3055
:1009B000BDE8F087CDE908893B4632462946204606
:1009C000BDE8F04703F012BE03689BB2022B07D0CC
:1009D00003689BB2042B03D003689BB2052BE2D1C2
:1009E000084B04EBC40213F82230022BDBD1014682
:1009F0002046FFF765FE0028DCD0D5DCD6E70920CD
:100A0000D2E700BF244002202DE9F84F0C461746DC
:100A1000064604F079FF00286DD0036805469BB2B6
:100A2000022B5AD121463A46304603F0B5FF044620
:100A3000002848D1F700DFF8C480BB1918F823302C
:100A4000012B02D02046BDE8F88FDFF8B4B047F2A2
:100A500081020BEB070ADAF80430A969304603F08B
:100A60000FFB8146002844D0DAF80420002A3AD14E
:100A7000B91908EB8101242209F1140009F0A0FA48
:100A8000D9F8083049462433C9F808302A680423C5
:100A9000120C120442F00A022A60284647F2810230
:100AA00003F00EFBE8B92B68DB0018D430464FF09A
:100AB000FF334FF6FF720B2103F016FB0028C1D065
:100AC000042304462B60002CBCDD20464FF0FF348D
:100AD000FEF7C8F82046BDE8F88F2D24F5E773240B
:100AE000F3E70446EFE75BF83610006809F068FAB0
:100AF000BEE70C24E9E70924E7E700BF2440022011
:100B000068410220F8B50E461746044604F0FCFE84
:100B1000E8B1134B04EBC40213F82230022B1CD1B2
:100B2000036805469BB2022B03D003689BB2042BDB
:100B300013D13A463146204603F084FE10B1002816
:100B400006DCF8BD29462046FFF7BAFDF7E7092085
:100B5000FEF788F84FF0FF30F8BD2D20F8E700BF12
:100B6000244002202DE9F04F83B00191054604F0A6
:100B7000CBFE002879D003690446012B73D10368AA
:100B80009BB2042B5FD023689BB20B2B6BD1EE0082
:100B9000374F731917F82330012B64D10122DFF886
:100BA000D4907319EE0007F8232009EB0608A16919
:100BB000D8F8043047F281022846D4F800A003F0A8
:100BC0005FFA834600284CD0D8F80420002A42D18E
:100BD000711907EB810124220BF1140009F0F0F9DF
:100BE000DBF8082059462432CBF808202268534607
:100BF000120C120442F00A022260204647F28102DF
:100C000003F05EFA68B92368DB000FD44FF0FF33BE
:100C10004FF6FF720B21284603F066FA70B1C4F854
:100C200000A0002803DC03B0BDE8F08F7320FEF7BE
:100C300019F84FF0FF3003B0BDE8F08F0199284656
:100C400003F040FFEDE7EE00094F731917F823306A
:100C5000022B98D1A2E759F83510006809F0B0F9D5
:100C6000B6E70C20E3E72D20E1E70920DFE700BF2E
:100C70002440022068410220F8B50C4616461F4663
:100C8000054604F041FE00283BD0006880B20628EB
:100C900037D121463B463246284603F089FF0446B9
:100CA00018B1002C2EDC2046F8BD284604F02CFE9E
:100CB0000368184F23F400330360036805EBC50590
:100CC00023F480130646036007EB8501242238468F
:100CD00009F076F902233B70336820461B0C1B0495
:100CE00043F00B0333604FF6FF724FF0FF330C21DC
:100CF00003F0FAF904460028D5D0002003F0CCFA1E
:100D0000CFE7092420464FF0FF34FDF7ABFF204624
:100D1000F8BD00BF244002202DE9F041B1F58D7FE0
:100D2000069E1ED11F460546002B00F08C80904683
:100D300004F0EAFD00287BD00468A4B2022C07D09E
:100D400003689BB2042B03D003689BB2052B6FD1C1
:100D500008F1FF32042A7CD8DFE802F0244E324149
:100D60000700BDE8F04104F05BB83B4C54F8350097
:100D700038B1FFF73DFC002204EBC50344F83520F1
:100D80005A6030464EB3FFF729FC44F8350000287E
:100D900057D004EBC50432463946666009F010F9B5
:100DA00000201AE0042E4AD13868002839D00128E2
:100DB00045D12A4A05EBC50402F8240000200CE0C6
:100DC000012E3CD13A780020003218BF0122234B7B
:100DD00005EBC50403EB84046270BDE8F081042ECA
:100DE0002DD13A68022A2AD81C4B05EBC50403EB27
:100DF0008404A2700020F0E75FEA960C1FD016F082
:100E000003041CD105EBC505AD00144B281D184487
:100E10002B443246394683F803C009F0D1F8204606
:100E2000DBE702210D4A05EBC50402F82410D4E7E4
:100E30000920FDF717FF4FF0FF30BDE8F0811620C5
:100E4000F7E70C20F5E70E20FDF70CFF4FF0FF3021
:100E5000C3E72A20EDE700BF6841022024400220BA
:100E60002DE9F041B1F58D7F069F12D11D466BB182
:100E700067B10646144604F047FD00284FD0013CF8
:100E8000032C52D8DFE804F0392115090E20BDE803
:100E9000F081BDE8F04104F07FB83B68042B3CD101
:100EA000234B06EBC60603EB8606B37800202B60C7
:100EB000EDE73B68012B30D11D4B06EBC60603EB7B
:100EC0008606737800202B70E1E706EBC60618490A
:100ED0003B68B6008A1913F00304D07821D19B082F
:100EE000834228BF03469A00DBB1043631443A609E
:100EF000284609F065F82046C9E73B68042B0CD169
:100F00000B4B06EBC60613F826300020A3F10103B5
:100F1000B3FA83F35B092B60B9E71620B7E7092022
:100F2000B5E70028F9D13860B1E72A20AFE700BF64
:100F300024400220F8B548F28105AB420C4662D04D
:100F400049F282018B4206462ED048F202018B42C2
:100F500001D00120F8BD002CFBD06369B3F5827F7E
:100F600002D0B3F5877FF4D1236823F000532360C8
:100F70005569002D56D123681B0C1B0443F0050353
:100F800023602368DA000DD52B4B06EBC60213F85D
:100F90002230022B06D130462146FFF791FB08B1E3
:100FA000732842D10020F8BD002CFBD023689BB2EF
:100FB0000B2BF7D11569002D34D1236843F08063E2
:100FC00023602368DB00EDD51C4F57F8300030B1AB
:100FD000FFF70EFB07EBC60347F836505D6023684A
:100FE000002023F08063236023681B0C1B0443F064
:100FF0000C032360236843F400332360236843F425
:1010000080132360F8BD0029CCD00B689BB20A2B5B
:10101000C8D1506938B90B681B0C1B0443F00B0393
:101020000B60F8BD284603F021F8606023680020BB
:1010300043F480232360F8BD24400220684102204D
:1010400008B5084AC16812880346B2EB114F05D0B3
:10105000006810B1FEF7FCFE002008BD024A012026
:10106000136008BD544C0220B4410220002310B587
:1010700008480949094A0A4C03800B601360236041
:10108000FEF7B0FE10B90123236010BD4FF0FF3012
:1010900010BD00BF544C0220B4410220B0410220D8
:1010A000A8410220012808B50BD140F203239A423F
:1010B00007D1094B1A68012A09D102221A60074890
:1010C00008BD1620FDF7CEFD4FF0FF3008BDFDF73F
:1010D000C9FD4FF0FF3008BDA841022032547649C7
:1010E000F0B5324C83B023689A1E012A57D8032BDF
:1010F00004D001230020236003B0F0BD0021684626
:10110000FEF776FE034600283DD10421284E0098C4
:1011100032880172013292B2110441F00601254D6C
:10112000C160037143718371C37143728372C3726F
:10113000062132802B60FEF76FFED8B94FF0FF33E7
:1011400002AE274646F8043D04E031463846FDF736
:10115000F5FCF0B928680028F7D00569FEF770FEA5
:10116000002DC6D0144B08201D60FDF77BFD4FF00D
:10117000FF30C1E7009803681BB11846FEF768FE10
:101180000098FEF75DFE0C20FDF76CFD4FF0FF3080
:10119000B2E73C20FDF766FD4FF0FF30ACE70120E1
:1011A000FDF760FD4FF0FF30A6E700BFA841022029
:1011B000544C0220B4410220AC4102202DE9F047FA
:1011C0005A4E1546336882B09A1E012A00F2A78053
:1011D0000F46002900F09D80002D00F09A80022B20
:1011E000E8464ED040462946FEF702FE064640B18C
:1011F0000C20FDF737FD4FF0FF35284602B0BDE863
:10120000F087009B394618682A4608F0D9FE042169
:10121000474C00982388456001339BB21A04238011
:101220000A43444CC26046728672C67201722660DE
:10123000FEF7F2FD002862D14FF0FF3302AE3B4FC4
:1012400046F8043D04E031463846FDF777FC78B9AE
:1012500020680028F7D00469FEF7F2FD002CCCD0FE
:10126000354B08201C604FF0FF35FDF7FBFCC4E751
:101270004FF0FF353C20FDF7F5FC284602B0BDE8F5
:10128000F08740460021FEF7B3FD02460028AFD1AB
:101290004FF0080C264929480B8804680133009850
:1012A0009BB20B801B0443F003030461214CC36019
:1012B000027142718271C27142728272C27280F88E
:1012C00008C003212260FEF7A7FDC0B94FF0FF332D
:1012D0000DF1080949F8043DB24605E0494650467B
:1012E000FDF72CFC0028C3D120680028F6D0046943
:1012F000FEF7A6FD002CB3D10323336072E70098FC
:1013000003681BB11846FEF7A3FD0098FEF798FD91
:101310006EE71620FDF7A6FC4FF0FF356DE70120C4
:10132000FDF7A0FC4FF0FF3567E700BFA8410220A2
:10133000544C0220B4410220AC410220B0410220B2
:10134000F0B5464883B000680238012877D840F2EB
:10135000032081426DD1043A032A5CD8DFE802F011
:101360004B024E510724254600216846FEF740FDFA
:101370000346002838D10427394E00983288294680
:10138000013292B244EA0245364CC56003714371A2
:101390008371C37143728372C37207723280236098
:1013A000FEF73AFDB8B94FF0FF3302AD2B4E45F8CA
:1013B000043D05E029463046FDF7C0FB002831D149
:1013C00020680028F6D00469FEF73AFD002C3CD1D5
:1013D000204603B0F0BD009803681BB11846FEF725
:1013E00037FD0098FEF72CFD0C20FDF73BFC4FF07D
:1013F000FF3003B0F0BD05242546B5E70824254697
:10140000B2E7B3B1089A042A13D100201A68164B28
:101410001A6003B0F0BD2A20FDF724FC4FF0FF3026
:1014200003B0F0BD3C20FDF71DFC4FF0FF3003B0D2
:10143000F0BD1620FDF716FC4FF0FF30C9E7012084
:10144000FDF710FC4FF0FF30C3E7084B08201C608D
:10145000FDF708FC4FF0FF30BBE700BFA8410220BA
:10146000544C0220B4410220B0410220AC41022081
:1014700040F203202DE9F041814282B0089E40F005
:10148000AE801D46002B00F0AA80002E00F0A78041
:101490005E4B1B68023B012B00F2A780013A132A26
:1014A00079D8DFE802F0175F787878787278787802
:1014B0007878787878787878780A3368042B40F0F0
:1014C0008E8000221046524B19681A60296002B0C3
:1014D000BDE8F0813368242B40F081800124A046D0
:1014E00000216846FEF784FC002846D14949009B4C
:1014F0000A88B8F1030F02F1010292B244EA0244F1
:1015000018710A80DC6058719871D8714BD0042131
:101510000022414F9960184641463A60FEF77CFC34
:1015200000284DD14FF0FF3302AC44F8043DDFF802
:10153000DC8005E021464046FDF700FB002837D15E
:1015400039680029F6D00C69002C54D13268143166
:10155000284608F035FD3868FEF772FC204602B0D8
:10156000BDE8F0813368042B39D10224002168469C
:10157000A046FEF73DFC0028B8D00C20FDF772FB1A
:101580004FF0FF3002B0BDE8F0813368042B26D164
:101590000924A046A4E72A20FDF764FB4FF0FF30A2
:1015A00002B0BDE8F0811D4A082112681A61AFE758
:1015B0003C20FDF757FB4FF0FF3002B0BDE8F08153
:1015C000009803681BB11846FEF742FC0098FEF72E
:1015D00037FC0C20FDF746FB4FF0FF30D2E716201A
:1015E000FDF740FB4FF0FF3071E70120FDF73AFBBC
:1015F0004FF0FF306BE7064B08201C60FDF732FB15
:101600003868FEF71DFC4FF0FF3060E7A84102206C
:10161000AC410220544C0220B4410220B0410220CF
:10162000704700BF08B5FFF7FBFF08BD10B5064CBB
:1016300023782BB900F026F808B90123237010BDD8
:101640004FF0FF3010BD00BF7E54022010B5054C96
:10165000237823B100F07CF800B9207010BD4FF062
:10166000FF3010BD7E5402200FB408B52D20FDF7C9
:10167000F9FABDE808404FF0FF3004B0704700BFF2
:10168000FFF7D0BFF0B593B0FEF71AFE00284CD19B
:10169000284901A8FEF788FE002846D1FDF798FBEF
:1016A00004F08CFA002840D120234FF48041082216
:1016B0004FF4405C204F214E039305930793204D38
:1016C00009910D911F4C2049204BCDE910000DEBE5
:1016D0000200CDF82CC0CDE90E22029704960695A3
:1016E00008940A910C9300F0E7FB08B113B0F0BD29
:1016F00003F0DEFFC8B9FEF729FAB0B902F008FD21
:1017000098B9FFF773F880B9FFF7B0FC68B901F03A
:10171000C3FA50B905F01CFD38B9FDF7D9FE003009
:1017200018BF0120404213B0F0BD4FF0FF3013B09E
:10173000F0BD00BF98BE0100000001204000012064
:101740002000012060700120600001206030012035
:1017500008B504F065F900F013FC002008BD00BFD7
:1017600005282AD008B514D90A2816D066280BD126
:1017700040F202239A4232D040F205239A4232D0FC
:1017800040F201239A422CD01620FDF76BFA00207C
:1017900008BD012816D00228F6D1A2F582720A2AC5
:1017A00019D8012340F20341104803FA02F20A4219
:1017B00000F1280318BF184608BD03290C4818BFBC
:1017C0000020704740F203239A4206D0B2F5017F11
:1017D000DAD1084808BD054808BD074808BD0748D4
:1017E00008BD074808BD074808BD00BF68BD010027
:1017F00058BE010008BE0100B8BD0100E0BD0100F7
:1018000040BD010030BE010038B5054604F07CF84B
:10181000044650B92A4BAB4332D02A4BAB4343D09A
:10182000294BAB4346D1294838BDC3684269052BD3
:1018300034D011D90A2B13D0662B2AD140F20223BF
:101840009A4231D040F205239A4231D040F201232E
:101850009A421ED11E4838BD012B13D0022B18D13D
:10186000A2F582720A2A21D8012340F203411948C5
:1018700003FA02F20A4200F1280418BF204638BDDC
:10188000154838BD40F203239A42F9D0B2F5017FE2
:10189000C9D01620FDF7E6F9002038BD03690F48CE
:1018A000032B18BF002038BD0D4838BD094838BD8E
:1018B0000C4838BD0920FDF7D5F9204638BD00BFDA
:1018C0003254764900009A784354764908BE0100A4
:1018D00040BD010068BD0100B8BD010058BE010057
:1018E000E0BD010030BE010003F058BB03F04CBC6A
:1018F0002DE9F04342EAE27283B00092002848D01A
:101900004B1E082B45D880460546002400EBC10736
:10191000AB88286803F0030301A943F01C0604F018
:1019200001F8019B0835334025F8023C03B101342E
:10193000AF42EDD19CBB69464046FDF7FFF8074634
:1019400008B13C281DD1C1460026B9F80430D9F8A9
:10195000000003F0030301A943F01C0403F0E2FFBD
:10196000019B09F10809234029F8023C03B1013623
:101970004D45EAD10EB9002FDDD0304603B0BDE8A9
:10198000F0832320FDF76EF94FF0FF3003B0BDE880
:10199000F0831620FDF766F94FF0FF30EEE72046A2
:1019A000ECE700BF08B5064B834303D0BDE8084011
:1019B00004F06AB82D20FDF755F94FF0FF3008BD4F
:1019C00032547649014B1860704700BFC441022071
:1019D000F0B56C4B83B01B78002B00F0AD806A4BE8
:1019E0001C68A26863689A422DD04BF6EF63ADF88D
:1019F000003023786E468DF80430636805219A42E2
:101A00002ABF27699F1ABF1A9A4294BF0025E5682A
:101A1000BFB288BF5B1B304688BF9DB2ADF8027075
:101A200008F0D1FEBDF80210A06808F0CCFEA36853
:101A300022691F44974208BFE368A76008BFA360FC
:101A4000002D40F08D80514B1C68A26863689A425B
:101A50002CD04BF6EF63ADF8003023786E468DF84E
:101A60000430636805219A422ABF27699F1ABF1A6A
:101A70009A4294BF0025E568BFB288BF5B1B304621
:101A800088BF9DB2ADF8027008F09DFEBDF802104F
:101A9000A06808F098FEA36822691F44974208BF17
:101AA000E368A76008BFA360002D48D1384B1C68CD
:101AB000A26863689A422BD04BF6EF63ADF8003012
:101AC00023786E468DF80430636805219A422ABF58
:101AD00027699F1ABF1A9A4294BF0025E568BFB2D2
:101AE00088BF5B1B304688BF9DB2ADF8027008F01E
:101AF0006AFEBDF80210A06808F065FEA3682269BE
:101B00001F44974208BFE368A76008BFA3600DB9F0
:101B100003B0F0BD30460521ADF8025008F053FE89
:101B2000BDF80210E06808F04EFEBDF80220E36840
:101B30001344A36003B0F0BDFDF742F94FE7052160
:101B40003046ADF8025008F03EFEBDF80210E068E5
:101B500008F039FEBDF80220E3681344A360A5E74E
:101B600005213046ADF8025008F02DFEBDF80210F8
:101B7000E06808F028FEBDF80220E3681344A36083
:101B800061E700BF7F540220C0410220B84102201B
:101B9000BC41022000222DE9F04FB04B83B01B68FE
:101BA00019695C69187C1A74587C5A74987C9A7408
:101BB000D87CDA74187D1A75587D5A75987D9A7597
:101BC000D87DDA75B9B10139032914D8DFE811F0ED
:101BD000D6000301040016000125032000226FF047
:101BE0005F019F4C25701C7A1872587A5A72987A45
:101BF0009A72DA7AD97203B0BDE8F08F042100221C
:101C00006FF05F001C7A1972597A5A7294499C7A63
:101C10009A72DC7AD8720A700B78002B00F0178168
:101C2000904B1C68A26863689A422DD04BF6EF6314
:101C3000ADF8003023786E468DF8043063680521D6
:101C40009A422ABF27699F1ABF1A9A4294BF002559
:101C5000E568BFB288BF5B1B304688BF9DB2ADF858
:101C6000027008F0B0FDBDF80210A06808F0ABFDEE
:101C7000A36822691F44974208BFE368A76008BFB2
:101C8000A360002D40F0D280774B1C68A268636887
:101C90009A422DD04BF6EF63ADF8003023786E46B4
:101CA0008DF80430636805219A422ABF27699F1A7C
:101CB000BF1A9A4294BF0025E568BFB288BF5B1B7C
:101CC000304688BF9DB2ADF8027008F07CFDBDF8CB
:101CD0000210A06808F077FDA36822691F449742AC
:101CE00008BFE368A76008BFA360002D40F08D80A7
:101CF0005E4B1C68A26863689A423FF47CAF4BF667
:101D0000EF63ADF8003023786E468DF804306368D9
:101D100005219A422ABF27699F1ABF1A9A4294BF87
:101D20000025E568BFB288BF5B1B304688BF9DB207
:101D3000ADF8027008F047FDBDF80210A06808F089
:101D400042FDA36822691F44974208BFE368A76069
:101D500008BFA360002D3FF44EAF05213046ADF81B
:101D6000025008F030FDBDF80210E06808F02BFDCD
:101D7000BDF80220E3681344A3603CE7384A1178B9
:101D800009B100211170A568002D39D04FF0000C69
:101D9000DFF8D4A0DFF8CCB03449E14666466246AD
:101DA000D1F800E0DAF80080DBF8007008E0632981
:101DB00016D0612904BF074601260132AA4213D07A
:101DC000911C04EB8101486801786229EFD18046BB
:101DD0004FF00109F1E7FCF7EBFF03B0BDE8F08F2E
:101DE00086464FF0010CE8E7A6BBB9F1000F01D021
:101DF000CAF80080BCF1000F02D01C4AC2F800E013
:101E0000012000226FF05F01EDE605213046ADF8BC
:101E1000025008F0D8FCBDF80210E06808F0D3FCCE
:101E2000BDF80220E3681344A36061E70521304652
:101E3000ADF8025008F0C7FCBDF80210E06808F0E9
:101E4000C2FCBDF80220E3681344A3601CE7FCF762
:101E5000B7FFE5E6CBF80070C7E700BFC44102203A
:101E60007F540220C0410220B8410220BC41022020
:101E7000014B1878704700BF7F5402200020704744
:101E80000B4BD3E90023134498420DD282420BD866
:101E900010B5044600F0FCFD40B1064A84600260C3
:101EA000BDE8104000F03CBDFEF7B8BB10BD00BF60
:101EB000C84102200100020000282BD030B589B0B3
:101EC00001AA6946044600F041FC034640B1134AAA
:101ED00004F1280003C882E80300184609B030BDA9
:101EE000DDE90012204600F057F803460028EED145
:101EF0000B4B0C490C480D4A03930D4D0D4B0491AF
:101F000005900D4902A807930695029203F0D8FFA9
:101F10000346DCE70E231846704700BFC841022085
:101F2000212A0100F12A0100B52501002129010023
:101F3000811E01007D1E0100D041022060B108B564
:101F40004368DBB2022B0ED003681B0C022B05D0BA
:101F5000042B0ED0002008BD002070478068FEF7DB
:101F60005DFB002008BD0146BDE80840034803F0C2
:101F700099BE024804F004F8002008BDD0410220B8
:101F800008B500F0BFFD00F04BFB00F0C1FDBDE85F
:101F9000084000F065BB00BF002800F0FF802DE97D
:101FA000F04F056895B0002D00F0EE808368002B9F
:101FB00000F0EA800769002F00F0E680846A002CB8
:101FC00000F0E28044681B2C40F2E380C4680B2CD4
:101FD00040F2DF80D0F814E0BEF1170F40F2D98054
:101FE000002604466F48CDE90012DFF8D8A16E49FB
:101FF0000680A06BDFF8D0C1DFF8D081DFF8D0B168
:10200000DFF8D09172460E60CAF8000031463846BB
:10201000CCF80060CBF80030C8F80060C9F8006068
:1020200007F0F8FFE36938463B60A3697B60FFF780
:10203000C9FC01224FF0040C5C4B5D49C3F81056FB
:102040000968802004915B49DDF810E0C3F814664C
:1020500009682E7003916E70EE70AA700399A16AE0
:10206000DBF800E06960E16A019CA960EC60009C1B
:102070005149AF61C5F814E02C61C3F890250C6894
:10208000A1F592610594059CC3F898C5D1F89844D0
:102090004FF480670694069C1024C3F8A045D1F83D
:1020A000A044464D0794079C4024C3F8A845D1F8A6
:1020B000A8440894089CC3F8AC05D1F8AC04099076
:1020C0000998C3F8006108680A900A98C3F8086183
:1020D00088680B900B98C3F8106108690C900C98F5
:1020E000C3F8186188690D900D98C3F81C61C86920
:1020F00001F501710E900E98D3F804031043C3F854
:1021000004030C682E480F940F9CD3F8044344EA50
:102110000C04C3F804430C681094109CD3F80443D7
:1021200044F01004C3F804430C681194119CD3F8D4
:10213000044344F04004C3F804430C681294129C16
:10214000D3F8044344F08004C3F80443DAF80030C1
:1021500009685B011391DBB21399C8F8002080F87D
:102160002A33C0F8847147600296C5F81066D5F826
:1021700010360293029BD8F80030012BFBD0D9F81F
:10218000000015B0BDE8F08F4CF20E0015B0BDE8B0
:10219000F08F4CF2090015B0BDE8F08F4CF20E0044
:1021A000704700BF564C0220E041022000A00240D0
:1021B00010A6024014A6024090A502400050004024
:1021C00000E100E0D8410220E4410220DC4102208D
:1021D000E8410220D44102202DE9F04F4FF4806500
:1021E000A74C87B0C4F88450BFF34F8FBFF36F8FF5
:1021F000A44EC4F88451D6F80C331F0600F1C880F1
:10220000A04BD3F80C23D00700F1D480D3F80C23D3
:1022100012F0400240F0B680D3F80C13490700F1E9
:10222000E680D3F80C33DA0640F19D800021954A10
:10223000954BC2F810111B680493049BDFF8708261
:10224000924FDFF87092D8F800A0DAF80010002959
:102250003FD00022144602E001348C4227D20AEB20
:10226000C405AB68002BF7D06E68F6B2012EF3D12F
:102270006868B9F80030B3EB104FEDD16A680133EC
:1022800022F0FF0242F002026A60A868A9F800305A
:10229000FFF754FE324628B96B6823F0FF0343F082
:1022A00003036B60DAF8001001348C42D7D3002AA4
:1022B000CDD171B113460AEBC3029068013330B13E
:1022C000D2F804B05FFA8BFBBBF1010F03D08B4255
:1022D000F1D14FF0000BD7F800A0DAF80020002A67
:1022E0003DD000210C4602E00134944227D20AEB93
:1022F000C405AB68002BF7D06E68F6B2012EF3D19F
:102300006868B9F80030B3EB104FEDD16A6801335B
:1023100022F0FF0242F002026A60A868A9F80030C9
:10232000FFF70CFE314628B96A6822F0FF0343F03C
:1023300003036B60DAF8002001349442D7D30029FC
:10234000CDD162B10B460AEBC3018868013320B1DD
:102350004968C9B201293FF476AF9342F3D1BBF18A
:10236000000F7FF470AF4FF48061494B444A1B6803
:102370005B01DBB282F82A33C2F88411516007B0E6
:10238000BDE8F08F0622434B1A6007B0BDE8F08F1E
:10239000FFF700FCFFF76CFD002849D13E4BC6F863
:1023A0001C011B680193019B364BD3F80C23D0070B
:1023B0007FF52CAF002048F202023849C3F8000133
:1023C000096802910299D3F81436934240D01ED87E
:1023D000002B4FD0022B42D948F20102934249D13F
:1023E000032007222B492E4B08601A60CDE7294DA8
:1023F0002968C3F8082101292A495DD00A68039297
:10240000039AD3F80C33DB063FF510AF16E7264AE4
:10241000934214D8B3F1886F14D848F20302934260
:1024200028D1032004221B491D4B08601A60ACE729
:10243000E02384F82A33656007B0BDE8F08F1B4ABB
:10244000934217D103201349154A086013609CE793
:10245000032006220F49124B08601A6095E70323F8
:1024600018460C490E4A0B60136007B0BDE8F04FE8
:10247000FFF706B903230749094A0B60136084E795
:1024800000E100E000A0024010A10240E041022073
:10249000D8410220DC4102201CA1024000A10240E0
:1024A000D441022008A1024004004004010050056C
:1024B000E4410220564C0220374A0B68126805930B
:1024C00093683648364903605468059A0C606BB1CE
:1024D00064B11B68102B02D82268102A0CD9032182
:1024E0004CF206022F4B29601A604EE7032110229E
:1024F0002C4B29601A6048E7DFF8B480002A42D0EC
:10250000002304F104091E4602E0013696422AD255
:10251000F700E11988680028F7D0D1F804A05FFA25
:102520008AFABAF1010FF0D1D1F804C0B8F800006E
:10253000B0EB1C4FE9D14B68421C23F0FF0343F082
:1025400002034B608868A8F80020FFF7F7FC5346A9
:1025500038B959F8072022F0FF0242F0030249F887
:1025600007202268D1E7002BC8D112B90BE09342B3
:1025700009D004EBC301886801330028F7D049680B
:10258000C9B20129F3D10220074B4FF48061074AF9
:102590001B682860ECE600BFE8410220E44102200D
:1025A000E0410220D4410220D841022000E100E0B5
:1025B000564C022030B4184B1C6825686DB1A368D6
:1025C000834227D0002302E08968814219D0013379
:1025D000DA00AB4204EB0201F6D1104B1C6825680F
:1025E0006DB1A368834215D0002302E0896881425F
:1025F00007D00133DA009D4204EB0201F6D130BC72
:1026000070470432A35823F0FF0343F00303A350A1
:1026100030BC70470422F5E7E4410220E04102208B
:1026200010B40024102004220A4B0B49C3F8A04523
:102630000C6883B00194019CA1F52671C3F80803CE
:102640000968064B009100991A6003B05DF8044BCD
:10265000704700BF00A00240A0A50240DC4102205C
:10266000F0B4324A8CB01368062BFCD10020012252
:102670000A212F4B0090C3F81026D3F810060090C3
:102680000098C3F814260191019B2BB1019B013BDB
:102690000193019B002BF9D100220126042510246F
:1026A0002349244BC1F8142601F51531C3F89025B0
:1026B00001F5C8710968402002911F49029FC3F8C3
:1026C00098250F68802103971C4FDDF80CC0C3F8D4
:1026D000A0253F6804971A4FDDF810C0C3F8A8255D
:1026E0003F680597059FC3F8AC25164A1268069205
:1026F000154A069FC3F8086316680796079EC3F835
:10270000085315680895089DC3F808431468099490
:10271000099CC3F8080310680A900A98C3F80813C4
:1027200013680B930B9B0CB0F0BC7047DC4102208C
:102730000050004000A0024098A50240A0A5024021
:10274000A8A50240ACA5024008A30240002800F062
:10275000B880002900F0B580002A00F0B2802DE991
:10276000F04F046A85B0002C00F0A680406A002873
:1027700000F0A28042F687454FF0000A554EA8426D
:1027800086F800A040F2A0800827DFF8809120465C
:1027900016460D4644225146C9F8004007F03AFC5F
:1027A000D9F8002004F14403DFF8648182F801A025
:1027B00082F802A082F803A01770184644225146FE
:1027C000C8F8003007F026FCD8F8002004F1880390
:1027D000DFF840B1177082F801A082F802A082F8F9
:1027E00003A018464FF400725146CBF8003007F0B2
:1027F00011FC394B04F5227CC3F800C051466046F9
:102800004FF4007207F006FC4FF4205C06214FF0F5
:10281000010E4FF401304FF48832304B04F59164CF
:102820005C602F4CC3F808C09981A3F800E01946FA
:102830001C612C4BDFF8E0C020612B48636003F57E
:10284000C073A060C4F800C02848E3606261FDF76F
:10285000ABFD002832D14FF0020C2024D9F8001033
:10286000DBF8002029601C4BD8F80010DFF8ACE042
:102870001F4D3160CEF800201B681E4902F5007222
:102880002A601D4E1D4A1E4D0B6003F500731D4945
:1028900033602880C2F814C509681B4B0391039963
:1028A000C2F81C7519683B4402910299C2F824458C
:1028B0001B680193019B01E04CF2070005B0BDE8E5
:1028C000F08F4CF20E0070474CF2040005B0BDE8EA
:1028D000F08F00BF805402201442022000420220E8
:1028E000244202208000040000010400EC41022088
:1028F000F8410220F4410220F041022000A00240F1
:10290000584C022014A502401CA50240204202207F
:10291000184202201C42022040000800FC41022014
:1029200000285FD070B4334B83B01A68324B8242B8
:102930001ED81B6831498342096803D8304C24688B
:10294000844247D881420ED92E4B1B78002B4CD1A4
:10295000831A2D499E099B060A682C4C4FF00301EF
:102960004FF0020514D04CF2100003B070BC704759
:102970001B689842F7D3224A12689042F3D2012191
:10298000C31A234A9E099B060D461268214CEAD1C0
:102990004368DBB29D4220D1202002EBC6021E4DCF
:1029A00053682E889BB243EA064323F0FF0343F0AB
:1029B0000103536000BF0138FCD10122174B43F8DB
:1029C000212022682B880192019A01332B8003B0C9
:1029D00070BC70478142D2D9B6E74CF2070003B011
:1029E00070BC70474CF20E0070474CF20F0003B001
:1029F00070BC7047FC410220F4410220F8410220E3
:102A0000F041022080540220204202200CA002400B
:102A10001842022004A00240584C022000A00240AC
:102A2000184B1B7863BBF0B4174A03F0FF0014681F
:102A3000164B25681E68A5B10746C10063185A6881
:102A4000D2B2032A04D19F605A6822F0FF025A6072
:102A50005A6812F0FF0F01D19B682BB10130A842D8
:102A6000EBD10020F0BC704706EB80102144886059
:102A7000436823F0FF0343F002034360F0BC704758
:102A80000020704780540220204202201C42022075
:102A9000F0B4154A154B14681E682568ADB10020C6
:102AA0000746C10063185A68D2B2032A04D19F6056
:102AB0005A6822F0FF025A605A6812F0FF0F01D1E3
:102AC0009B682BB101308542EBD10020F0BC7047F0
:102AD00006EB801021448860436823F0FF0343F035
:102AE00001034360F0BC70471842022014420220E8
:102AF000034B1B780BB9FDF787BD0020704700BF63
:102B0000805402200122014B1A7070478054022029
:102B1000F0B4164A164B14681E682568ADB1002241
:102B20001746D00023185968C9B2032904D19F6001
:102B3000596821F0FF015960596811F0FF0F01D168
:102B40009B6823B10132AA42EBD1F0BC70479201DD
:102B50000444B018A0604368064923F0FF0343F023
:102B600001034360B150F0BCFFF7DABE1842022007
:102B7000144202200100030000207047002270B5BB
:102B80000B7884B00E46CDE90022CDE9022223B3B2
:102B90000C46202B0D461BD00B70013214F8013F60
:102BA000B1180D46002BF4D100220D4B2A7053F8BA
:102BB00020300C4A1B6810216846FBF779FA6946F9
:102BC000304607F083F9003018BF012004B070BD13
:102BD00014F8013F002BDCD1E6E70D46E4E700BF27
:102BE0004043022054BF010070B50B78064613B372
:102BF000084600240A46202B154617D013700134CE
:102C000010F8013F0A191546002BF4D1002308469D
:102C10002B703A2107F094F930B1013007F0BAF87F
:102C2000064B53F826305860002070BD10F8013F65
:102C3000002BE0D1EAE70D46E8E700BF4043022061
:102C400070B50B78064613B3084600240A46202BBD
:102C5000154617D01370013410F8013F0A191546B4
:102C6000002BF4D1002308462B703A2107F068F9B5
:102C700030B1084B013053F8264007F08BF8206044
:102C8000002070BD10F8013F002BE0D1EAE70D46AF
:102C9000E8E700BF404302204FF0FF3310B5094C76
:102CA000282200210848236007F0B4F940F20122ED
:102CB00000216620FCF74CFF00282060B4BF0320F1
:102CC000002010BD3C420220404302202DE9F04389
:102CD000662883B040F0BC80B1F5007F40F0AA8048
:102CE00040F202239A4240F0A580624C25684DB321
:102CF0006368002B00F09880A368002B00F096809A
:102D0000E368002B00F094802369002B00F098808A
:102D10006369002B00F09880A369002B00F0968077
:102D2000E369002B00F08E80236A53B1636A0925A2
:102D300043B10C20FBF796FF4FF0FF3003B0BDE826
:102D4000F08308257420FDF749FC44F8250000288D
:102D5000EFD07422002107F05DF9012103204FF02C
:102D6000FF3754F82530444A996054F825304FF421
:102D7000807118675F604148DFF80C81FBF798F9B4
:102D80003E48D8F80090002607F0E8F8334602469F
:102D90003A49484601960096FCF784FE814637483A
:102DA00007F0DCF8484559D13346CDE900664FF4C9
:102DB00080723249D8F80000FCF75CFF06463048C4
:102DC00007F0CCF8864215DB02462C492C4807F068
:102DD000D8F878B929492846FFF732FFB0B902225E
:102DE00054F8253045F0F14040F4D0109A6003B01B
:102DF000BDE8F083234807F0B1F820490246214896
:102E000007F0BFF860B90820FBF72CFF54F8250045
:102E1000FDF7EEFB00234FF0FF3044F825308DE73F
:102E20000520FBF71FFFF1E701258BE7022589E766
:102E3000032587E71620FBF715FF4FF0FF307DE7EE
:102E400004257FE707257DE705257BE7062579E74C
:102E50002F20FBF707FF4FF0FF306FE70520FBF750
:102E600001FF54F82500FDF7C3FB44F82560384600
:102E700064E700BF4043022030BF0100404202200F
:102E800040BF01004CBF01003C4202202DE9F04F41
:102E900083B0002900F03E81642A914600F23A8115
:102EA00005460846884607F059F8642800F2328142
:102EB000A54BAB4340F0258125F0F14525F4D01515
:102EC000092D00F31E81A14F57F82530002B00F08B
:102ED00018819A68002A00F01481002DC0F2118137
:102EE0009B68022B40F00D81994E9A4A4FF48071F5
:102EF0003046FBF7DDF857F825300446C0F5807101
:102F00001B68954A3018FBF7D3F857F8253004446E
:102F10001B6F03F00302032A00F0EA809B0706EB15
:102F20000400C4F580714CBF8C4B8D4B8D4AFBF770
:102F3000BFF8044443468C4AC4F580713019FBF74E
:102F4000B7F82044B0F5807F00F3F780DFF838A2AF
:102F50007F48DAF800B0002407F000F82346024664
:102F60007B49584601940094FCF79CFD83467848C1
:102F700006F0F4FF584508D00520FBF773FE4FF02C
:102F8000FF34204603B0BDE8F08F2346CDE900446E
:102F90004FF480726E49DAF80000FCF76BFE0446CD
:102FA000724806F0DBFF8442C0F291800246684915
:102FB0006E4806F0E6FF002840F089806449284604
:102FC000FFF7DAFD04460028DBD1694A4FF480712F
:102FD0005F48FBF76DF857F82530C0F580711B6826
:102FE000644A3044FBF764F85948DAF800B006F058
:102FF000B5FF234602465649584601940094FCF713
:1030000051FD8346524806F0A9FF5845B4D12346E6
:103010004FF480724E49DAF80000CDE90044FCF725
:1030200029FE8346514806F099FF83454FDB02464F
:1030300047494E4806F0A5FF002848D1032157F81C
:1030400025304A46996057F8250041460C3006F075
:10305000B7FF494A4FF480713D48FBF729F8014614
:1030600057F82530C1F580711B68424A3018FBF7CC
:103070001FF83748DAF8006006F070FF2346024672
:103080003349304601940094FCF70CFD0646304865
:1030900006F064FFB04253D123464FF480722C49AE
:1030A000DAF80000CDE90044FCF7E4FD06463348B9
:1030B00006F054FF864233DB024625492F4806F0CE
:1030C00060FF68BB28462249FFF78EFD59E72C4870
:1030D00006F044FF1E490246294806F052FF002828
:1030E0007FF44AAF0820FBF7BDFD4FF0FF3448E7FF
:1030F000C4F580713019234B1A4AFAF7D9FF0444FA
:1031000018E74FF0FF340920FBF7ACFD204603B071
:10311000BDE8F08F1620FBF7A5FD4FF0FF3430E738
:10312000174806F01BFF0A490246154806F029FF1A
:1031300030B90820FBF796FD23E74FF0FF3420E776
:103140000520FBF78FFD1CE700009A784043022022
:1031500040420220B8BE0100C4BE0100D8BE01003A
:10316000E0BE0100D0BE010014BF0100E4BE0100BA
:10317000E8BE0100F4BE0100F8BE010008BF010076
:103180004CBF0100C8BE01003C4202202DE9F043C3
:10319000634B83B0834340F09D8020F0F14424F4DE
:1031A000D014092C00F396805E4D55F824000028B9
:1031B00000F090808368002B00F08C808368032BE4
:1031C00008D0FDF715FA0023184645F8243003B05F
:1031D000BDE8F083544E554A4FF480713046FAF7FB
:1031E00067FF55F82430C0F580711B68504A3044A1
:1031F000DFF84C81FAF75CFF3046D8F800900027E2
:1032000006F0ACFE314602463B4648460197009721
:10321000FCF748FC8146304606F0A0FE484576D1D2
:103220003B46CDE900774FF480723146D8F8000074
:10323000FCF720FD07463F4806F090FE87424FDA34
:103240003D4806F08BFE384902463B4806F099FEA1
:1032500000285CD10820FBF705FD384A4FF4807147
:103260003148FAF725FF014655F82430C1F5807141
:103270001B682F4A3018FAF71BFF2B48D8F800704C
:10328000002606F06BFE3346024627493846019673
:103290000096FCF707FC0746234806F05FFEB8429D
:1032A00039D13346CDE900664FF480721E49D8F813
:1032B0000000FCF7DFFC06461E4806F04FFE864283
:1032C00016DB024618491B4806F05BFE80B955F82C
:1032D000240076E70920FBF7C5FC4FF0FF3076E7C6
:1032E00002463146134806F04CFE0028B5D0A7E749
:1032F000114806F033FE0C4902460F4806F041FE25
:1033000048B90820FBF7AEFC55F8240059E7052022
:10331000FBF7A8FCA1E70520FBF7A4FCD7E700BF5B
:1033200000009A784043022040420220ACBE0100D7
:10333000F4BE0100E4BE01004CBF0100B8BE0100B4
:103340003C42022010B540F20224A1420BD153B1FD
:10335000029941B1254981430BD00920FBF782FC3A
:103360004FF0FF3010BD1620FBF77CFC4FF0FF3014
:1033700010BD20F0F14020F4D0100928EDDC1C49EC
:1033800051F820100029E8D08C68002CE5D00028E6
:10339000E3DB012A01D02D20E6E78A68FAB18A68CA
:1033A000032A1CD08A68042A19D0029A9008421E67
:1033B000012AD8D8029A9207D5D11A68022A10D0C9
:1033C0000A2AD0D10222022806D15B68022B0AD039
:1033D0000A2BC8D142F002020A670020C4E70E207F
:1033E000C2E70122EFE742F00102F5E700009A7818
:1033F000404302202DE9F04340F2022483B0A14271
:103400000A9D40F0A9801E46002B00F0A580002DEB
:1034100000F0A280564B834340F0848020F0F144BA
:1034200024F4D014092C7DDC524B53F82430002BAB
:1034300078D09968002975D0002C73DB022A0ED051
:10344000032A08D0012A15D02D20FBF70BFC002001
:1034500003B0BDE8F0832B6823BB1620F5E72A688C
:10346000002AFAD0012200201B6833702A6003B0C2
:10347000BDE8F0839A68002A52D09A68042A4FD097
:103480002A68072AE9D912F00302E6D11B6F9907CF
:103490005DD40421DB0702D50223B3500A462A601B
:1034A0000020D5E7344A4FF480713448DFF8D880E3
:1034B000FAF7FEFD3148D8F80090002706F04EFDDF
:1034C0003B4602462D49484601970097FCF7EAFA29
:1034D00081462A4806F042FD484543D13B46CDE9A6
:1034E00000774FF480722549D8F80000FCF7C2FB42
:1034F0000746234806F032FD874219DB02461F4982
:103500001F4806F03EFD074690B920461B49FFF7CD
:1035100035FB002899DB0123307038462B6097E794
:103520000E2092E70920FBF79DFB4FF0FF308FE75D
:10353000144806F013FD11490246124806F021FD19
:1035400080B90820FBF78EFB4FF0FF307DE70A22A1
:103550000821326004229DE71620FBF783FB4FF021
:10356000FF3075E70520FBF77DFB4FF0FF306CE780
:1035700000009A78404302201CBF01004042022014
:1035800028BF01004CBF01003C420220002900F08E
:10359000B9832DE9F043A34C022883B00D4623687C
:1035A00000F094800A283FD01BB19B68032B00F0E9
:1035B000278163681BB19B68032B00F01081A3680F
:1035C0001BB19B68032B00F0F980E3681BB19B687B
:1035D000032B00F0E28023691BB19B68032B00F0F2
:1035E000238163691BB19B68032B00F06181A36990
:1035F0001BB19B68032B00F04A81E3691BB19B68F8
:10360000032B00F03381236A1BB19B68032B00F06E
:103610001C81636A1BB19B68032B00F0AD804FF0E7
:10362000FF3003B0BDE8F0831BB19B68032B00F0B3
:10363000358363681BB19B68032B00F0FD82A36890
:103640001BB19B68032B00F0D582E3681BB19E6819
:10365000032E00F0F08123691BB19B68032B00F05F
:10366000038263691BB19B68032B00F01582A36979
:103670001BB19B68032B00F02782E3691BB19B6899
:10368000032B00F03982236A1BB19B68032B00F0E7
:103690004D82636A002BC2D09B68032BBFD12846A2
:1036A00006F05CFC0646606A0C3006F057FCB0423F
:1036B000B5D1616A28460C3106F057FC0028AED11E
:1036C000636A1A6F9207AAD509261AE11BB19B6893
:1036D000032B00F0FD8263681BB19B68032B00F095
:1036E000C582A3681BB19B68032B00F06982E36865
:1036F0001BB19E68032E00F0EC8023691BB19B6810
:10370000032B00F04A8163691BB19B68032B00F017
:103710005E81A3691BB19B68032B00F07281E36992
:103720001BB19B68032B00F01B82236A1BB19B68B3
:10373000032B00F02D82636A002B3FF470AF9B686F
:10374000032B7FF46CAF284606F008FC0646606A3F
:103750000C3006F003FC86427FF461AF616A2846B4
:103760000C3106F002FC00287FF459AF636A1A6F2F
:10377000D2077FF554AFA7E7284606F0EFFB0646D1
:10378000606A0C3006F0EAFBB0427FF448AF616A31
:1037900028460C3106F0E9FB41E7284606F0DEFB3F
:1037A0000646E0680C3006F0D9FB86427FF413AF82
:1037B000E16828460C3106F0D8FB0CE7284606F0F5
:1037C000CDFB0646A0680C3006F0C8FB86427FF4AD
:1037D000FCAEA16828460C3106F0C7FBF5E628468A
:1037E00006F0BCFB064660680C3006F0B7FB86426C
:1037F0007FF4E5AE616828460C3106F0B6FBDEE6E4
:10380000084606F0ABFB064620680C3006F0A6FB27
:1038100086427FF4CEAE216828460C3106F0A5FB27
:10382000C7E600BF40430220284606F097FB064645
:1038300020690C3006F092FB86427FF4D2AE2169FB
:1038400028460C3106F091FBCBE6284606F086FBB5
:103850000646206A0C3006F081FB86427FF4D9AE22
:10386000216A28460C3106F080FBD2E6284606F095
:1038700075FB0646E0690C3006F070FB86427FF46B
:10388000C2AEE16928460C3106F06FFBBBE6284664
:1038900006F064FB0646A0690C3006F05FFB86422A
:1038A0007FF4ABAEA16928460C3106F05EFBA4E6BE
:1038B000284606F053FB064660690C3006F04EFBC6
:1038C00086427FF494AE616928460C3106F04DFBC8
:1038D0008DE6284606F042FB0746E0680C3006F00D
:1038E0003DFB87427FF409AFE16828460C3106F0C2
:1038F0003CFB00287FF401AFE3681A6FD1077FF526
:10390000FCAE5868431C7FF48CAEC64DC64A4FF4DB
:1039100080712846FAF7CCFB54F82630C0F5807148
:103920001B68C24A2844DFF80C83FAF7C1FB28461B
:10393000D8F80090002706F011FB294602463B46C6
:10394000484601970097FCF7ADF88146284606F0F7
:1039500005FB484540F0E9813B464FF48072CDE9D4
:1039600000772946D8F80000FCF784F90746B048EC
:1039700006F0F4FA87420246C0F2C7812946AC48F5
:1039800006F0FFFA002840F0C08129463046FFF7D4
:103990002BF954F82630586843E6284606F0DEFA3C
:1039A000064620690C3006F0D9FA86427FF4ABAEA9
:1039B000216928460C3106F0D8FA00287FF4A3AE1E
:1039C00023691A6FD2077FF59EAE042699E7284631
:1039D00006F0C4FA064660690C3006F0BFFA86426B
:1039E0007FF497AE616928460C3106F0BEFA0028D4
:1039F0007FF48FAE63691A6FD7077FF58AAE05260D
:103A00007FE7284606F0AAFA0646A0690C3006F0C1
:103A1000A5FA86427FF483AEA16928460C3106F0F0
:103A2000A4FA00287FF47BAEA3691A6FD6077FF54E
:103A300076AE062665E7284606F090FA0746E06867
:103A40000C3006F08BFA87427FF405AEE168284619
:103A50000C3106F08AFA00287FF4FDADE3681A6F96
:103A600091073FF54EAFF6E5284606F077FA064691
:103A700020690C3006F072FA86427FF4F2AD2169BB
:103A800028460C3106F071FA00287FF4EAAD23696C
:103A90001A6F920799D4E4E5284606F05FFA0646C5
:103AA00060690C3006F05AFA86427FF4E0AD616935
:103AB00028460C3106F059FA00287FF4D8AD636926
:103AC0001A6F97079BD4D2E5284606F047FA0646B8
:103AD000A0690C3006F042FA86427FF4CEADA169AF
:103AE00028460C3106F041FA00287FF4C6ADA369E0
:103AF0001A6F96079DD4C0E5284606F02FFA0646B1
:103B0000E0690C3006F02AFA86427FF4BCADE16928
:103B100028460C3106F029FA00287FF4B4ADE36999
:103B20001A6F90077FF5AFAD0726EAE6284606F044
:103B300015FA0646206A0C3006F010FA86427FF429
:103B4000A8AD216A28460C3106F00FFA00287FF450
:103B5000A0AD236A1A6F91077FF59BAD0826D0E6CA
:103B6000284606F0FBF90646E0690C3006F0F6F947
:103B700086427FF4DAADE16928460C3106F0F5F9AA
:103B800000287FF4D2ADE3691A6FD007CCD4CCE51E
:103B9000284606F0E3F90646206A0C3006F0DEF906
:103BA00086427FF4C8AD216A28460C3106F0DDF963
:103BB00000287FF4C0AD236A1A6FD107CED4BAE5CE
:103BC000284606F0CBF90646A0680C3006F0C6F988
:103BD00086427FF48CADA16828460C3106F0C5F909
:103BE00000287FF484ADA3681A6FD0077FF57FADFE
:103BF000022686E6284606F0B1F90646A0680C3093
:103C000006F0ACF986427FF420ADA16828460C315D
:103C100006F0ABF900287FF418ADA3681A6F90077F
:103C2000E6D412E540420220F8BE0100F4BE0100D5
:103C300008BF01003C420220284606F08FF90646E4
:103C400060680C3006F08AF986427FF4F8AC61684F
:103C500028460C3106F089F900287FF4F0AC63683F
:103C60001A6F96077FF5EBAC01264AE6284606F068
:103C700075F9064660680C3006F070F986427FF4EC
:103C800030AD616828460C3106F06FF900287FF4EA
:103C900028AD63681A6FD607E6D422E5084606F019
:103CA0005DF9064620680C3006F058F986427FF42C
:103CB000C0AC216828460C3106F057F906460028AA
:103CC0007FF4B7AC23681A6F97073FF51AAEB0E4DC
:103CD000084606F043F9064620680C3006F03EF927
:103CE00086427FF4F8AC216828460C3106F03DF995
:103CF000064600287FF4EFAC23681A6FD7073FF51C
:103D000000AEE8E44FF0FF3070470B4806F026F9AC
:103D10000A490246084806F034F930B90820FAF793
:103D2000A1FF54F8263058687BE40520FAF79AFF83
:103D300054F82630586874E44CBF01004042022019
:103D400028B100230360C0E90133184670470720FB
:103D5000704700BF0268034601320ED000220A609D
:103D600002683AB18268116081601A6800200132ED
:103D70001A607047C0E90111F7E70420704700BFDF
:103D80000346006828B158681A680168013A59600A
:103D90001A60704703680BB1406870471846704757
:103DA000006870470068704770B504460D461646B7
:103DB000FDF7D6FC30B10368324629462046BDE8FF
:103DC000704018474FF0FF3070BD00BF10B504467B
:103DD000FDF71AFD20B143682046BDE810401847A2
:103DE0004FF0FF3010BD00BF2DE9F0470D46DDE973
:103DF000088916461F460446FDF706FD58B1CDE971
:103E00000889D0F808E03B46324629462046F44669
:103E1000BDE8F04760474FF0FF30BDE8F08700BFD6
:103E20002DE9F04182B00E46174698460546FDF74B
:103E3000EBFC60B104460020CDE9000043463A4661
:103E400031462846A468A04702B0BDE8F0814FF093
:103E5000FF30F9E72DE9F0470D46DDE90889164600
:103E60001F460446FDF7D0FC58B1CDE90889D0F8CB
:103E70000CE03B46324629462046F446BDE8F04772
:103E800060474FF0FF30BDE8F08700BF2DE9F041FB
:103E900082B00E46174698460546FDF7B5FC60B160
:103EA00004460020CDE9000043463A463146284604
:103EB000E468A04702B0BDE8F0814FF0FF30F9E7B9
:103EC00070B50D4616460446FDF79EFC30B14369B9
:103ED000324629462046BDE8704018474FF0FF3073
:103EE00070BD00BF70B50D460446FDF78DFC28B1CE
:103EF000836929462046BDE8704018474FF0FF30DF
:103F000070BD00BF2DE9F0410D4616460446FDF791
:103F10007BFC40B1C769324629462046BC46BDE815
:103F2000F041002360474FF0FF30BDE8F08100BF53
:103F300070B50D4616460446FDF766FC30B10369C0
:103F4000324629462046BDE8704018474FF0FF3002
:103F500070BD00BF2DE9F041DDF818800D46164612
:103F60001F460446FDF750FC58B1CDF81880D0F834
:103F700020E03B46324629462046F446BDE8F04163
:103F800060474FF0FF30BDE8F08100BF2DE9F04100
:103F9000DDF818800D4616461F460446FDF734FC32
:103FA00058B1CDF81880D0F824E03B463246294677
:103FB0002046F446BDE8F04160474FF0FF30BDE8D1
:103FC000F08100BFFDF790BCFDF790BCFDF790BC01
:103FD000FDF7E8BC20B150F8081B090CFBF7AABE9E
:103FE000704700BF014801F0F3BD00BF60BF010092
:103FF00080B1002310B582B002AA044642F8043D05
:10400000032002F01DF818B9019B0BB1083323609F
:1040100002B010BD0E20704750B1034630F8082C96
:10402000032042EA014143F8081D194601F0F0BFA0
:104030000E20704720B1A0F10801032002F032B831
:104040000E20704718B10146032002F03DB90E2042
:10405000704700BF10B504460068FCF729FBA06854
:1040600018B1BDE81040FCF7C3BA10BD10289ABFC4
:10407000024B53F820002D20704700BF70BF010095
:1040800070B5002582B002AC44F8045D06460D46CA
:10409000204619461446FCF7D9FA60B9019B08225C
:1040A00058729872D872184644EA0644DC601D6162
:1040B0001A7202B070BD019B184602B070BD00BFFD
:1040C00070B50C460546114620461E46FCF7D2FA4E
:1040D00000B970BD206808B1FCF7EAFA2046FCF789
:1040E000DFFA2E60232070BD38B5054601F098FB3D
:1040F000044608B1204638BD284601F005FC0028DA
:10410000F8D04468002CF5D000234360204638BD29
:1041100038B50023074D084C1946242207482B6068
:10412000236005F077FFFCF78BFA003018BF012001
:10413000404238BD7843022074430220804302206D
:104140002DE9F0410646002026F0080382B0022B3C
:104150000C461746009002D0052E40F08480631E66
:10416000022B5CD8002F54D1012C67D0032C18BF30
:104170000227484A2146684601F0A6FA009B80467D
:10418000002B59D0002102A840F8041DC3E90364A4
:104190005F61FCF75BFA00284BD147F201024FF058
:1041A000FF330821019D42EA0842EA606872A87262
:1041B000E87229722B746B74AB74EB74AB68052EC8
:1041C00003F10C03AB6003D00A2E14BF01260226B4
:1041D0006E61EF61AC6147F201012846009FFCF778
:1041E00049FA064660B3286808B1FCF761FA284628
:1041F000FCF756FA012323253B60404601F0C2FA42
:104200002846FAF72FFD4FF0FF38404602B0BDE8D0
:10421000F081012C09D0022C09D1022FA9D016203F
:10422000FAF720FD4FF0FF38EFE7012FF7D1022713
:104230009FE7019D002DC1D10C25DEE7274698E7B9
:104240004FF0FF334FF6FF720221404601F0E8FACB
:1042500005460028D1D1404601F056FB48B14568DB
:104260003DB14660C9E72F20FAF7FCFC4FF0FF385C
:10427000CBE7023C012CC8D84046009B1A6842F4A8
:1042800000321A601A6842F480121A6002B0BDE867
:10429000F08100BF554001002DE9F04182B0064693
:1042A00001F032FB002863D00446002102A82768F1
:1042B00040F8041DD4F81880FCF7C8F900283AD15A
:1042C00047F209030822019D43EA0643EB60C5F863
:1042D00010806872A872E8722A72236847F2090196
:1042E0001B0C1B0443F00D0323602368284623F4B2
:1042F00000332360236823F480132360FCF7BAF9AA
:1043000040BB4FF0FF334FF6FF720E21304601F0F5
:1043100087FA0446A0B1174C54F8260020B1FCF7E8
:10432000BFF9002344F82630304601F02BFA002074
:1043300002B0BDE8F081019D0C20002DCDD112E02E
:10434000304601F0E1FA0028E5D04368002BE2D0C6
:104350004460E0E7286808B1FCF7AAF92846FCF7B2
:104360009FF923202760FAF77DFC4FF0FF30DFE74D
:104370000920F8E7804302202DE9F04F002589B09D
:1043800003911446019307950746129E01F0BCFA6B
:10439000002800F02481B4F5805F00F318810369E0
:1043A0000546012B00F0D1802A68900323D42A68A7
:1043B000910006D4012B00F0ED802B681A0340F128
:1043C00002812B681B0340F10681A868DFF8189270
:1043D000002840F096802B68180140F182802B68FD
:1043E00023F000632B6059F8270000287CD1204679
:1043F00009B0BDE8F08F47F206084FF00C0A3B0405
:10440000DFF8E4910493214607A8FCF71FF904287C
:10441000F9D0002871D1079B83F808A058729872D0
:10442000D8723EB3EA6871688A420AD1022A03F15F
:104430001C00317800F090800A2A02D1242900F073
:10444000AF80186810B1FCF733F9079B1846FCF7EA
:1044500027F916202B681A0353D42B689BB20D2B17
:10446000B6D02B6823F400132B602B6843F4003381
:104470002B60ADE7424601995961A9690498196119
:1044800003990243DA605C6019B11868224605F0AE
:1044900097FD2B68414605932B6823F400332B606E
:1044A0002B6843F400132B60079B18460293FCF71C
:1044B000E1F8029B834658BB4FF400324FF0FF33C4
:1044C0001146384601F0ACF970B32B68190337D4A4
:1044D0000C28BFD159F82700002894D0FCF7E0F849
:1044E00091E759F827008469FCF7DAF800232046A1
:1044F00049F8273009B0BDE8F08F2B680C201A036B
:10450000ABD5FAF7AFFB4FF0FF3459F827006CE753
:1045100018689B4608B1FCF7CBF85846FCF7C0F882
:10452000059B23202B6095E7384601F0EDF9034603
:10453000F0B14068E0B1C3F804B02B681903C7D5E7
:10454000A8682B681E0388D542E7002E3FF42CAFE5
:104550001620DFF89490D4E710297FF472AF04227C
:1045600031895A83198306F10C0105F029FD1EE0FB
:104570002B681B033FF52FAF2B689BB20D2B3FF42D
:104580002AAF2B6823F400132B602B6843F400330D
:104590002B6020E72B689BB2052B7FF412AF0CE752
:1045A000102231895A831983B11805F009FD47F2A9
:1045B0000702079B90469968588B04310144019883
:1045C0009960586159E72320DFF81C9099E728206B
:1045D000DFF8149095E73920DFF80C9091E7092077
:1045E000DFF804908DE700BF804302202DE9F04FF3
:1045F00085B0002A00F010818A4699460746164683
:1046000001F082F90446002800F00D810368D90208
:1046100065D519F0020F18BF4FF000084FF0FF3BAF
:1046200008BF036809F0100504BF83F08058C8F381
:1046300000782368DA036DD52368E06923F48033BA
:1046400023600368DB689847B0F1FF3F834600F0C2
:104650008180864203DD2369012B00F0A7800025BD
:10466000E0690F9B03B11B680E9ACDE900A6CDE966
:10467000022303684A469B68694698478346E06977
:10468000BBF1FF3F036818BF0126DB680ABF0026A5
:104690004FF000084FF023089847013035D1002D26
:1046A00000F0B680002E00F0A6802368190306D51E
:1046B00023689BB20D2B02D02369012B25D02368E0
:1046C00013F0804F236840F0B1801A0375D4B8F11D
:1046D000000F40F08A80584605B0BDE8F08F0368AF
:1046E0009BB2062B73D003689BB2072B0CBF4FF015
:1046F00009084FF03908E0690368DB689847B0F1B2
:10470000FF3F8346DBD04FF0FF3B236843F4803309
:104710002360DCE7B8F1000F00F081804FF48032B5
:10472000236A1146002B08BF4FF0FF33384601F0D3
:1047300077F8804658B32368E0691B0321D52368C6
:104740009BB20D2B1DD02569A5F10105B5FA85F5A4
:104750006D0986E723681803DCD523689BB20D2B0F
:10476000D8D02369E069012B34D04FF03908236891
:104770001B0C1B0443F00D032360236823F48013F8
:1047800023600368DB6898470130BED197E738465D
:1047900001F0BAF838B1D0F80480B8F1000F02D0B7
:1047A00000234360C7E74FF0010842E71DB12368CB
:1047B000DB00B3D553E7E06953E723689BB20D2BC9
:1047C00085D1A368002B82D0D4F808807FE74FF012
:1047D000090890E70368DB68984701300BD04FF079
:1047E0002308236843F4803323604046FAF73AFAFB
:1047F0004FF0FF3B6FE723684FF0000B1B0C1B04CF
:1048000043F00D032360236823F48013236062E7E1
:10481000002E7FF44AAF52E74FF01608E5E74FF05D
:104820002308E069ADE74FF00908DEE723F0804395
:10483000236023684FF069081B0C1B0443F00D0331
:104840002360D2E72DE9F04182B0002944D0002A4C
:1048500042D006460F4601F057F80546002800F002
:10486000968003689BB2022B04D003689BB2042B92
:1048700040F08D80296811F0005140F0848002A83A
:1048800040F8041DD5F81880FBF7E0FE70BB082146
:104890003304019C43F4E04242F00202E260C4F8B7
:1048A00010806072A072E072217243F4E04343F022
:1048B0000203E360A368AA6904332261A360EB6882
:1048C0007A68934208D1022B04F118003A783AD062
:1048D0000A2B01D1242A0ED016242046FAF7C2F959
:1048E0004FF0FF34204602B0BDE8F081019C002C5F
:1048F0004FD03304D9E710223B89B918E282A38252
:1049000005F05EFBA368E28A47F202011344A3604C
:104910002F682B68204643F000532B60FBF7AAFE5C
:10492000E0B92B6813F080582FD14FF0FF334FF6CA
:10493000FF720521304600F073FF0446C0B1732CAE
:10494000CBD02F60C9E7102AC6D104223B8907F1DA
:104950000C01E282A38205F033FBD3E7206808B1A3
:10496000FBF7A6FE2046FBF79BFE23242F60B4E74F
:10497000304600F0C9FF0028B4D04468002CB1D004
:10498000C0F80480DBE77224A7E77324A5E70924B5
:10499000A3E70C24A1E700BF2DE9F04182B089B361
:1049A00082B307460E4600F0AFFF054600287BD0D5
:1049B00003689BB2022B77D1002102A840F8041DA6
:1049C000D5F81880FBF742FE30BB47F205030822FA
:1049D000019C43EA0743E360C4F810806072A07250
:1049E000E0722272A3680433A360EB68726893429A
:1049F00008D1022B04F1180032783CD00A2B01D1E7
:104A0000242A0ED016242046FAF72CF94FF0FF3452
:104A1000204602B0BDE8F081019C002CE2D10C24BC
:104A2000F1E710223389B118E282A38205F0C8FAB7
:104A3000A368E28A47F205011344A3602B6820466D
:104A40001B0C1B0443F003032B602E68FBF712FEC4
:104A50008046D8B94FF0FF334FF6FF720421384635
:104A600000F0DEFE044608B32B681B0C1B0443F069
:104A700002032B60C7E7102AC4D10422338906F150
:104A80000C01E282A38205F09BFAD1E7206808B10D
:104A9000FBF70EFE360C3604204646F00206FBF706
:104AA000FFFD23242E60AEE70924ACE7384600F072
:104AB0002BFF0028ACD04468002CA9D0C0F804809B
:104AC000D2E700BF2DE9F04182B0064600F01CFF9E
:104AD000002867D0036805469BB2042B62D10021F1
:104AE000324A304600F064FE014600285CD102A83C
:104AF00040F8041DAF69FBF7A9FDA8BB47F2080306
:104B00000822019C43EA0643E36027616072A072B9
:104B1000E0722272A36847F208010433A3602B6895
:104B200020461B0C1B0443F006032B602F68FBF789
:104B3000A1FD8046E8B94FF0FF334FF6FF72072121
:104B4000304600F06DFE044608B32B681B0C1B04B6
:104B500043F004032B602046FAF784F84FF0FF344B
:104B6000204602B0BDE8F081019C002CD2D10C247B
:104B7000F1E7206808B1FBF79BFD3F0C3F0420469E
:104B800047F00407FBF78CFD23242F60E3E7304652
:104B900000F0BAFE0028E3D04468002CE0D0C0F852
:104BA0000480D2E70924D6E72324D4E75540010046
:104BB0002DE9F04F002585B00F4690460295064638
:104BC00000F0A2FE0446002800F01C8103689BB29E
:104BD000072B0AD103680568DB0016D415F480356D
:104BE00019D0056815F4803524D14FF00909029BCE
:104BF00013B1284600F0C6FD48464FF0FF39FAF7DA
:104C000031F8484605B0BDE8F08F15F480356DD118
:104C10004FF02309EBE74FF480324FF0FF3311469A
:104C2000304600F0FDFD814600287ED0256815F451
:104C30008035DCD04FF0FF300023CDE90003754A0A
:104C4000216902A800F040FD029B0546002B00F000
:104C5000DD800021626904A85A61E26840F8041D01
:104C6000DA6022691A61D4F81890FBF7EFFC00288B
:104C700043D147F20C030821DDF80CB043EA0643A8
:104C8000CBF80C30CBF810908BF809008BF80A00A9
:104C90008BF80B008BF80810236847F20C011B0CF3
:104CA0001B0443F0080323605846D4F80090FBF738
:104CB000E1FC824648BB226800994FF0FF330A406E
:104CC000226009214FF6FF72304600F0A9FD8146AF
:104CD000002800F085802368019A1A432260236827
:104CE0001B0C1B0443F00703236080E76FF0805226
:104CF0004FF08053CDE90023A1E7DDF80CB04FF071
:104D00000C09BBF1000FC7D171E7DBF8000008B157
:104D1000FBF7CEFC4FEA194958464FEA0949FBF721
:104D2000BFFC49F00703236072E7304600F0ECFD5A
:104D300030B1D0F80490B9F1000F01D0456075E7AB
:104D40002368D9033FF576AF334D029955F82630E5
:104D50009B698B6147B1CB680A2B24D0022B03D10E
:104D6000D8F80020102A32D00A682C48024042F0BD
:104D700005020A60029A116841F40031116011685D
:104D800041F4801111602368034043F0070323605E
:104D900055F82600FBF784FC0023484645F82630EA
:104DA00005B0BDE8F08FD8F80020242ADCD13A7095
:104DB00010227B6055F8263007F110009B8B3B8159
:104DC00055F82610203105F0FBF80299CCE73A702F
:104DD0007B6055F8263007F10C009B8B0422EEE730
:104DE000304600F091FD38B1D0F80490B9F1000FD1
:104DF00002D0C0F804A06EE72368019AA9461343C5
:104E00002360A1E705464FF00909F0E64FF00C09D1
:104E1000F2E600BF55400100804302200000FFFF82
:104E20002DE9F041012984B040F09C800E46904667
:104E30001D46074600F068FD0446002800F0A580E6
:104E4000B8F1190F6ED1002D00F09280284605F0C0
:104E500085F80A9B984240F08B8023689BB2022B16
:104E600073D12946E068FEF791FB0290013008BF3C
:104E700016254ED023685B024AD4236813F400033E
:104E800046D12668226804A842F4800222600421E8
:104E900040F8043DD4F81880FBF7D8FB00284ED129
:104EA00047F2030200230821039D42EA0742EA6019
:104EB000C5F8108029726B72AB72EB724FF0080C60
:104EC000002310203021AA686B756244AA60AB757C
:104ED000EB75AB76EB7685F814C0287669760422FC
:104EE0000DEB0C01286805F06BF847F2030128462A
:104EF000FBF7C0FB804650BB4FF400024FF0FF337E
:104F00001146384600F08CFC054698B3266000E058
:104F100023252846F9F7A6FE4FF0FF35284604B0B2
:104F2000BDE8F0810A9B4246009331462B46384645
:104F300000F012FD0546284604B0BDE8F081039D4F
:104F4000002DBBD126600C25E3E70925E1E72868A1
:104F500008B1FBF7ADFB2846FBF7A2FB2325266033
:104F60002660D6E72A20F9F77DFE4FF0FF35D5E71A
:104F70000E25CEE7384600F0C7FC20B1456815B1D4
:104F8000C0F80480C2E72660C8E70920F9F76AFE86
:104F90004FF0FF35C2E700BF00F014BD2DE9F04F20
:104FA0004FF0000C0124724EDFF8D0A1DFF8D09151
:104FB00085B0074615460193A6F800C0CAF8004020
:104FC000C9F8004071B108460A22614604F008FFA2
:104FD0004FF6FE73421E9A4200F28380030243EAB8
:104FE00020203080DFF89C81D8F80030002B74D16D
:104FF000604A1360604A1360002F62D0384604F0A4
:10500000ADFF834625B1EA6912B1516866296CD0BB
:105010004FF0FF32002104AE46F8041D30465946D9
:105020000092FBF713FB009A00284CD147F20D01C8
:105030004FF0080C039C41EA0241E160226160727A
:10504000A072E07284F808C0002D76D06A6822F061
:10505000080102295CD0052A78D1A9680229C9F87B
:10506000001061D0A261EA682262AA68E2612A683F
:105070006261A2681032A2602FB1206818B15A464E
:10508000394604F09DFF012347F20D012046C8F880
:105090000030FBF7EFFA002856D14FF0FF330393AF
:1050A00031462046F9F74AFDD8F80030012BF7D0F9
:1050B000314B186800283BD12E4B019A1B681360B6
:1050C0000CE0BB469EE7039C002CBDD10C200023C6
:1050D000C8F8003005B0BDE8F08F732005B0BDE81A
:1050E000F08F162005B0BDE8F08F9168B1F5007F14
:1050F0008ED140F20221D068884289D1916900297D
:1051000086D06868FEF742FA431C81D0024681E7E8
:10511000A9680229C9F8001006D0052AA2D00A2AD7
:1051200014BF012202229DE70221CAF80010F4E711
:10513000114B18680028D1D0C9E72946102204F184
:10514000140004F067FF94E72320C0E72F20F9F74D
:1051500089FDA2681032A26017B94FF0FF30B6E7A0
:1051600020680028F9D05A46394604F029FFF4E7B0
:105170005A4C0220784302207043022068430220E8
:105180006C4302207443022038B50B4C2368022B79
:1051900000D038BD30B105464069FBF729FA2846F2
:1051A000FBF726FA0023054A0549236013600868C7
:1051B000BDE83840FBF77CBA7443022070430220FC
:1051C0007C43022048F20D032DE9F04F994289B04B
:1051D000054662D048F20F0399420C464BD001F4C9
:1051E0001043B3F5104FC0687BD0070C384600F071
:1051F0008BFB064600285FD0014623462A463846E8
:10520000FBF798FE002853D048F207039C427CD954
:1052100048F20C039C4268D040F2188149F2020324
:105220009C4200F0918149F203039C4200F0A68168
:1052300049F201039C423FD1346814F4801400F019
:10524000BE81AB68042B00F2F48100242746296854
:105250006A68CDE90674CDE90412F06904A903680F
:105260005B689847013000F0D0813368002043F438
:10527000803333600EE043690120102BB54988BFAD
:105280002D2208704FF000009CBFB34A52F8232033
:10529000B24B1A6009B0BDE8F08FDFF8D49207680E
:1052A000D9F80030012B0BD017B13846FBF700FAC4
:1052B000002009B0BDE8F08F28680028F6D1F7E794
:1052C0004369002B45D0102B96BFA34A2D2352F8DB
:1052D00023300222A2490B60C9F80020002FE4D13C
:1052E000E6E700F0BFFA074680E733689BB2082B79
:1052F000DED16B69002B00F08A81102B00F25D81FA
:10530000954A52F823307360D2E748F206039C4274
:1053100080F0098148F202039C4200F0EC8040F2E8
:10532000BE8048F203039C4200F0CA8048F20503A5
:105330009C42C1D133689BB2032BB9D16B69002B5E
:10534000DBD1336800201B0C1B0443F004033360E3
:10535000A0E7844B1F608469630118460393FBF741
:105360003DF90290002800F08A80E50028198000AD
:10537000FBF734F9002800F01C81002C5ED01035BA
:1053800043190193029B0424DFF8E8A1DFF8E8B198
:1053900000F1100803F120061DE00A2248F80C2C49
:1053A0004FF02402404608F8102C28F8083C56F824
:1053B000102C04F005FE56F8103C08F108081C44B7
:1053C0003B1946F8083C019B46F8046C98452C4470
:1053D00006F120062CD03B593A1946F8203C536878
:1053E000DAF80010022B14BF02200A20DBF800308C
:1053F00046E9070146F8143C108AA8F1100346F864
:10540000100C558A46F80C3C574B1434042807EB13
:1054100004011B88C1D11022022028F8083C48F85A
:105420000C0C08F8102C56F8102CA8F10400C0E75A
:105430000022DDE902130B4443F8042C02224B4BFB
:10544000C9F80020029A00201A6023E748F20803F6
:105450009C4241D048F209039C427FF42DAF33684F
:105460009BB20D2B7FF424AF6869002800F0DA802E
:10547000102800F2A280384B53F8203043E7FBF7A6
:10548000B7F80C2002233649384A08602F68029981
:10549000C9F800301160002F7FF407AF08E748F229
:1054A00001039C427FF408AF3368012B7FF400AF07
:1054B00068690028DCD102233360AB69B361E9E697
:1054C00033685B027FF5F4AE68690028D0D1336899
:1054D00043F400033360DDE633689BB2062B7FF4B0
:1054E000E7AE68690028C3D133681B0C1B0443F086
:1054F00007033360CEE6336899007FF5D9AE336891
:1055000023F0005333606869002866D010288EBFEE
:105510002D23114B53F8203000207360336843F47F
:1055200080233360B6E633689A027FF5C1AE6B69BB
:10553000002B61D06B2B7FF4E0AE3369012B7CD064
:105540000C2300207360A5E633689BB2072B7FF421
:10555000AFAE8AE68154022070BF0100A44302204E
:10556000704302207C4302205A4C022078430220E0
:10557000744302206C43022068430220336843F4E2
:1055800000233360336823F400133360336823F45B
:10559000003333602B696C2B16D0102B8CBF2D235E
:1055A000404A4FF0000098BF52F823307360B36058
:1055B00070E60C223C4B1A6040E72D23A3E62868D6
:1055C000FBF776F8204665E639223368002043F081
:1055D000804333607260B2605CE6336843F400334A
:1055E0003360336843F48013336033681B0C1B044F
:1055F00043F0050333604DE633682C4A43F400332F
:105600003360012042F8275044E6022042E6274B4F
:10561000012043F8275033681B0C1B0443F0090397
:10562000336037E633681B0C1B0443F00E03336012
:1056300030E66C8A4CB9274609E60C223368002014
:1056400043F000633360726024E62420FAF7C6FF5B
:10565000074618B36A8A102A14D0042A06D028688C
:10566000FBF726F83846FAF7C3FF21E60223102499
:10567000436004702B8A05F1140103810C3004F09F
:105680009FFCE4E50A232424436004702B8A05F17F
:1056900014010381103004F093FCD8E52868FBF76F
:1056A00007F805E670BF0100704302208043022026
:1056B00008B54FF4A2720021024804F0ABFC0020B0
:1056C00008BD00BF84540220F8B52D4B06461D6866
:1056D000084615B35C6A002C43D09C6C002C42D069
:1056E000DC6E002C41D0D3F8901000293FD0D3F8C5
:1056F000B41089B1D3F8D81000293CD0D3F8FC10ED
:1057000000293AD0D3F8201199B34FF0FF350C207F
:10571000F9F7A8FA2846F8BD05254FF0010C4FF01F
:10572000FF3705EBC504A40043F804C01C44114630
:10573000A761224601F0EEFF0346E06158B11B6805
:105740001B68984710B934602846F8BDE06902F03C
:1057500001F80023E36120462422002104F05AFCD2
:10576000D3E70125D9E70225D7E70325D5E70425A7
:10577000D3E70825D1E70625CFE70725CDE700BF0A
:1057800084540220082800D9704710B5074C00EB5C
:10579000C00004EB8004E06908B101F0DBFF2046A3
:1057A000BDE810402422002104F034BC84540220BF
:1057B00008282DE9F8431ED84FEAC008174E08EB19
:1057C00000039B00F458F518ACB10B460446114693
:1057D00018462A46D5F81C9001F09CFFE861D0B12C
:1057E00003681B689847074648B9484601F0B2FF6E
:1057F0003846BDE8F88305273846BDE8F883E869F0
:1058000001F0A8FF08EB040006EB8006C6F81C9028
:105810003846BDE8F8830427F4E700BF845402202B
:10582000F0B500EBC0000E4C8000255883B0154049
:105830008D420193044410D0636873B90F46164635
:10584000254606E06B6843B901A92046F9F776F9C9
:1058500020B92B683340BB42F4D1002003B0F0BD27
:1058600084540220274B1A6812B19A69824239D0B7
:105870005A6A12B1DA6B824236D09A6C12B11A6E41
:10588000824233D0DA6E1AB1D3F8842082422FD00C
:10589000D3F890201AB1D3F8A82082422AD0D3F8A6
:1058A000B4201AB1D3F8CC20824225D0D3F8D82026
:1058B0001AB1D3F8F020824220D0D3F8FC201AB1DC
:1058C000D3F8142182421BD0D3F820213AB1D3F867
:1058D0003831834214BF4FF0FF30082070474FF03B
:1058E000FF3070470020704701207047022070474A
:1058F000032070470420704705207047062070473A
:105900000720704784540220082807D800EBC00005
:10591000034B80001A580AB11844704700207047A2
:105920008454022019B1082802D910230B60704753
:1059300000EBC000074B80001A58002AF5D01B5816
:105940001B0C03F00A020A2A14BF03F00F0303F032
:105950000D03EBE784540220082870B527D800EB2C
:10596000C000164C800025580DB3012919D1142A06
:1059700017D183B1049A082A0DD14FF47A755A6869
:105980000F4E1968A6FB02239B0905FB0133204437
:105990000362002070BD1620F9F764F94FF0FF3064
:1059A00070BD2A20F9F75EF94FF0FF3070BD092075
:1059B000F9F758F94FF0FF3070BD00BF8454022052
:1059C000D34D621070B50828049D21D8134C00EB0C
:1059D000C000800026580444D6B1012912D1042AFF
:1059E00010D14BB145B12A68042A05D10022616863
:1059F00010461960626070BD1620F9F733F94FF058
:105A0000FF3070BD2A20F9F72DF94FF0FF3070BD3F
:105A10000920F9F727F94FF0FF3070BD84540220B8
:105A2000184B1A680AB170225A605A6A0AB1702279
:105A30009A629A6C0AB17022DA64DA6E0AB1702244
:105A40001A67D3F8902012B17022C3F89420D3F8CB
:105A5000B42012B17022C3F8B820D3F8D82012B104
:105A60007022C3F8DC20D3F8FC2012B17022C3F8F6
:105A70000021D3F8202112B17022C3F82421002084
:105A8000704700BF84540220082810B518D800EBD6
:105A9000C000114C8300E05890B1012905D00229C3
:105AA00014D1E058C0F3007010BD12F00100E258AC
:105AB0001ABF002042F0805222F08052E25010BD06
:105AC0000920F9F7CFF84FF0FF3010BD1620F9F795
:105AD000C9F84FF0FF3010BD845402202DE9F04189
:105AE000334CF9F75DF94FF00308324D324F04F1B2
:105AF000800604E0042B06D00834B4423BD014F8EE
:105B0000043C022BF6D120682A8803689BB29A4293
:105B100033D02A8A9A4232D02A8C9A4231D02A8EA5
:105B20009A4230D0B5F840209A4236D0B5F850208D
:105B30009A4234D0B5F860209A4232D0B5F870203D
:105B40009A4230D0B5F880209A422ED0B5F89020F5
:105B50009A4208BF0923CFD105EB03135A68D968CD
:105B6000904790B90122206804F8042CFB6808349F
:105B70009847B442C3D1BDE8F0810023ECE701238C
:105B8000EAE70223E8E70323E6E702280ABF042343
:105B900004F8048C04F8043CAEE70423DCE7052396
:105BA000DAE70623D8E70723D6E70823D4E700BFC0
:105BB000E4440220A84302204844022008B5A02261
:105BC0000021024804F026FA002008BDA843022064
:105BD0000388002B45D042680146002A50D0304A45
:105BE000108883423DD02DE9F047148AA34235D076
:105BF000158CAB4232D0168EB3422FD0B2F8407023
:105C0000BB422BD0B2F850C0634527D0B2F860E059
:105C1000734523D0B2F8708043451FD0B2F880900E
:105C20004B451BD0B2F890A0534517D0E0B15CB300
:105C300065B36EB377B3BCF1000F2DD0BEF1000F8A
:105C400020D0B8F1000F29D0B9F1000F0BD00920F6
:105C5000BAF1000F08D00420BDE8F0870720BDE8A6
:105C6000F087072070470820000113524B68024458
:105C700053608B6800209360CB68D360BDE8F087E9
:105C80000E2070470620EFE70120EDE70220EBE74A
:105C90000320E9E70420E7E70520E5E70720E3E73D
:105CA000A843022038B5824A0B6810889BB29842FC
:105CB00027D0108A984224D0108C984221D0108E80
:105CC00098421ED0B2F8400098421AD0B2F8500064
:105CD000984216D0B2F86000984212D0B2F8700024
:105CE00098420ED0B2F8800098420AD0B2F89020C4
:105CF0009A4206D0886818B16E4B1B6998470020FD
:105D000038BD8868002800F098806B4A1468002C21
:105D10003CD09468002C00F09A801469002C00F0AC
:105D20009A809469002C00F09A80146A002C00F08C
:105D30009A80946A002C00F08480146B002C00F090
:105D40009880946B002C00F09680146C002C00F06E
:105D50009680946C002C00F09680146D002C00F05E
:105D60009680946D002C00F09880146E002C00F04A
:105D70009880946E002C00F09680146F002C00F038
:105D80009480946F0CB1012038BD0F2402EBC40540
:105D900042F83400AB80494B1A78012A53D01A7A62
:105DA000012A41D01A7C012A4FD01A7E012A50D0F4
:105DB00093F82020012A50D093F82820012A50D0AF
:105DC00093F83020012A3AD093F83820012A4CD099
:105DD00093F84020012A4AD093F84820012A4CD059
:105DE00093F85020012A4CD093F85820012A4CD027
:105DF00093F86020012A4CD093F86820012A4AD0F9
:105E000093F87020012A4AD093F87820012A0AD00A
:105E1000102CB8D00022284B012003EBC4018A804B
:105E200043F8342038BD0F22022403EBC20003F8EC
:105E300032404160F8F7ACFFA5E71024ABE706223B
:105E4000F2E70524A2E70022EEE70222ECE70124B4
:105E50009CE70322E8E7022498E70422E4E703240E
:105E600094E70522E0E7042490E70722DCE7082214
:105E7000DAE706248AE7072488E70922D4E708241A
:105E800084E70A22D0E7092480E70B22CCE70A2422
:105E90007CE70C22C8E70D22C6E70B2476E70E222A
:105EA000C2E70C2472E70D2470E70E246EE700BFF2
:105EB000A84302204844022060440220E04402201B
:105EC000F0B4002952D0002850D08368002B4DD068
:105ED0000369002B4AD04368002B47D0C368002BCE
:105EE00044D00368002B41D04369002B3ED00126EB
:105EF000002504460F461F4A1F4BDFF880C016746A
:105F0000167682F8206082F8286082F8306082F885
:105F1000386082F8406082F8486082F8506082F809
:105F2000586082F8606082F8686082F8706082F879
:105F300078601D619D611D629D621D639D631D648E
:105F40009D641D659D651D669D661D679D67167038
:105F500016721D609D600FCCACE80F0094E8030042
:105F60008CE803003E602846F0BC70470E252846AA
:105F7000F0BC7047E0440220604402204844022004
:105F800000283AD02DE9F04780461D4C04F1A005C9
:105F9000A368103403B19847AC42F9D14FF001091E
:105FA0000026184C184DDFF864A004F1800714F89F
:105FB000043C012B05D0DAF80C302068984704F82F
:105FC000049C55F8040C083428B1DAF810309847CE
:105FD0002E8045F8046CBC4205F10805E7D1D8F8DD
:105FE00000001822013800EB40000AEBC00000213D
:105FF00004F010F80020BDE8F0870E20704700BFC5
:10600000A8430220E44402206444022048440220C1
:1060100068B171B1094A53686BB14B68088023F0CD
:10602000FF0343F0020312684B6008461047072045
:1060300070470E2070470820704700BF4844022078
:106040005AB330B300232DE9F041154F13607B683C
:106050000BB315460C46064659B998470346A8B1F6
:10606000A046DC60C3F808801E802B600020BDE8DD
:10607000F081BB6808469847804638B17B689847EE
:1060800003460028EDD13B69404698470420BDE80F
:10609000F081072070470820F9E70E20704700BF05
:1060A00048440220002800F08C80002900F0E9809C
:1060B00038B5834A5368002B00F08580814C084630
:1060C0006368994200F08580E368984200F08E8012
:1060D0006369984200F09080E369984200F09280F2
:1060E000636A984200F09580E36A984200F09880D5
:1060F000636B984200F09B80E36B984200F09E80B7
:10610000636C984200F0A180E36C984200F0A48098
:10611000636D984200F0A780E36D984200F0AA807A
:10612000636E984200F0AF80E36E984200F0B28058
:10613000636F984200F0B580E36F834200F0B8804F
:10614000D36898472378042B3FD0237A042B3CD084
:10615000237C042B39D0237E042B36D094F82030B6
:10616000042B32D094F82830042B2ED094F8303001
:10617000042B2AD094F83830042B26D094F84030E1
:10618000042B22D094F84830042B1ED094F85030C1
:10619000042B1AD094F85830042B16D094F86030A1
:1061A000042B12D094F86830042B0ED094F8703081
:1061B000042B0AD094F87830042B18BF002004D0A8
:1061C00038BD07207047082038BDF8F7E1FD0020F2
:1061D00038BD217803297FF477AF002101251846C7
:1061E000D26804F831509047002038BD217A032945
:1061F0007FF46EAF0121F1E7217C03297FF46CAFBE
:106200000221EBE7217E0329E8D0636A98427FF4FC
:106210006BAF94F8201003297FF466AF0421DDE70B
:1062200094F8281003297FF463AF0521D6E794F88A
:10623000301003297FF460AF0621CFE794F83810BF
:1062400003297FF45DAF0721C8E794F840100329C4
:106250007FF45AAF0821C1E794F8481003297FF46E
:1062600057AF0921BAE794F8501003297FF454AFCF
:106270000A21B3E794F8581003297FF451AF0B219A
:10628000ACE70E20704794F8601003297FF44CAF00
:106290000C21A3E794F8681003297FF449AF0D217E
:1062A0009CE794F8701003297FF446AF0E2195E720
:1062B00094F87830032B7FF443AF03460F218DE72A
:1062C00048440220E0440220002800F09180002988
:1062D00000F0E48038B5814A5368002B00F08A80D2
:1062E0007F4B1C68A14200F087809C68A14200F0AF
:1062F0008F801C69A14200F091809C69A14200F04E
:1063000093801C6AA14200F095809C6AA14200F033
:1063100097801C6BA14200F099809C6BA14200F019
:106320009B801C6CA14200F09D809C6CA14200F0FF
:10633000A0801C6DA14200F0A3809C6DA14200F0E2
:10634000A6801C6EA14200F0AB809C6EA14200F0C2
:10635000AE801C6FA14200F0B1809C6F8C4200F0B7
:10636000B4801369084698475E4B1A78042A3BD0DC
:106370001A7A042A38D01A7C042A35D01A7E042AC4
:1063800032D093F82020042A2ED093F82820042A13
:106390002AD093F83020042A26D093F83820042AF3
:1063A00022D093F84020042A1ED093F84820042AD3
:1063B0001AD093F85020042A16D093F85820042AB3
:1063C00012D093F86020042A0ED093F86820042A93
:1063D0000AD093F87020042A06D093F87830042B62
:1063E00018BF002000D038BDF8F7D2FC002038BD1F
:1063F00007207047082038BD9C8884427FF475AF21
:106400000024002003EBC40543F83400A880A8E76B
:106410009C8984427FF46DAF0124F2E79C8A844218
:106420007FF46BAF0224ECE79C8B84427FF469AF6E
:106430000324E6E79C8C84427FF467AF0424E0E702
:106440009C8D84427FF465AF0524DAE79C8E8442FC
:106450007FF463AF0624D4E79C8F84427FF461AF5E
:106460000724CEE7B3F8444084427FF45EAF0824AB
:10647000C7E7B3F84C4084427FF45BAF0924C0E720
:10648000B3F8544084427FF458AF0A24B9E7B3F814
:106490005C4084427FF455AF0B24B2E70E20704776
:1064A000B3F8644084427FF450AF0C24A9E7B3F8FA
:1064B0006C4084427FF44DAF0D24A2E7B3F87440E2
:1064C00084427FF44AAF0E249BE7B3F87C408442B9
:1064D00008BF0F247FF445AF93E700BF4844022074
:1064E00060440220E044022010B5044618B1006860
:1064F00008B101F029F8A06818B1BDE81040FAF71A
:1065000077B810BD2DE9F041644B064600681B8842
:106510000268634FB3EB124F84B00D46386038D039
:1065200005F53F43FF339BB2022B10D85D4C236827
:106530005A0710D423689B0703D544F203039D42F6
:1065400009D0306818B100F0FFFF00233B60002045
:1065500004B0BDE8F0810220FAF740F88046002838
:1065600000F0938002230580316872684E488DE800
:10657000060100680393036869465B689847013029
:1065800070D00020236843F48033236004B0BDE85A
:10659000F081444C2368D90123D542F202139D4275
:1065A0001FD143681BB9236843F00073236023683D
:1065B00023F08073236023685A0230D442F205032B
:1065C0009D422CD12368990229D54368002B57D1CD
:1065D000236823F400132360236843F4003323600B
:1065E0001DE023685B020ED542F203139D420AD1DF
:1065F00043681BB9236843F400032360236823F432
:10660000800323600BE042F201039D420CD14368FA
:106610002BB923681B0C1B0443F00203236000F01A
:1066200093FF00233B607BE742F204039D42C5D108
:10663000436893B9236843F40003236023689BB243
:10664000032B236816D09BB2042BD7D123681B0CD5
:106650001B0443F002032360D0E723689BB2032BA3
:10666000CCD1F3E74046F9F7C3FF306800287FF448
:106670006AAF6CE71B0C1B0443F004032360BDE707
:10668000236823F400132360C9E7306800283FF42F
:106690005EAF00F059FFC7F8008058E75C4C02205D
:1066A0006445022060450220684502202DE9F04340
:1066B000754A9FB09042269D40F0D480002900F09A
:1066C000C980002D00F0C680279A022A40F0C280BF
:1066D0006E4C226892B2022A04D0226892B2042A36
:1066E00040F0C680980700F1C980206810F400309F
:1066F00065D022682B8822F4003222602268013B98
:1067000042F400122260072B00F2A480DFE803F0BD
:1067100078736E69645A5F04084602A900F0C8FEE7
:106720007221684600F0DEFE05460098002D6CD10F
:10673000002871D041F205064FF0490C72224FF04B
:10674000760E4FF043094FF05408514F1EA93B8875
:1067500080F80FC001339BB246EA034C41F874CD78
:1067600045718571C571057245728572C572027178
:1067700080F80C9080F80D8080F80EE000683B8077
:1067800003F01EFC434B314600981D6000F0BEFE36
:10679000002848D1236899020DD53F4E3A4D01E0BB
:1067A000002850D131462846F8F7C8F923689A02E4
:1067B000F6D4002847D123689B033FD500201FB0A3
:1067C000BDE8F083084602A900F02AFEA8E70846C3
:1067D00002A900F04DFEA3E7084602A900F006FE5C
:1067E0009EE7084602A900F0DDFD99E7084602A9E8
:1067F00000F0A6FD94E7084602A900F04FFD8FE7E0
:10680000084602A900F028FD8AE728B103681BB1F9
:10681000184600F099FE009800F08EFE2320F8F74D
:1068200021FA4FF0FF30236823F40013236023681C
:1068300043F4003323601FB0BDE8F08305202368D4
:1068400043F400332360F8F70DFA4FF0FF301FB028
:10685000BDE8F0831620F8F705FA4FF0FF301FB0BF
:10686000BDE8F0830920F8F7FDF94FF0FF30A6E707
:106870003920F8F7F7F94FF0FF30A0E72D20F8F7AF
:10688000F1F94FF0FF309AE7435476496045022012
:106890005C4C022064450220AC9D02202DE9F04FA3
:1068A0004A4CB7B0A04240F0EC818846002900F085
:1068B000E281D72A40F2DF81454D99462B689BB291
:1068C000042B04D02B689BB2022B40F0E081022104
:1068D000B62000242B680DF10E0223F480332B60C8
:1068E000DFF8F4A008AB3B4F384E059007910493B6
:1068F000069209EA010BDAF800004A46036804A987
:106900009B689847002811DABBF1000F38D12B683B
:10691000D803F0D40CB1EEE730B939463046F8F779
:106920000DF92B68D903F7D50446E4E744F20202D7
:10693000BDF80E30934239D044F2010293424DD05B
:1069400044F20302934240F0968103221424089BF0
:1069500088F80020099AC8F80830BDF82830C8E93E
:106960000323DAF800000368DB689847002803DD9A
:106970002B6843F480332B60204637B0BDE8F08F9E
:10698000421C0346D2D13CB91C462320F8F76AF9D1
:10699000204637B0BDE8F08F01902046F8F762F945
:1069A000019B1C46204637B0BDE8F08F08A803F0D5
:1069B000D5FA0223441CA4B208F8083B224608A9D1
:1069C000404603F0FDFA0834CBE700BF4354764954
:1069D00060450220AC9D022068450220012409A8E0
:1069E0000FC8C8E90201C8E904230D990E9A88F876
:1069F00000400F9BC8F818101099C8F81C20C8F860
:106A000020309DF85D20DDF84D30C8F82410DDF809
:106A1000511088F84420DDF85520C8F83430DDF8EE
:106A20005930C8F83810BDF84410C8F83C20C8F8F0
:106A30004030DDF846209DF84A30A8F8281088F844
:106A40002E30C8F82A209DF84B009DF84C20189B4A
:106A50009DF86C4040EA02209DF86B20C3F30F21A3
:106A60001D9B42EA0422A8F83000A8F84A10BDF89D
:106A70005E10C3F30F23A8F856209DF86020A8F8F5
:106A80006230DDF86330A8F8461088F84820BDF879
:106A900068209DF86710C8F84C309DF86A3088F877
:106AA0005010A8F8522088F85430BDF87230DDF844
:106AB0006D109DF87120C8F8581088F85C209DF87A
:106AC0007410DDF87720A8F85E309DF87B3088F8E8
:106AD0006010C8F8642088F868309DF880309DF810
:106AE0007F10229A9DF8940041EA03219DF893308B
:106AF000C2F30F22A8F86E10BDF87C1043EA002301
:106B0000A8F87A209DF87E20A8F88630DDF881303C
:106B1000A8F86A1088F86C20BDF886209DF88510CA
:106B2000C8F870309DF8883088F87410A8F876207E
:106B300088F87830BDF89030DDF88B109DF88F2004
:106B4000C8F87C1088F880209DF89210DDF8952018
:106B5000A8F882309DF8993088F88410C8F8882009
:106B600088F88C30BDF89A00279B9DF8A8409DF8C6
:106B7000A720C3F30F212C9B42EA0422A8F892100D
:106B80009DF89C10A8F89E20C3F30F23DDF89F20EA
:106B9000A8F88E00A8F8AA3088F890109DF8A330C5
:106BA000BDF8A410C8F894209DF8A62088F8983065
:106BB000DDF8A930A8F89A1088F89C20BDF8AE201E
:106BC0009DF8AD10C8F8A0309DF8B03088F8A4103A
:106BD000A8F8A62088F8A830BDF8B830DDF8B310C2
:106BE0009DF8B720C8F8AC1088F8B020A8F8B230EB
:106BF0009DF8BC309DF8BB109DF8D000319A41EA59
:106C000003219DF8CF309DF8BA4043EA0023C2F338
:106C10000F22A8F8B610A8F8CE3088F8B440A8F82B
:106C2000C220BDF8C2209DF8C1109DF8C430DDF827
:106C3000BD0088F8BC10A8F8BE20C8F8B80088F8D5
:106C4000C030BDF8CC30DDF8C7109DF8CB20C8F8B7
:106C5000C41088F8C8209DF8CE10DDF8D120A8F81F
:106C6000CA309DF8D53088F8CC10C8F8D02088F804
:106C7000D430D82475E61620F7F7F4FF4FF0FF3430
:106C80007AE60920F7F7EEFF4FF0FF3474E639207B
:106C9000F7F7E8FF4FF0FF346EE600BF2DE9F0474D
:106CA00041F20214224286B09C4D04D02C68A4B25A
:106CB000022C40F004812C68640200F12881B1F5B7
:106CC000017F40F01E819649884240F01481013ACC
:106CD000082A00F2EC80DFE812F07500D800C2004C
:106CE000CC0081008C009800AF0009000E9A012AA8
:106CF00040F0DD8041F20316402237461B780292B5
:106D00008DF815302B68122143F4800368462B6000
:106D100000F0E8FB04460098002C40F0D6800028E4
:106D200000F0DA8012224FF076084FF0490E4FF053
:106D3000430A4FF05409DFF8F0C106A9BCF800304F
:106D400080F80E8001339BB246EA034641F8146D89
:106D500044718471C471047244728472C472027189
:106D600080F80CA080F80D9080F80FE0DFF8BC816F
:106D70000068ACF8003003F023F939460098C8F8F1
:106D8000004000F0C3FB002840F0AB80654F644E2C
:106D900039463046F7F7D2FE2C6814F48004F7D158
:106DA000D8F8000018B100F0CFFBC8F800402B68FD
:106DB0001B0276D500202B6823F400032B6006B05D
:106DC000BDE8F0870E9A022A71D1082241F203161B
:106DD0001B880292ADF80F30374693E70E9A012ACE
:106DE00065D141F203161B7802928DF80C303746BC
:106DF00088E70E9A012A5AD1022241F203161B7823
:106E000002928DF80D3037467CE72A6892B2022A4A
:106E100055D10E9A042A4AD1012141F204062A686A
:106E20001868130C1B0443F00303CDF809002B6012
:106E30008DF80810374665E72B689BB2042B3ED1CE
:106E4000002341F204068DF808308DF809308DF8E2
:106E50000A308DF80B308DF80C30374652E70E9A19
:106E6000012A24D11B78012B21D141F20316374688
:106E700048E70E9A022A1AD1202241F203161B88F3
:106E80000292ADF8133037463CE70E9A022A0ED133
:106E9000102241F203161B880292ADF811303746DA
:106EA00030E70E20F7F7DEFE4FF0FF3083E71620C5
:106EB000F7F7D8FE4FF0FF3006B0BDE8F0870E20A0
:106EC000F7F7D0FE4FF0FF3079E728B103681BB128
:106ED000184600F039FB009800F02EFB2320F7F74E
:106EE000C1FE2B680E2023F480032B60F7F7BAFE57
:106EF0004FF0FF3063E70920F7F7B4FE4FF0FF30A3
:106F00005DE72A20F7F7AEFE4FF0FF3057E773201A
:106F1000F7F7A8FE4FF0FF3051E700BF60450220B1
:106F200043547649AC9D02205C4C0220644502200B
:106F30002DE9F04F814C87B025689846ADB2022DFF
:106F4000109B40F0DD802568EE0300F1EB802568A2
:106F5000ED0100F1ED80B1F5017F40F0D780784977
:106F6000884240F0D980B8F1000F0BD053B1571EC2
:106F7000052F07D8DFE807F00F0F030F03031B6887
:106F8000012B0BD01620F7F76DFE4FF0FF3528468A
:106F900007B0BDE8F08F1B68022BF3D123681222E3
:106FA00043F08073002101A8236003F033F812211D
:106FB000684600F097FA05460098002D40F08A8058
:106FC000002800F08E8041F202164FF0490E122286
:106FD0004FF076094FF0430B4FF0540ADFF868C1C9
:106FE00080F80FE0BCF8003080F80E9001339BB2BF
:106FF00046EA034ECDF804E045718571C57105720E
:1070000045728572C57201A9027180F80CB080F8D2
:107010000DA0DFF838910068ACF8003002F0D0FF26
:1070200031460098C9F8005000F070FA00285DD190
:10703000444E434D31462846F7F780FD2368DB0177
:10704000F8D4D9F80000D8B1256815F000750FD034
:10705000052F37D8DFE807F01A20262B310300254B
:10706000437B88F8003000F06FFA0023C9F8003045
:10707000236823F000732360284607B0BDE8F08F33
:107080002368054623F000732360F5E7B0F80F305E
:107090000025A8F80030E6E7B0F811300025A8F880
:1070A0000030E0E7837B002588F80030DBE7B0F8AC
:1070B00013300025A8F80030D5E7037B002588F8B9
:1070C0000030D0E71620F7F7CDFD4FF0FF35D9F8A7
:1070D0000000C8E728B103681BB1184600F034FA75
:1070E000009800F029FA2320F7F7BCFD23680E2052
:1070F00023F0807323604FF0FF35F7F7B3FD46E7C9
:107100000E20F7F7AFFD4FF0FF3540E72A20F7F7E5
:10711000A9FD4FF0FF353AE70920F7F7A3FD4FF03F
:10712000FF3534E70520F7F79DFD4FF0FF352EE7DB
:107130007320F7F797FD4FF0FF3528E760450220F1
:1071400043547649AC9D02205C4C022064450220E9
:10715000002138B5094C0A4D22680A480A4B2A40DA
:1071600022600180196000F0B7F928B923682B402C
:1071700043F00103236038BD032038BD6045022081
:107180000000FFFF5C4C022064450220012810B57E
:1071900020D1B2F5017F1DD102291BD1134C2368E8
:1071A0009BB2012B1CD1236808461B0C1B0443F027
:1071B000020300220E49236000F0ACFA0D4A106071
:1071C00070B12368026843F400331268236090476B
:1071D000094810BD1620F7F745FD4FF0FF3010BDF0
:1071E0000E20F7F73FFD4FF0FF3010BD6045022045
:1071F000E9640100684502204354764930B5134BD9
:1072000083B098421CD1124C23689BB2042B0FD040
:10721000104D286818B100F09DFA00232B60002063
:1072200023681B0C1B0443F00103236003B030BD33
:107230000023082200934FF40171FCF78BFEE7E76F
:107240000920F7F70FFD4FF0FF30EFE74354764981
:1072500060450220684502200346D8B1D1B1002024
:10726000012248700A705A681020C1F806201A6876
:10727000C1F8022093F90A200A7393F90D20CA730A
:1072800093F90C208A731A7A8A72DA7A4A735B7AD3
:10729000CB7270474FF0FF30704700BF03460028A5
:1072A0004BD0002949D00020022248700A70DA68C9
:1072B0004020C1F80B20B3F90820A1F8092093F968
:1072C00006200A72B3F944208A87B3F93E20CA86A1
:1072D000B3F942204A87B3F93C208A86B3F94620A5
:1072E000CA87B3F940200A87B3F91C200A839A6A37
:1072F000C1F822209A7C4A745A78CA705A6BCA62C2
:10730000B3F92C20CA845A888A801A6AC1F81A20D4
:107310009A6B0A635A6AC1F81E201A6B8A621A783D
:107320008A7093F91020CA739A88CA809A8A4A820E
:107330005A7C0A749B694B6170474FF0FF3070476D
:10734000034660B359B30020032248700A70B3F9B2
:107350001C202120A1F81D20B3F91E20A1F81F2018
:10736000B3F906200A819A88CA80DA784A719A6944
:10737000C1F819201A69C1F81120B3F908204A810F
:10738000DA68C1F80D209A7A0A731A788A709A78A6
:107390000A715A69C1F815205B78CB7070474FF0BD
:1073A000FF3070470346F0B1E9B100200422487075
:1073B0000A7093F900200A208A7093F90120CA709C
:1073C00093F902200A7193F903204A7193F904207A
:1073D0008A7193F90520CA7193F906200A7293F90C
:1073E00007304B7270474FF0FF307047034698B13B
:1073F00091B10020052248700A70B3F900200A20DC
:107400004A80B3F902208A80B3F90420CA809A79AD
:107410000A72DB794B7270474FF0FF30704700BF44
:1074200010B309B370B4002506260C464D700E70DB
:107430002B46058802464D80C568C1F80A5005896B
:107440000D8140684860158A03EB43000844C581FC
:10745000907C0133202B207402F1040204F1030418
:10746000F1D16E2070BC70474FF0FF30704700BF05
:107470000346C8B1C1B10020072248700A70B3F9B1
:10748000082011204A819A7B0A741A68C1F80220E8
:107490005A68C1F806201A7B8A735A7BCA739A7A93
:1074A0000A73DB7A4B7370474FF0FF30704700BFB1
:1074B00048B141B1002208234A700B7003680620CE
:1074C000C1F8023070474FF0FF30704750F8081B8A
:1074D000090CFFF717B800BF0148FEF779BB00BFE2
:1074E000B4BF0100002310B582B0019358B1044627
:1074F00001AA0720FEF7A4FD18B9019B0BB10833C0
:10750000236002B010BD072002B010BD01F470432B
:10751000B3F5805F0BD160B1034630F8082C07202B
:1075200042EA014143F8081D1946FEF771BD0F20DC
:1075300070470720704700BF20B1A0F10801072065
:10754000FEF7B0BD0720704718B101460720FEF7CF
:10755000BBBE0720704700BF10B504460C20F9F7EA
:107560003DF8E06018B1BDE81040FCF7E9BB04202D
:1075700010BD00BF70B5064614200D46F9F72EF871
:1075800078B12B68044643606B6801468360EB6802
:10759000C360AB680361F068FCF7DCFB20B9686886
:1075A00070BD4FF0FF3070BD2046F9F721F84FF065
:1075B000FF3070BDF0B5064685B0C0680C46174672
:1075C000FCF7E8FB002837D082680546D4E90003C1
:1075D0009A4228BF1A46626010B1696802F0F0FC56
:1075E000A06818B12B690BB1EA68E2B90023E36027
:1075F0003B0702D5606805B0F0BDF068FCF7C0FB42
:1076000005460028F6D0D0E9013102690093C3682D
:10761000CDE9011203936846D6E90131984728461F
:10762000F8F7E6FFE6E7E3689A4228BF1A46E26009
:10763000296902F0C5FCDBE74FF0FF30DBE700BF54
:1076400008B5C068FCF7A6FB08B1806808BD4FF01C
:10765000FF3008BD30B50546C06885B0A8B91AE04E
:10766000E868FCF78DFB044670B1D0E90101D4E96C
:107670000332CDE90001CDE90223D5E901316846A5
:1076800098472046F8F7B4FFE868FCF789FB002824
:10769000E6D105B030BD082005B030BD30B5054697
:1076A000C06885B0A0B91CE0FCF76AFB044670B165
:1076B000D0E90101D4E90332CDE90001CDE902238B
:1076C000D5E90131684698472046F8F791FFE86808
:1076D000FCF766FB0446E868002CE5D1F8F788FF64
:1076E000EC6005B030BD00BF0020704710B50C46FF
:1076F000D0E9013120469847606810BD4FF0FF3057
:10770000704700BF4FF0FF30704700BF0020704748
:10771000704700BF012838B50D4614460DD011DB67
:1077200003280FDC1020F8F759FF182220B1084B6E
:10773000456013448460036038BD1420F8F74EFFA1
:107740003022F3E70C20F8F749FF0022EEE700BFF4
:10775000C4BF010010B5044603681B69984723683D
:1077600020465B6998472046BDE81040F8F740BFC7
:1077700010B504460C20F8F731FFE06028B1002373
:107780002361BDE81040FCF7DBBA042010BD00BF48
:1077900070B5064614200D46F8F720FF78B12B6827
:1077A000044643606B6801468360EB68C360AB6866
:1077B0000361F068FCF7CEFA20B9686870BD4FF03D
:1077C000FF3070BD2046F8F713FF4FF0FF3070BD5B
:1077D0002DE9F04F824687B0C06889469346FCF792
:1077E000D9FA002872D00546D9F8080020B12B69D3
:1077F00013B1EA68002A5CD10023C9F80C30D9F82B
:107800000020D9F80480DAF810100192B8F1000FC6
:107810005AD00BF008030024009310E0DAF810307F
:107820003B44CAF810302846FCF7BCFA3C440546F5
:10783000002838D0A04536D90021D9F80020AE68FC
:10784000A8EB040B761A5E45374628BF5F4632B177
:107850006868019B01443A46181902F0B1FB009B8D
:10786000002BE0D15E45D9D8DAF80C00FCF788FA95
:10787000064670B1D0E90123D0E90301CDE9022326
:10788000CDE90410DAE9013102A898473046F8F74B
:10789000AFFE00232846CAF81030FCF783FA3C44B8
:1078A00005460028C6D12046C9F8044007B0BDE807
:1078B000F08FD9F80C309A4228BF1A46C9F80C202C
:1078C000296902F07DFB9AE74446ECE74FF0FF3070
:1078D000ECE700BF10B50446C068FCF75BFA50B196
:1078E0002469644283681C44FCF75CFA0028F9D1DF
:1078F00024EAE47010BD4FF0FF3010BD30B50546EE
:10790000C06885B0A8B91AE0E868FCF739FA0446FF
:1079100070B1D0E90101D4E90332CDE90001CDE92C
:107920000223D5E90131684698472046F8F760FE02
:10793000E868FCF735FA0028E6D105B030BD08202C
:1079400005B030BD30B50546C06885B0A0B91CE0B3
:10795000FCF716FA044670B1D0E90101D4E903320C
:10796000CDE90001CDE90223D5E901316846984708
:107970002046F8F73DFEE868FCF712FA0446E8688E
:10798000002CE5D1F8F734FEEC6005B030BD00BF47
:10799000074AD2F8883043F47003C2F88830BFF346
:1079A0004F8FBFF36F8F034B034A1A60704700BFBE
:1079B00000ED00E0B09D02200090D00370B50026DD
:1079C000084B53F82040013053F82050A54200D80E
:1079D00070BD236820465B68984700B166600C3430
:1079E000F4E700BF0CC00100104B70B505461E4601
:1079F0000F4C9C4204D10E4CB44209D1002412E039
:107A000062681AB122681268AA420CD00C34F0E7FE
:107A100063680BB90C34EFE723682846196802F055
:107A2000A4FA0028F6D1204670BD00BF0CA00220A9
:107A30001C9F0220044A054B02609B1A044A9B10BB
:107A400053430B60704700BF1C9F02200CA0022014
:107A5000ABAAAAAA014B986874307047304B022039
:107A600008B50B4D4FF02002EFF3118382F311881C
:107A7000BFF36F8F03F050FD012104460228D8BFE9
:107A8000084603F059FD2C62F5F78EFAEAE700BFCD
:107A9000304B02200248034A0021121A02F0BABAFF
:107AA00000000220C855022008B50648064A0749CA
:107AB000121A02F085FABDE80840054A0549064851
:107AC00002F07EBAB89702207CA2022078C10100A1
:107AD0000000000078C1010000000220012208B56A
:107AE0000B4B02201A70FFF769FF0A4A0A490B483C
:107AF00001F057FF0320FFF761FF01F013F901F0D8
:107B000015FC074A137B23F00103137308BD00BF64
:107B10008254022054C1010021C101002EC1010084
:107B20003C46022080B5344BBAB083F30888002469
:107B3000E023324D012785F82230EC772C766C76E5
:107B4000AC766B6A2E4E43F4E0236B62F5F70AFCC9
:107B5000F5F724FA4FF0FF33AB62EB6206ABD022AD
:107B60002146184602F056FAB06020468DF825707E
:107B7000FFF724FF3846FFF721FF224D00F008FFF2
:107B8000214B4FF40062CDE90473CDE902441F4B51
:107B9000CDE900441E492846756201F04DF86B7B23
:107BA00023F0040213F01B0F6A7304D1AB6913B9FD
:107BB000284600F0B3FC174B012205930F23CDE9B3
:107BC00003320023144DCDE9013300934FF4A0722A
:107BD000124B1349284601F02FF86B7B4FF40062DB
:107BE00023F004036B730F4B0949C6E906330548BC
:107BF000064BF560F5F784FA087B022000ED00E003
:107C0000304B02203C46022055C10100DD7A0100C4
:107C1000C86902205AC101006C450220617A010046
:107C2000C8710220484B0220334B2DE9F14F9B686D
:107C3000D1F82480CB61074689469346C8F81410D2
:107C400000F1100A4FF02003EFF3118683F311883F
:107C5000BFF36F8F014651F8084F8C4216D1BBF12C
:107C6000000F36D186F31188BFF36F8F6FF04F0589
:107C70002BE04FF0FF333146504601B0BDE8F04FE6
:107C800000F002BEFB689C42E9D02468002CE6D0DC
:107C90006169484603F080F905460028F2D1204684
:107CA00003F027FB637BC4F88850DA0604D1A3698C
:107CB00013B9204600F032FC98F80D2012F00102B2
:107CC000D7D03146504603F0F3FA284601B0BDE85C
:107CD000F08F98F80D30DB070BD54FF0FF323946A7
:107CE000404603F05BFB86F31188BFF36F8F0025DE
:107CF000EBE75B463A46BEE7304B022070B5002505
:107D0000094C0A4E002301221946204603F0E6FBE7
:107D100021463046013503F096FB0A2D04F1540448
:107D2000F0D1002070BD00BF70940220D8A10220C5
:107D3000436A10B50446002B33D0436923B1143095
:107D400003F090F9002363610023616A63624A696A
:107D5000636853604B7B13F0010009D0946A1148AB
:107D600003F071FBECB12046BDE8104000F096BE78
:107D700023F0020213F01D0FC1F888004A7304D1EA
:107D80008B6913B9084600F0C9FB4FF02003EFF3ED
:107D9000118083F31188BFF36F8FBDE8104003F0AB
:107DA00092BA10BDD8A102202DE9F34107460C4636
:107DB00090464FF0FF3201A90E4800F0C1FE0E4B75
:107DC000019E9B6806F128059B7BB3730FCC0FC502
:107DD0000FCC0FC594E8070085E80700C6E91368D3
:107DE0004FF0FF3206F128013846FFF71DFF02B0C1
:107DF000BDE8F081D8A10220304B02202DE9F047E8
:107E0000254F9A46BB6806460D4690460B624FF0DA
:107E10002003EFF3118983F31188BFF36F8F046898
:107E2000A04213D1BAF1000F29D189F31188BFF311
:107E30006F8F6FF04F0020E06B68EBB92846FFF7BB
:107E400077FF19E073689C42ECD02468002CE9D0DD
:107E50002946606903F0A0F80028F3D1204603F01A
:107E600048FA89F31188BFF36F8FB8F1000FE3D0A0
:107E70004146284603F0C1F80020BDE8F087BB6802
:107E800006F108025D614946534606F1100000F014
:107E9000FBFC0028F1D1E8E7304B022070B50E4B17
:107EA0000E4CA34201D3002070BDD3E9030141EA87
:107EB000000212F003020BD19D685A61AA4201D15F
:107EC0001C33EEE75E6901320E6059610144F5E74B
:107ED0006FF01500E8E700BFD0A00220ECA0022060
:107EE00010B513460C464FF02002EFF3118182F3D8
:107EF0001188BFF36F8F42695AB1226013684361E2
:107F0000836901338361002081F31188BFF36F8F90
:107F10000DE01BB923606FF00B00F5E70246044843
:107F200000F0B2FC18B9034B9B685B69236010BD7D
:107F300083540220304B022070B504460D464FF0AA
:107F40002003EFF3118683F31188BFF36F8F03F0E3
:107F500027FA88B100212A68C0F888104261427B64
:107F6000D20603D183690BB900F0D8FA3146BDE8D7
:107F70007040084803F09CB92B6862691A602B684E
:107F80006361A369013BA36186F31188BFF36F8F1F
:107F900070BD00BF8354022038B5074C074DAC427A
:107FA00001D3002038BD04F114032046C4E9053391
:107FB00001F0E5F91C34F2E7ECA002205CA10220FC
:107FC0002DE9F04F1C1E85B007460D4692463BDD5D
:107FD00003F0D0FA10EB04081D4B1E4EFB1A9B1049
:107FE0005E4307F1140BF6B203AB02AA00955146AB
:107FF000384601F00AFA6B79029A2E7162F3030394
:108000006B716B68039A62F31F336B60C8B1C4B1C4
:1080100010F10C0F15D14FF02003EFF3118083F313
:108020001188BFF36F8F2246594600F009FC631C8C
:10803000DAD003F09FFAA8EB0004002CD4DC6FF038
:108040000A0005B0BDE8F08F4FF00008C4E700BF9C
:10805000ECA00220B76DDBB670B5047802684178F9
:10806000114EC4EBC404A400120B01F00F0130192F
:1080700001F07DFA4FF02003EFF3118583F31188AF
:10808000BFF36F8F04F11400304403F0B6F928B148
:108090002946BDE87040054803F00AB985F3118808
:1080A000BFF36F8F70BD00BFECA00220835402208D
:1080B0000146014802F0D9BF40A1022010B5044694
:1080C00003F0F5F950B9074B9B68D3F880303BB10A
:1080D0002146BDE81040184602F0C7BF024BF7E743
:1080E00010BD00BF304B022040A102202DE9F0411D
:1080F000134604460F4600F108084FF02002EFF344
:10810000118682F31188BFF36F8F016AC2689142B2
:108110002FD203F045F9A26805463946A0B140695F
:1081200001F04EFF0023C5F888306B7BDB0604D1DD
:10813000AB6913B9284600F0F1F94046314603F027
:10814000B7F80020BDE8F081E06901F039FF0020B8
:10815000E369A26813446269E361934204BF23693F
:10816000E361236A0133236286F31188BFF36F8FC3
:10817000E8E74BB1064A31469268576102464046ED
:10818000BDE8F04100F080BB6FF04F00ECE700BFAE
:10819000304B02202DE9F04104461346084604F115
:1081A00008074FF02002EFF3118682F31188BFF326
:1081B0006F8F226A002A38D0A268A16901F000FFFF
:1081C000A369A268204613446269A361934204BF75
:1081D0002369A361236A013B236203F0E1F80546AA
:1081E00000282FD0A2684169E06901F0E9FEE36947
:1081F000A26813446269E361934204BF2369E361A7
:10820000236A013323620023C5F888306B7BDB06C9
:1082100004D1AB6913B9284600F080F938463146DD
:1082200003F046F80020BDE8F0814BB1084A38461B
:108230009268516122463146BDE8F04100F024BB0E
:108240006FF04F0086F31188BFF36F8FEBE700BF2D
:10825000304B0220F8B504460F464FF02003EFF3F1
:10826000118583F31188BFF36F8FC26830495AB10B
:1082700080688E68B04215D0B7B985F31188BFF316
:108280006F8F6FF00F000CE08B6893F90E30236155
:108290008B680132E260A36085F31188BFF36F8FB2
:1082A0000020F8BD2369F2E790F90E3096F90E1020
:1082B0009942A8BF194621EAE17199422BDA00F0F0
:1082C00025FB06463B46224629461A4800F0DCFAC2
:1082D0000028E6D04FF02003EFF3118583F31188D7
:1082E000BFF36F8F236821699C4207D033B193F9A4
:1082F0000E309942A8BF194621EAE171A06890F9B1
:108300000E30994209D16EB129460A4802F0D0FFD9
:108310006FF00A00C5E70026D4E700F0F7FA00285E
:10832000F2D1F0E785F31188BFF36F8FF0E700BF5C
:10833000304B02208354022038B583680446002B5A
:108340003CD0214A926893423BD1DA7B013ADA73FE
:10835000C368012B05D0013BC36000F0C3F80020C7
:1083600038BD4FF02003EFF3118583F31188BFF37D
:108370006F8F0169806890F90E30994201D000F04A
:10838000C5FA204603F00CF8A06088B190F90E20E1
:1083900022610022C0F88820427BD20603D1836983
:1083A0000BB900F0BBF82946084802F081FFD4E77A
:1083B000E06085F31188BFF36F8FCEE76FF0150093
:1083C000CEE74FF0FF30CBE7304B02208354022042
:1083D00010B5084C23685BB1F4F7EAFC2368064A41
:1083E000184410610021BDE81040184603F0A4B8FD
:1083F00010BD00BF6C4B0220304B0220F8B50D467B
:108400004FF02003EFF3118483F31188BFF36F8FD4
:108410004FF4004140F2E73600270022E1FB0067FD
:10842000094B30461A6139464FF47A720023F3F74C
:1084300005FF064B1860064B1D60FFF7C9FF84F36C
:108440001188BFF36F8FF8BD304B02206C4B0220B8
:10845000684B02204FF02003EFF3118183F3118862
:10846000BFF36F8F044B9A68D37B013BD37381F3C7
:108470001188BFF36F8F7047304B0220094B03F117
:108480002802824205D19B688B4202D14B7BDB06DE
:1084900006D1D1E9003213605A600023C1E90033EC
:1084A000704700BF304B022038B50D4C024604F136
:1084B000280002F03CFF054600B9E568A3684AB908
:1084C0005A7BD20606D1AA6922B9DA897F2A01D954
:1084D000636238BD9D4201D0FFF77AFF6562F8E71D
:1084E000304B022010B54FF02003EFF3118483F3DB
:1084F0001188BFF36F8F084B00209A68D37B01333C
:10850000D373FFF7D1FF84F31188BFF36F8FBDE8FA
:10851000104002F0E4BE00BF304B0220F8B54FF02F
:108520002003EFF3118483F31188BFF36F8F154A93
:10853000114651F8283F8B421DD0E3B1D66A90F91D
:108540000E5093F90E70AF4210DD5A68C0E9003248
:1085500010605860437B63F07F0343730020FFF794
:10856000A3FF84F31188BFF36F8FF8BDB34202D02D
:108570001B68002BE5D1D36A01604360D36A1860A1
:10858000D062E7E7304B0220F8B504464FF02003F5
:10859000EFF3118583F31188BFF36F8F90F90D30DE
:1085A000002B03DA01461848FFF768FF174A02F16B
:1085B0002801D2E90A308B421FD0F3B194F90E6042
:1085C00093F90E70B74213DD5968C4E900310C60AD
:1085D0005C60637B906863F07F036373031B5842A6
:1085E0005841FFF761FF85F31188BFF36F8FF8BD26
:1085F000984202D01B68002BE2D1C4E90010D36A74
:108600001C60D462E5E700BF584B0220304B0220CB
:10861000154A164938B50C689368A342144603D12D
:10862000BDE83840FFF7D4BE00250D601049096849
:10863000B9B1D9897F2914D80E4993F90E50096828
:108640008D420EDB0C498B420BD0996949B91169F7
:10865000814203DC1846FFF797FFE1E7091A116131
:1086600038BD00232361FBE7304B0220644B02201E
:108670006C4B0220684B02206C45022070B504460A
:10868000183002F033FF4FF02003EFF3118683F32D
:108690001188BFF36F8F94F90D30002B07DA214654
:1086A0000E48FFF7EBFE637B03F07F0363730C4D13
:1086B000637BA86843F010036373031B584258415F
:1086C000FFF7F2FE86F31188BFF36F8FAB68A3420A
:1086D00003D1BDE8704002F002BE70BD584B0220CD
:1086E000304B0220036D70B5044603B1984704F186
:1086F000180002F0FBFE4FF02003EFF3118583F327
:108700001188BFF36F8F204602F097FD0646D8B15F
:1087100094F90D30002B07DA21461248FFF7AEFE20
:10872000637B03F07F0363730F4B9868021B504217
:108730005041FFF7B9FE637B43F00803637385F391
:108740001188BFF36F8F70BD637B9B07F3D5214604
:10875000A068FFF793FE637BA66023F002036373B8
:10876000E9E700BF584B0220304B022038B50446E1
:108770004FF02003EFF3118583F31188BFF36F8F60
:1087800090F90D30002B07DA01460948FFF776FE15
:10879000637B03F07F036373064B9868031B5842A7
:1087A0005841FFF781FE85F31188BFF36F8F38BD05
:1087B000584B0220304B022070B504460D46164639
:1087C000FFF7D4FF637B43F0020363737DB12B6833
:1087D000A5609D4229D043B394F90E2093F90E1061
:1087E00091421CDD5A68C4E9003214605C60731C5D
:1087F00022D04FF4004540F2E730002126EAE67629
:108800004FF47A72C5FB06010023F3F717FD0B49FD
:10881000421C04F11800BDE8704000F03BBB6968E1
:108820008B4202D01B68002BD8D16B682560636037
:108830006B681C606C60DAE770BD00BF3BB3010081
:1088400070B506460E4D0F4CA868FFF7B5FFAB6834
:1088500030462360F4F7DCFB4FF02002EFF3118386
:1088600082F31188BFF36F8F2268A968914204BF19
:108870000022226083F31188BFF36F8F70BD00BFA9
:10888000304B0220644B022010B50C461146064ABC
:108890009068064A10601A46FFF78EFF2046BDE832
:1088A0001040F4F7B5BB00BF304B0220644B0220F0
:1088B000F8B5461C02F05AFE34184FF02003EFF3CF
:1088C000118783F31188BFF36F8F0D4D0D4BA8688F
:1088D0001860FFF74BFFA8680B493246183000F0CC
:1088E000D9FAAA683846537B43F010035373F4F760
:1088F0008FFB02F03BFE201A20EAE070F8BD00BFBB
:10890000304B0220644B02203BB301002DE9F843B9
:1089100004464FF02003EFF3118983F31188BFF36E
:108920006F8F02F08AFC4EB2804660B3174D21462D
:1089300005F128073846FFF7A1FDAB6AA673BB42D5
:108940002A4619D0C3B1E96A93F90E00B0420EDD90
:108950005A68C4E9003214605C600120FFF7A4FD8E
:1089600089F31188BFF36F8F4046BDE8F8839942C1
:1089700002D01B68002BE7D1D36A27606360D36AFB
:108980001C60D462E9E7A673EAE700BF304B02201F
:108990000021044B084603F12802C3E90A22FFF72D
:1089A0002DBD00BF304B0220F8B5234C234BA268ED
:1089B0009A4229D04FF02003EFF3118683F31188F8
:1089C000BFF36F8F04F12805A1682846FFF756FD15
:1089D000A26AA368AA4228D03AB3E06A93F90E10BB
:1089E00092F90E708F421BDD5168C3E900210B60C4
:1089F00053605A7B012062F07F025A73FFF754FDE7
:108A000086F31188BFF36F8F4FF02003EFF31180CF
:108A100083F31188BFF36F8FBDE8F840F4F7F8BA1D
:108A2000824202D01268002ADAD1E26A1D605A60DE
:108A3000E26A1360E362DCE7304B02206C450220FF
:108A400038B5431C044605D1104B986800F04AF92C
:108A5000204638BD4FF4004540F2E73000214FF486
:108A60007A72E5FB04010023F3F7E8FB044648B9FA
:108A7000FFF79AFF4FF47A7084FB0001C40B44EABD
:108A80004144E5E7FFF714FF0446F3E7304B0220CB
:108A9000014B9868704700BF304B022070B5044608
:108AA0004FF02003EFF3118683F31188BFF36F8F2C
:108AB00002F076FC054678B1437BDB0603D183697F
:108AC0000BB9FFF72BFD0023C5F888303146BDE810
:108AD0007040074802F0ECBBD4E902329A4218BF5A
:108AE00001330221A36004F1100002F077FEEDE7EC
:108AF0008354022010B402460B464FF02000EFF3DF
:108B0000118180F31188BFF36F8F94684CB1013CE1
:108B1000946081F31188BFF36F8F00205DF8044BE0
:108B2000704733B981F31188BFF36F8F6FF00F0077
:108B3000F4E702485DF8044BFFF7A6BE8354022019
:108B400038B50D4613464FF02002EFF3118182F342
:108B50001188BFF36F8FD0E9022494420AD9231FF2
:108B6000C36054F8043C2B6081F31188BFF36F8F0E
:108B7000002006E033B981F31188BFF36F8F6FF0E7
:108B80000F0038BD02460830FFF77EFE10F10B0FD4
:108B9000F7D0024B9B685B692B60E9E7304B022002
:108BA00010B5084C4FF0FF334FF480620649204661
:108BB00000F012F9054904F1100000F009F8002056
:108BC00010BD00BF704B0220087B02205FC1010076
:108BD00010B5044608B9054B9C68202204F15400E6
:108BE00001F09BF9002084F8730010BD304B022087
:108BF00010B54FF02002EFF3118482F31188BFF318
:108C00006F8F427B510704D484F31188BFF36F8FB9
:108C100010BD22F0040112F01B0F417303D18369D0
:108C20000BB9FFF77BFC2146BDE81040014802F07C
:108C30003FBB00BF8354022070B586B0DDE90E65EE
:108C400004960D9E044603960C9E02960B9E01967A
:108C50000A9E0096F4F72EFA45B11F22294604F128
:108C6000540001F05AF9002384F87330044B9B68D8
:108C70000BB1D3F88030C4F8803006B070BD00BFAF
:108C8000304B022070B5002686B005960E9E0F9DD3
:108C900004960D9E044603960C9E02960B9E01962A
:108CA0000A9E0096FFF7C8FF6B1C03D02DB9204623
:108CB000FFF79EFF204606B070BD4FF4004640F21D
:108CC000E73000214FF47A720023E6FB0501F3F749
:108CD000B5FA0349421C04F1180000F0DBF8E9E79B
:108CE0003BB3010038B505464FF02003EFF3118484
:108CF00083F31188BFF36F8FFFF7C0FC074B9B68AE
:108D0000AB4205D12146BDE83840054802F0D0BA53
:108D100084F31188BFF36F8F38BD00BF304B022042
:108D2000835402202DE9F04F284E294DB04687B0DC
:108D3000B54205F1300410D3FFF78CFB4FF4004926
:108D400040F2E7360027224CDFF888A0444521D3C3
:108D500007B0BDE8F04FFFF7C5BB54F8043C0593DE
:108D600054F8103C049354F8143C039354F8183C02
:108D7000029354F81C3C019354F8203C009354E9AE
:108D80000A2354E90C01FFF757FF54F8303CDD6427
:108D90002546CDE7616A4B1C04D0256821B92846D9
:108DA000FFF726FF3034D1E7B346BC46E9FB01BCF0
:108DB0004FF47A72002358466146F3F73FFA514662
:108DC000421C05F1180000F065F8EBE7D0A0022086
:108DD00010A002203BB301002DE9F041054686B00A
:108DE0000E461746984602F0B6F905F11004002029
:108DF000094BCDE90400CDE90208CDE900503A461F
:108E000031462046FFF73EFF2046044906B0BDE844
:108E1000F041FFF7DDBE00BFD199010068C101003C
:108E2000034B1B680BB9F3F7C3BF0020704700BFAB
:108E3000504C0220036840B1074A5268904204D067
:108E40001BB19A6881680A449A60426813605A604C
:108E50000023C0E900337047149F02200B4B10B56C
:108E60001C689C4208BF0024FFF7DAFF54B1A368D6
:108E7000181A20EAE070064B1B6913B19842A8BF8C
:108E8000184610BD6FF00040F5E700BF149F0220A8
:108E9000304B022070B504461646C1604FF02003E7
:108EA000EFF3118583F31188BFF36F8FFFF7B8FFDE
:108EB000012EACBF80190130164BA0601A689A428F
:108EC00001D05E6832B95A68236062605A681460E3
:108ED0005C600AE09068A168884215DD411A9160E3
:108EE0005168C4E900210C6054601A689A4206D0A7
:108EF000944204D1FFF7B2FF0021F3F703FF85F39B
:108F00001188BFF36F8F70BD091A9642A160DAD045
:108F10001268D7E7149F02202DE9F04B0446FFF7B3
:108F200077FB4FF02003EFF3118583F31188BFF334
:108F30006F8F214F214EB846DFF884903460D9F806
